:100000000C945D4B0C94DF4B0C94DF4B0C94DF4B4A
:100010000C94DF4B0C94DF4B0C94DF4B0C94DF4BB8
:100020000C94DF4B0C94DF4B0C94DF4B0C94DF4BA8
:100030000C94DF4B0C94FF5D0C94DF4B0C94DF4B66
:100040000C94DF4B0C94DF4B0C94DF4B0C94DF4B88
:100050000C94DF4B0C94DF4B0C94DF4B0C94DF4B78
:100060000C94DF4B0C94DF4B0C94DF4B0C94DF4B68
:100070000000000000000000000000000000000080
:100080000000000000000000000000000000000070
:100090000000000000000000000000000000000060
:1000A0000000000000000000000000000000000050
:1000B0000000000000000000000000000000000040
:1000C00000000049000000495252000052525C2DCD
:1000D0000000000000000000000000000000000020
:1000E0000040000000494A52004952525B1C5253E2
:1000F0001C25241B2425251B0A0A2D1C12120A0A62
:100100000000000000000000404949494949525B95
:100110005B5B525B1C1C1312241C12090909120997
:100120000909090A0A0A0A0A0A13120A0A12130A10
:100130000000000000009252525252521312130952
:10014000001C0A1212401B65090A0009241B120038
:1001500000251C1C010025241C1C0024252424240B
:100160000000000000005249494000001B135249A2
:100170004900641C1C5B4A481C651C2552491C1C18
:10018000652464491C1C652564491C1C6D2E5C4952
:100190000000000000000000000000490000000016
:1001A000535200000053522500004A5225250000FA
:1001B0005B251300005B53000A1C095B1C657F373D
:1001C0004052522E2E1C525C2E251B1324251C1C23
:1001D00012002525120000121B0000132E37001BF1
:1001E00037372E2E37372E2E2E2E2E2E6E6E6E1C5D
:1001F0001313120009131200001213130012251C0E
:1002000013132E371C131313361C131B1B1B251320
:100210001C1C1B1B1B1C1C1C1C1C1C1C1C1C1C132A
:100220001312121313001313131C000913131C01D0
:100230000037131C13002E2E1C1C001C772E2500CB
:10024000137F251C010A37241C1C0A2E25250900B2
:10025000132E242525252E252525252525252D2E3E
:10026000251B2E2E251C1325251C1C1C1C011C1CAB
:100270001300011C0A000165775C016E7F6E521B42
:1002800025256D1C524925251C1353001C1C1C528E
:100290004A001B135B5B000009525C0000005B5CC2
:1002A000000000001B000000000000000000000033
:1002B000135B7F776E6E136577766E6E1B65777650
:1002C00076761B5BBF76B67609136DBFB7B6001B9B
:1002D000125C76BF0000121B125B00000000090ACE
:1002E0006E6E6E77241C6E6E77251C1C6E776E1CEE
:1002F0001C1C76761C1C2425B765646D6D1B766D01
:100300006D5B09125B5C5B125B641213131B1212B0
:100310001C1C1C1C1C241C1C242525242425251BDA
:1003200000002513000064BF00096EBFBF6D6EBFE3
:100330006D5B12135B12131209000901000000002B
:100340002E1C0900096E010009767F7F12777F7FDE
:100350006412BF775B121B095B121B0900001B09AB
:10036000000000000000000000000000000000008D
:100370007F7F5313130064121B0100001B12000047
:10038000000000000000000000000000000000006D
:10039000000000000000000000000000000000005D
:1003A0000000000000002600000026002F000000D2
:1003B0002F00370000003700FF000000FF00BF00E3
:1003C0000000BF00370000370000002626000000B4
:1003D000000000000000262626262600000000005F
:1003E0002F000000003700000000FF00000000BFE9
:1003F0000000000037000000000026262626260008
:100400000000000000002626262626002F000000FF
:100410000000370000000000FFFFFFFF0000BF00EA
:1004200000000000370000000000262626262600D7
:100430000000000000002626262600002F000000F5
:100440002F00370000003700FFFFFFFF0000BF0054
:100450000000BF00370000003700262626260000D7
:10046000000000000000000026262600002F0000EB
:100470002F00370000003700FF000000FF00BF0022
:100480000000BF00370000370000262626000000CD
:100490000000000000002600000026002F000000E1
:1004A0002F000037003700000000FF00000000BFF1
:1004B00000BF0000370000003700260000002600C3
:1004C000000000000000000000000000000000002C
:1004D000000000000000000000000000000000001C
:1004E0000000009B000000529BA400005B9B6D7706
:1004F00000000000000000000000000000000000FC
:10050000005B000000E4F6FF099BEDF6FFBFA4AD21
:10051000BFBFBFBF767F7FB7B7BF7F766EB7B7BFAE
:1005200000000000000000005BB6F6F6F6FFFFFFDB
:10053000FFBFFFFFFFBFBFAEFFFFFFB7AD65FFFF10
:10054000B7B6AD65FFFFBFB7AE6EFFFFBFB7B7650C
:10055000000000000000F6F6EDEDADA4B66D6D5C98
:10056000526E6565655265765C5C52536E246552C9
:10057000526E25255B52772D2525526E6E2D252531
:10058000000000000000A49B9B4900006564A49B40
:1005900092006D2525649349656E652E9B52242536
:1005A0006D25655225246D2D655225256E2E6452CC
:1005B00000000000000000000000004A00000000F1
:1005C0005B9B0000005B5B2D0000525B2E2E000148
:1005D0005B2D1C01005C5B014A654A5B1C6E7F77EA
:1005E000495B9B77776D5B65776E65656D2D25251E
:1005F0005C522E25130949641C09095C7F7F091C84
:100600007F7F777F777F77777F7F7776777F7F6E44
:10061000656E6EA4B6FF655BA4B7BFFF526DBFBF2A
:10062000BFFF7FBFBFBFBFFFBFBFB7BFFFFF7FB76A
:10063000BFBFFFFF6EB7BFBFFFFF77BFBFBFFFFFEB
:10064000FFFFBFBFB75BFFFFBFBFA464FFFFBFAD2E
:10065000A47FFFFFBFA4BF7FFFBFADBFBFBFFFB67B
:10066000BFBFBF77F7BFBFBF7777FFBFBFBF6452C2
:100670006D7F6E2E2D2D7F766E6E6E2E7777777650
:100680002E1C7F776E251C25776525251C096E6E2F
:100690001C0949255B494A6E7F645377BF775B5CD1
:1006A000256E6E255B4A25651C1B5B002524245B9B
:1006B00053001C1B5B5C00000A5B64000000646468
:1006C000000000005C0000000000000000000000CE
:1006D0005B5C7FBF77765C6D7FB777775C6D7FBF44
:1006E00077775C64BFBFBFBF0A5C6EBFBFBF0065EA
:1006F000646DBFBF00005B6D646D00000000125BA5
:100700007777777F6E6E77777F766D7677BF776D49
:100710006E76BF7F6D6E767FBF7676BFBF76BFBFCA
:10072000BFB664ADADB6B6ADBFFF646DADB6AD647A
:1007300077BFBFBFFFFF77BFBFBFFFFF7FBFBFBF99
:10074000FFF6BFB7ADF6FFFFA4ADFFFFFFFFFFFF52
:10075000FFFFFFFFFFFFFFF6A4005B520000000059
:10076000BFBFAD5B64BFB6ADADBFFFBFFFFFFFFF57
:10077000BF64FFFFBFB6765BFFBFBF5B0000FF5CDF
:100780000000000000000000000000000000000069
:10079000BFBF645C5C006E5C654900006D5B00007F
:1007A0000000000000000000000000000000000049
:1007B0000000000000000000000000000000000039
:1007C0000600040000000100020003000400050010
:1007D00006000700080009000A000B000C000D00CD
:1007E0000E000F0010000000110012001300140092
:1007F000150016000600030000001700180019007D
:100800001A001B001C001D001E001F0020002100FC
:10081000220023002400250026000000000208001A
:10082000085504085A0000F8000990000A1E320515
:100830000000FF0000001C0800000000374C454C81
:10084000234DAA509650484C574C664C7E50744CE1
:10085000824C0000000100020003000400050100BA
:10086000010101020103010401050200020102026B
:10087000020302040205030003010302030303044D
:100880000305040004010402040304040405050034
:10089000050105020503050405050600060106021B
:1008A00006030604060507000701070207030704FD
:1008B00007050800080108020803080408050900E4
:1008C000090109020903090409050A000A010A02CB
:1008D0000A030A040A050B000B010B020B030B04AD
:1008E0000B050C000C010C020C030C040C050D0094
:1008F0000D010D020D030D040D050E000E010E027B
:100900000E030E040E050F000F010F020F030F045C
:100910000F05100010011002100310041005110043
:10092000110111021103110411051200120112022A
:10093000120312041205130013011302130313040C
:1009400013051400140114021403140414051500F3
:1009500015011502150315041505160016011602DA
:1009600016031604160517001701170217031704BC
:1009700017051800180118021803180418051900A3
:10098000190119021903190419051A001A011A028A
:100990001A031A041A051B001B011B021B031B046C
:1009A0001B051C001C011C021C031C041C051D0053
:1009B0001D011D021D031D041D051E001E011E023A
:1009C0001E031E041E051F001F011F021F031F041C
:1009D0001F050300010101010000000000000000EC
:1009E0000000000001000001010000010000000003
:1009F00000000000000000010101010000000000F3
:100A000000000001000001010000010000000000E2
:100A100000000003020000020202000000000000CB
:100A200000000000000202000200000200000000BE
:100A300000000000000000020202000002000000AE
:100A4000000000000002000002000202000000009E
:100A50000000000003000003030303000000000087
:100A6000000000000000030000030000030300007A
:100A7000000000000000000003030303000000006A
:100A8000000000000003030000030000030000005A
:100A90000000000000020404040400000000000044
:100AA0000000000000000404040400000000000036
:100AB0000000000000000404040400000000000026
:100AC0000000000000000404040400000000000016
:100AD00000000000000003000500050505000000FF
:100AE00000000000000000000500000505000500F2
:100AF00000000000000000000000050505000500E2
:100B000000000000000000000500050500000500D1
:100B100000000000000000040000000006060606B9
:100B200000000000000000000000060000000600B9
:100B300000000600000006000000000000000000A9
:100B40000606060600000000000600000006000081
:100B5000000600000006000003070700000707006A
:100B60000000000000000000000000070007070070
:100B70000700000000000000000000000707000060
:100B8000070700000000000000000700070700073B
:100B90000000000000000000003230303820414CDE
:100BA000454320424F555251554500485454503A00
:100BB0002F2F5757572E42454C4F4749432E434FEF
:100BC0004D2F555A45424F58004C4943454E4345D9
:100BD0004420554E44455220474E552047504C2006
:100BE0005633003120504C41594552003220504C70
:100BF0004159455200565320435055004F505449D7
:100C00004F4E530047414D45204F56455221005904
:100C10004F552057494E2100594F55204C4F5345B1
:100C20002121005052455353005354415254004720
:100C3000414D45204F5054494F4E5300534F4E475E
:100C40003A004241434B20544F204D454E55004DF4
:100C5000454E5500504C41590047484F535420428F
:100C60004C4F434B3A00594553004E4F200000FF74
:100C700006015300C00000904C6B00C20000922897
:100C80006B00C1000091476B1792346B1890476B53
:100C90000092286B0091446B1890486B0092346B63
:100CA0000091456B18904A6B0092286B0091476B3E
:100CB00018904C6B0092346B0091446B0C904A6B13
:100CC0000C486B0092286B0091456B1890476B00A5
:100CD00092346B0091446B1890456B00922D6B0021
:100CE00091406B1892396B1890456B00922D6B00F8
:100CF00091406B1890486B0092396B0091456B18CE
:100D0000904C6B00922D6B0091486B1892396B18C8
:100D1000904A6B00922D6B0091476B1890486B00C6
:100D200092396B0091456B1890476B00922C6B00C9
:100D300091446B1892386B1890476B00922C6B00A3
:100D400091446B1890486B0092386B0091456B187A
:100D5000904A6B0092286B0091476B1892346B1885
:100D6000904C6B0092286B0091476B1892346B1873
:100D700090486B00922D6B0091456B1892396B185F
:100D800090456B00922D6B0091406B1892396B1857
:100D900090456B00922D6B0091406B1892396B1847
:100DA0002D6B00912F6B1892306B0091396B18925C
:100DB000266B0091326B18904A6B0092326B009157
:100DC000456B1892266B18904D6B0092326B009118
:100DD0004A6B1890516B0092266B00914D6B1892E4
:100DE000326B18904F6B0092266B00914C6B1890F1
:100DF0004D6B0092326B00914A6B18904C6B0092D5
:100E00002D6B0091486B1892396B182D6B18904818
:100E10006B0092396B0091456B18904C6B00922DD2
:100E20006B0091456B1892396B18904A6B00922DAC
:100E30006B0091476B1890486B0092396B0091459D
:100E40006B1890476B00922C6B0091446B18923892
:100E50006B1890476B00922C6B0091446B18904874
:100E60006B0092386B0091456B18904A6B0092288A
:100E70006B0091476B1892346B18904C6B00922862
:100E80006B0091476B1892346B1890486B00922D51
:100E90006B0091456B1892396B1890456B00922D41
:100EA0006B0091406B1892396B1890456B00922D36
:100EB0006B0091406B1892396B182D6B18396B18B9
:100EC000904C6B0092286B0091476B1892346B1713
:100ED00090476B0092286B0091446B1890486B0010
:100EE00092346B0091456B18904A6B0092286B000E
:100EF00091476B18904C6B0092346B0091446B0CD3
:100F0000904A6B0C486B0092286B0091456B1890CF
:100F1000476B0092346B0091446B1890456B0092C4
:100F20002D6B0091406B1892396B1890456B0092B5
:100F30002D6B0091406B1890486B0092396B0091BB
:100F4000456B18904C6B00922D6B0091486B18927A
:100F5000396B18904A6B00922D6B0091476B18907B
:100F6000486B0092396B0091456B1890476B00926B
:100F70002C6B0091446B1892386B1890476B009261
:100F80002C6B0091446B1890486B0092386B009169
:100F9000456B18904A6B0092286B0091476B189232
:100FA000346B18904C6B0092286B0091476B189231
:100FB000346B1890486B00922D6B0091456B189222
:100FC000396B1890456B00922D6B0091406B189215
:100FD000396B1890456B00922D6B0091406B189205
:100FE000396B182D6B00912F6B1892306B00913973
:100FF0006B1892266B0091326B18904A6B009232FC
:101000006B0091456B1892266B18904D6B009232D5
:101010006B00914A6B1890516B0092266B00914DBA
:101020006B1892326B18904F6B0092266B00914CAC
:101030006B18904D6B0092326B00914A6B18904C7C
:101040006B00922D6B0091486B1892396B182D6BC9
:101050001890486B0092396B0091456B18904C6B5F
:1010600000922D6B0091456B1892396B18904A6B6A
:1010700000922D6B0091476B1890486B0092396B72
:101080000091456B1890476B00922C6B0091446B5C
:101090001892386B1890476B00922C6B0091446B40
:1010A0001890486B0092386B0091456B18904A6B12
:1010B0000092286B0091476B1892346B18904C6B20
:1010C0000092286B0091476B1892346B1890486B14
:1010D00000922D6B0091456B1892396B1890456BFF
:1010E00000922D6B0091406B1892396B1890456BF4
:1010F00000922D6B0091406B1892396B182D6B1874
:10110000396B1890406B00922D6B00913C6B1892DC
:10111000346B182D6B17346B18903C6B00922D6B51
:101120000091396B1892346B182D6B18346B189032
:101130003E6B00922C6B0091386B1892346B182C1C
:101140006B18346B18903B6B00922C6B0091386BD2
:101150001892346B182C6B18346B18903C6B0092FF
:101160002D6B0091396B1892346B182D6B18346B02
:10117000182D6B0091396B1892346B182D6B183445
:101180006B182C6B0091386B1892346B182C6B1801
:10119000346B182C6B18346B182C6B18346B18903C
:1011A000406B00922D6B00913C6B1892346B182DA4
:1011B0006B18346B18903C6B00922D6B0091396B5F
:1011C0001892346B182D6B18346B18903E6B00928C
:1011D0002C6B0091386B1892346B182C6B18346B95
:1011E00018903B6B00922C6B0091386B1892346B0B
:1011F000182C6B18346B18903C6B00922D6B00917F
:10120000396B1892346B1890406B00922D6B0091E3
:101210003C6B1892346B1890456B00922D6B0091CB
:10122000406B1892346B1890456B00922D6B1834FC
:101230006B1890446B00922C6B0091406B189234A9
:101240006B182C6B18346B182C6B18346B182C6BB8
:1012500018346B18FF06014500FF2F0000C0110075
:10126000C10300C20B0092326900C30700930D3224
:1012700001903E7F169232690093073E02903E7FB6
:101280000A9232690093073E03903E7F0A922D69CD
:101290000093073E0290397F16922D690093073E16
:1012A0000290397F1692326900930D3202903E7F90
:1012B000179232690093073E02903E7F0A9232698C
:1012C0000093073E01903E7F0A922D690093073EEE
:1012D0000390397F16922D690093073E0390397F62
:1012E0001692326900930D3201903E7F1792326957
:1012F0000093073E02903E7F0A9232690093073EB8
:1013000003903E7F0A922D690093073E0190397F3A
:1013100016922D690093073E0390397F1692326929
:1013200000930D3202903E7F169232690093073E81
:1013300002903E7F0A9232690093073E02903E7F00
:101340000B922D6900930D320290397F16922D6910
:1013500000930D370290397F16FF06015300923239
:101360006900930D3C02903E7F0091395D179232E7
:10137000690093073E0290457F0091415D0A9232D9
:10138000690093073E0C922D690093073E01904A35
:101390007F0091415D17922D690093073E029049AD
:1013A0007F0091435D179232690093073E02904A95
:1013B0007F0091415D159232690093073E0390458D
:1013C0007F0091405D0A9232690093073E0290458A
:1013D0007F0091415D0A922D690093073E0390467C
:1013E0007F0091435D16922D690093073E01904363
:1013F0007F0091405D179232690093073E0290454D
:101400007F0091415D179232690093073E01904140
:101410007F00913D5D0A9232690093073E02904140
:101420007F00913E5D0A922D690093073E03904331
:101430007F0091405D16922D690093073E02904017
:101440007F00913D5D169232690093073E02904104
:101450007F00913E5D179232690093073E02903EF5
:101460007F0091385D0A9232690093073E02903EF8
:101470007F0091395D0A922D690093073E029040EA
:101480007F00913D5D16922D690093073E02903DCD
:101490007F0091395D179232690093073E02903EBA
:1014A0007F0091395D169232690093073E019039B1
:1014B0007F0091355D0B9232690093073E0C9231AB
:1014C000690093073E02903A7F0091375D17922D95
:1014D000690093073E02903D7F0091375D1592327F
:1014E000690093073E03903E7F0091395D1692326A
:1014F000690093073E0390397F0091355D0A92326F
:10150000690093073E0C9231690093073E01903ABF
:101510007F0091375D17922D690093073E0290403E
:101520007F00913D5D179232690093073E01903E26
:101530007F0091395D169232690093073E03904512
:101540007F0091415D0A9232690093073E0C922D13
:10155000690093073E02904A7F0091415D16922DEB
:10156000690093073E0290497F0091435D179232D4
:10157000690093073E02904A7F0091415D169232C6
:10158000690093073E0290457F0091405D0A9232C8
:10159000690093073E0290457F0091415D0A922DBC
:1015A000690093073E0290467F0091435D17922D9C
:1015B000690093073E0290437F0091405D1692328E
:1015C000690093073E0190457F0091415D1792327B
:1015D000690093073E0290417F00913D5D0A92327F
:1015E000690093073E0390417F00913E5D0A922D72
:1015F000690093073E0290437F0091405D15922D54
:10160000690093073E0390407F00913D5D16923242
:10161000690093073E0390417F00913E5D15923231
:10162000690093073E02903E7F0091385D0A923236
:10163000690093073E03903E7F0091395D0A922D29
:10164000690093073E0290407F00913D5D17922D07
:10165000690093073E01903D7F0091395D169232FB
:10166000690093073E02903E7F0091395D179232E8
:10167000690093073E0290397F0091355D0A9232EE
:10168000690093073E0C9231690093073E02903A3D
:101690007F0091375D16922D690093073E02903DC1
:1016A0007F0091375D179232690093073E02903EAA
:1016B0007F0091395D169232690093073E0290399E
:1016C0007F0091355D0A9232690093073E0C92319A
:1016D000690093073E03903A7F0091375D16922D83
:1016E000690093073E0190407F00913D5D17923263
:1016F000690093073E02903E7F0091395D17923258
:10170000690093073E0C9232690093073E0B922EBC
:10171000690093073E19922B690093073E18923295
:10172000690093073E199232690093073E0C92328A
:10173000690093073E0D9231690093073E01904086
:101740007F0091395D16922D690093073E02903D0E
:101750007F0091395D179232690093073E02903EF7
:101760007F0091395D169232690093073E0C9232E8
:10177000690093073E0C922E690093073E19922B45
:10178000690093073E189232690093073E1892321F
:10179000690093073E0D9232690093073E0C922B2D
:1017A000690093073E0190407F00913C5D179224B1
:1017B000691929690093073E0190417F16923569A6
:1017C0000093073E0390417F0A9229690093073EE8
:1017D0000290417F0A9224690093073E0390437F61
:1017E000159230690093073E0290407F1792296955
:1017F0000093073E0290417F179235690093073EA0
:101800000190417F0A9229690093073E0290417F2F
:101810000A9224690093073E0290437F1792306931
:101820000093073E0290407F169229690093073E7D
:101830000290417F169235690093073E0D92296907
:101840000093073E0C9224690093073E189230697A
:101850000093073E189229690093073E1992356953
:101860000093073E0B9229690093073E0D9224696D
:101870000093073E0290437F0091405D17923069CC
:101880000093073E179229690093073E0390457F16
:101890000091415D169235690093073E0390457FA4
:1018A0000091415D0A9229690093073E0190457FAE
:1018B0000091415D0A9224690093073E0290467FA1
:1018C0000091435D179230690093073E0290437F79
:1018D0000091405D169229690093073E0290457F72
:1018E0000091415D169235690093073E0290457F55
:1018F0000091415D0A9229690093073E0390457F5C
:101900000091415D0A9224690093073E0290467F50
:101910000091435D169230690093073E0290437F29
:101920000091405D169229690093073E0290457F21
:1019300000913C5D179235690093073E0C9229692E
:101940000093073E0B9224690093073E1992306979
:101950000093073E199229690093073E1892356952
:101960000093073E0C9229690093073E0D922B6964
:101970000093073E0190477F00913E5D16923769C4
:101980000093073E199224690093073E0290487F16
:101990000091405D169230690093073E0290487FA7
:1019A0000091415D0A9224690093073E0290487FAE
:1019B0000091435D0B9224690093073E0290487F9B
:1019C0000091405D169230690093073E0290487F77
:1019D0000091435D169229690093073E02904A7F69
:1019E0000091455D179235690093073E0290487F4C
:1019F0000091455D0A9229690093073E0C9229697E
:101A00000093073E0190487F0091455D179235692C
:101A10000093073E0290477F00913E5D1792246934
:101A20000093073E0290487F0091405D1592306917
:101A30000093073E0390487F0091415D0A9224691C
:101A40000093073E0290487F0091435D0A9224690B
:101A50000093073E0390487F0091405D16923069E5
:101A60000093073E0190487F0091435D17922969DA
:101A70000093073E02904A7F0091445D17923569BA
:101A80000093073E0190487F0091445D0A922969C6
:101A90000093073E0C9229690093073E0390487F0C
:101AA0000091445D169235690093073E0290477F8E
:101AB00000913E5D169224690093073E0290487F94
:101AC0000091405D179230690093073E0290487F75
:101AD0000091415D0A9224690093073E0290487F7D
:101AE0000091435D0A9224690093073E0290487F6B
:101AF0000091405D169230690093073E0290487F46
:101B00000091435D179224690093073E0290477F3E
:101B100000913E5D169230690093073E0190477F29
:101B20000091405D0B9224690093073E0290477F2D
:101B30000091415D0A9224690093073E0290477F1D
:101B400000913E5D179230690093073E0290477FF7
:101B50000091415D159224690093073E0390467FF2
:101B600000913E5D169230690093073E0390467FD8
:101B70000091405D0A9224690093073E0190467FE0
:101B80000091415D0B9224690093073E0190467FCE
:101B90000091405D179230690093073E0290437FA9
:101BA0000091405D179224690093073E0190407FA9
:101BB0000091375D169230690093073E0390417F94
:101BC00000913E5D0A9224690093073E0C922469BD
:101BD0000093073E0290437F0091405D169230696A
:101BE0000093073E02903C7F0091345D1792266976
:101BF0000093073E0290437F0091395D169232694F
:101C00000093073E0290417F0091395D0A92266958
:101C10000093073E0290417F0091395D0A92266948
:101C20000093073E02903C7F0091395D1792326924
:101C30000093073E0290417F0091395D169226691C
:101C40001832690093073E02903C7F0091395D0A8B
:101C50009226690093073E03903E7F00913B5D0A08
:101C60009226690093073E02903C7F0091395D15F2
:101C70009232690093073E0390397F0091355D16DB
:101C80009226690093073E0390437F0091385D15CB
:101C90009232690093073E0290417F0091385D0ABD
:101CA0009226690093073E0390417F0091385D0AB8
:101CB0009226690093073E02903C7F0091385D17A1
:101CC0009232690093073E0190417F0091385D1682
:101CD0009226691932690093073E02903C7F009179
:101CE000385D0A9226690093073E02903E7F00917C
:101CF0003A5D0A9226690093073E02903C7F00916C
:101D0000385D169232690093073E0290387F009149
:101D1000355D179224690093073E02903C7F009145
:101D2000345D169230690093073E0C92246900934B
:101D3000073E0C9224690093073E19923069009384
:101D4000073E189224690093073E19923069009368
:101D5000073E0C9224690093073E0B92246900937E
:101D6000073E199230690093073E18922469009348
:101D7000073E199230690093073E0C922469009344
:101D8000073E0D9224690093073E17923069009335
:101D9000073E199224690093073E18923069009318
:101DA000073E0C9224690093073E0C92346900931D
:101DB000073E02903D7F0091375D2F92326900937C
:101DC000073E02903E7F169232690093073E0390D1
:101DD0003E7F0A9232690093073E02903E7F0A924C
:101DE0002D690093073E0190397F17922D6900936A
:101DF000073E0290397F179232690093073E0190A7
:101E00003E7F169232690093073E03903E7F0A920E
:101E100032690093073E02903E7F0A922D6900933B
:101E2000073E0390397F15922D690093073E02907B
:101E3000397F179232690093073E02903E7F1792D6
:101E400032690093073E01903E7F0A923269009307
:101E5000073E02903E7F0A922D690093073E029052
:101E6000397F17922D690093073E0290397F1692B1
:101E700032690093073E02903E7F169232690093CA
:101E8000073E02903E7F0B9232690093073E02901C
:101E90003E7F0A922D690093073E0290397F169289
:101EA0002D690093073E0290397F16FF0601450019
:101EB0009232690093073E03903E7F0091395D1690
:101EC0009232690093073E0190457F0091415D0A7F
:101ED0009232690093073E0D922D690093073E02EE
:101EE000904A7F0091415D17922D690093073E0152
:101EF00090497F0091435D169232690093073E033B
:101F0000904A7F0091415D169232690093073E032B
:101F100090457F0091405D0A9232690093073E012F
:101F200090457F0091415D0A922D690093073E0222
:101F300090467F0091435D17922D690093073E0202
:101F400090437F0091405D169232690093073E02F4
:101F500090457F0091415D169232690093073E02E1
:101F600090417F00913D5D0A9232690093073E03E4
:101F700090417F00913E5D0A922D690093073E02D9
:101F800090437F0091405D16922D690093073E02B9
:101F900090407F00913D5D169232690093073E02AA
:101FA00090417F00913E5D179232690093073E0297
:101FB000903E7F0091385D0A9232690093073E019E
:101FC000903E7F0091395D0A922D690093073E0390
:101FD00090407F00913D5D16922D690093073E036E
:101FE000903D7F0091395D169232690093073E0162
:101FF000903E7F0091395D179232690093073E024F
:1020000090397F0091355D0A9232690093073E0D49
:102010009231690093073E01903A7F0091375D1637
:10202000922D690093073E03903D7F0091375D1626
:102030009232690093073E02903E7F0091395D160F
:102040009232690093073E0290397F0091355D0A14
:102050009232690093073E0D9231690093073E0268
:10206000903A7F0091375D16922D690093073E02EA
:1020700090407F00913D5D169232690093073E02C9
:10208000903E7F0091395D179232690093073E02BE
:1020900090457F0091415D0A9232690093073E0CA2
:1020A000922D690093073E01904A7F0091415D1790
:1020B000922D690093073E0290497F0091435D177E
:1020C0009232690093073E02904A7F0091415D156C
:1020D0009232690093073E0390457F0091405D0A6C
:1020E0009232690093073E0290457F0091415D0A5C
:1020F000922D690093073E0390467F0091435D1641
:10210000922D690093073E0190437F0091405D1737
:102110009232690093073E0290457F0091415D171E
:102120009232690093073E0190417F00913D5D0A24
:102130009232690093073E0290417F00913E5D0A12
:10214000922D690093073E0390437F0091405D16F6
:10215000922D690093073E0290407F00913D5D16ED
:102160009232690093073E0290417F00913E5D17D5
:102170009232690093073E02903E7F0091385D0ADB
:102180009232690093073E02903E7F0091395D0ACA
:10219000922D690093073E0290407F00913D5D16AD
:1021A000922D690093073E02903D7F0091395D17A3
:1021B0009232690093073E02903E7F0091395D168E
:1021C0009232690093073E0190397F0091355D0B93
:1021D0009232690093073E0C9231690093073E02E8
:1021E000903A7F0091375D17922D690093073E0268
:1021F000903D7F0091375D159232690093073E0351
:10220000903E7F0091395D169232690093073E033C
:1022100090397F0091355D0A9232690093073E0C38
:102220009231690093073E01903A7F0091375D1724
:10223000922D690093073E0290407F00913D5D170B
:102240009232690093073E01903E7F0091395D16FE
:102250009232690093073E0D9232690093073E0C5B
:10226000922E690093073E18922B690093073E193E
:102270009232690093073E189232690093073E0C30
:102280009232690093073E0C9231690093073E0237
:1022900090407F0091395D16922D690093073E03AF
:1022A000903D7F0091395D169232690093073E019F
:1022B000903E7F0091395D179232690093073E0C82
:1022C0009232690093073E0D922E690093073E17E4
:1022D000922B690093073E199232690093073E18CA
:1022E0009232690093073E0C9232690093073E0DCB
:1022F000922B690093073E0290407F00913C5D174E
:102300009224691729690093073E0290417F179232
:1023100035690093073E0290417F0A922969009334
:10232000073E0290417F0A9224690093073E029083
:10233000437F169230690093073E0290407F1792C8
:1023400029690093073E0290417F169235690093F8
:10235000073E0290417F0A9229690093073E02904E
:10236000417F0A9224690093073E0390437F1692AF
:1023700030690093073E0190407F179229690093CE
:10238000073E0290417F179235690093073E0C92F9
:1023900029690093073E0B9224690093073E199226
:1023A00030690093073E189229690093073E1992FD
:1023B00035690093073E0C9229690093073E0D9200
:1023C00024690093073E0190437F16923069009381
:1023D000073E199229690093073E0290457F1692A5
:1023E00035690093073E0290457F0A922969009360
:1023F000073E0290457F0A9224690093073E0290AF
:10240000467F179230690093073E0290437F1692F1
:1024100029690093073E0290457F16923569009323
:10242000073E0390457F0A9229690093073E029078
:10243000457F0A9224690093073E0190467F1792D8
:1024400030690093073E0290437F14FF2F0000C0C5
:102450000300C10C00C20C009239310093074B02FB
:1024600090486800914151179239310093074B020F
:10247000904868009141510B923B310093074B0209
:10248000904A680091435124923C310093074B02DB
:10249000904D68009145510B923C310093074B02DF
:1024A000904C68009143510B9237310093074B02D7
:1024B000904868009140510B923B310093074B02CA
:1024C000904A680091435124923C310093074B029B
:1024D000904D68009145510B923E310093074B029D
:1024E000904F68009146510B923F310093074B0289
:1024F000905068009148510B9242310093074B0273
:1025000090516800914A510493074B06074B070707
:102510004B06074B07074B0C07370D07370D0737DF
:102520000D073718FF2F000000000000000000001A
:10253000000000000000000000000000000000009B
:10254000000000000000000000000000000000008B
:10255000000000000000000000FF00000000FFFF7E
:10256000FF000000FFFFFF00000000FF0000000070
:1025700000FF0000000000000000000000FF00005D
:1025800000000000000000FFFF00FFFF00FFFF0051
:10259000FFFF00FF0000FF0000000000000000003F
:1025A000000000000000000000000000000000002B
:1025B0000000000000000000000000000000FF001C
:1025C000FF0000FFFFFFFFFF0000FF00FF00000013
:1025D000FF00FF0000FFFFFFFFFF0000FF00FF0004
:1025E0000000000000000000FF0000000000FFFFEE
:1025F000FF0000FF000000000000FFFF00000000DF
:102600000000FF0000FFFFFF0000000000FF0000CF
:1026100000000000000000FFFF0000FF00FFFF00BF
:1026200000FF00000000FF00000000FF00000000AD
:10263000FF00000000FF0000FFFF00FF0000FFFFA1
:102640000000000000000000FF00000000FF00FF8D
:10265000000000FF00FF00000000FF00000000FF7E
:1026600000FF00FF00FF0000FF000000FFFF00FF71
:102670000000000000000000FFFF00000000FFFF5E
:1026800000000000FF00000000000000000000004B
:10269000000000000000000000000000000000003A
:1026A000000000000000000000FF00000000FF002C
:1026B00000000000FF0000000000FF00000000001C
:1026C000FF0000000000FF000000000000FF00000D
:1026D0000000000000000000FF000000000000FFFC
:1026E0000000000000FF0000000000FF00000000EC
:1026F00000FF0000000000FF00000000FF000000DD
:102700000000000000000000000000000000FF00CA
:10271000FF000000FFFFFF0000FFFFFFFFFF0000C2
:10272000FFFFFF000000FF00FF00000000000000AE
:10273000000000000000000000000000000000FF9A
:102740000000000000FF000000FFFFFFFFFF00008F
:1027500000FF0000000000FF00000000000000007B
:102760000000000000000000000000000000000069
:102770000000000000000000000000000000000059
:10278000000000000000FFFF00000000FFFF00004D
:102790000000FF000000000000000000000000003A
:1027A000000000000000000000FFFFFFFFFF00002E
:1027B0000000000000000000000000000000000019
:1027C0000000000000000000000000000000000009
:1027D00000000000000000000000000000000000F9
:1027E000000000000000FFFF00000000FFFF0000ED
:1027F00000000000000000000000000000000000D9
:1028000000FF00000000FF00000000FF00000000CB
:10281000FF00000000FF00000000000000000000BA
:1028200000000000000000002F2F2F00002F0000EC
:10283000002F002F00002F2F002F002F002F002F20
:102840002F00002F002F0000002F00002F2F2F003F
:102850000000000000000000002F000000002F2FEB
:1028600000000000002F00000000002F000000000A
:10287000002F00000000002F000000002F2F2F006D
:1028800000000000000000002F2F2F00002F00008C
:10289000002F00000000002F0000002F2F0000007C
:1028A0002F000000002F00000000002F2F2F2F2FDF
:1028B00000000000000000002F2F2F00002F00005C
:1028C000002F00000000002F00002F2F2F0000001D
:1028D0000000002F002F0000002F00002F2F2F00DE
:1028E000000000000000000000002F000000002F8A
:1028F0002F0000002F002F00002F00002F00002FBE
:102900002F2F2F2F000000002F00000000002F00AD
:10291000000000000000002F2F2F2F2F002F00009D
:102920000000002F00000000002F2F2F2F000000BC
:102930000000002F002F0000002F00002F2F2F007D
:102940000000000000000000002F2F0000002F00FA
:102950000000002F00000000002F2F2F2F00002F5D
:102960000000002F002F0000002F00002F2F2F004D
:10297000000000000000002F2F2F2F2F000000006C
:10298000002F000000002F000000002F00000000BA
:102990002F00000000002F00000000002F000000AA
:1029A00000000000000000002F2F2F00002F00006B
:1029B000002F002F0000002F00002F2F2F00002FCE
:1029C0000000002F002F0000002F00002F2F2F00ED
:1029D00000000000000000002F2F2F00002F00003B
:1029E000002F002F0000002F00002F2F2F2F00009E
:1029F0000000002F000000002F0000002F2F00001B
:102A000000000000000000000000000000000000C6
:102A100000000000FFFF00000000FFFF00000000BA
:102A2000000000000000FFFF00000000FFFF0000AA
:102A30000000000000000000000000000000000096
:102A400000000000FFFF00000000FFFF000000008A
:102A5000000000000000FFFF00000000FFFF00007A
:102A60000000FF0000000000000000FF0000000068
:102A7000FF00000000FF00000000FF000000000059
:102A800000FF000000000000FF000000000000FF49
:102A90000000000000000000000000000000000036
:102AA000000000FFFFFFFFFF00000000000000002B
:102AB0000000000000FFFFFFFFFF0000000000001B
:102AC0000000000000000000FF000000000000FF08
:102AD000000000000000FF000000000000FF0000F8
:102AE0000000FF00000000FF00000000FF000000E9
:102AF0000000000000000000FFFFFF0000FF0000DA
:102B000000FF0000000000FF000000FFFF000000C9
:102B100000FF0000000000000000000000FF0000B7
:102B20000000000000000000FFFFFF0000FF0000A9
:102B300000FF00FF00FFFFFF00FF00FF00FF00FF9E
:102B400000FFFFFF00FF000000000000FFFFFF008C
:102B50000000000000000000FFFFFF0000FF000079
:102B600000FF00FF000000FF00FF000000FF00FF6B
:102B7000FFFFFFFF00FF000000FF00FF000000FF5D
:102B800000000000000000FFFFFFFF0000FF00004A
:102B900000FF00FF000000FF00FFFFFFFF0000FF3D
:102BA000000000FF00FF000000FF00FFFFFFFF002C
:102BB0000000000000000000FFFFFF0000FF000019
:102BC00000FF00FF0000000000FF0000000000FF09
:102BD0000000000000FF000000FF0000FFFFFF00FA
:102BE00000000000000000FFFFFFFF0000FF0000EA
:102BF00000FF00FF000000FF00FF000000FF00FFDB
:102C0000000000FF00FF000000FF00FFFFFFFF00CB
:102C100000000000000000FFFFFFFFFF00FF0000BA
:102C2000000000FF0000000000FFFFFFFF0000FFAA
:102C30000000000000FF0000000000FFFFFFFFFF9A
:102C400000000000000000FFFFFFFFFF00FF00008A
:102C5000000000FF0000000000FFFFFFFF0000FF7A
:102C60000000000000FF0000000000FF0000000066
:102C70000000000000000000FFFFFF0000FF000058
:102C800000FF00FF0000000000FF00FFFFFF00FF4B
:102C9000000000FF00FF000000FF0000FFFFFFFF3B
:102CA00000000000000000FF000000FF00FF000027
:102CB00000FF00FF000000FF00FFFFFFFFFF00FF1D
:102CC000000000FF00FF000000FF00FF000000FF09
:102CD0000000000000000000FFFFFF00000000FFF8
:102CE0000000000000FF0000000000FF00000000E6
:102CF00000FF0000000000FF00000000FFFFFF00D9
:102D00000000000000000000000000FF00000000C4
:102D100000FF0000000000FF0000000000FF00FFB7
:102D2000000000FF00FF000000FF0000FFFFFF00A9
:102D300000000000000000FF000000FF00FF000096
:102D4000FF0000FF00FF000000FFFF00000000FF89
:102D500000FF000000FF0000FF0000FF000000FF78
:102D600000000000000000FF0000000000FF000065
:102D7000000000FF0000000000FF0000000000FF56
:102D80000000000000FF0000000000FFFFFFFFFF49
:102D900000000000000000FF000000FF00FFFF0037
:102DA000FFFF00FF00FF00FF00FF000000FF00FF2B
:102DB000000000FF00FF000000FF00FF000000FF18
:102DC00000000000000000FF000000FF00FFFF0007
:102DD00000FF00FF00FF00FF00FF0000FFFF00FFFB
:102DE000000000FF00FF000000FF00FF000000FFE8
:102DF0000000000000000000FFFFFF0000FF0000D7
:102E000000FF00FF000000FF00FF000000FF00FFC8
:102E1000000000FF00FF000000FF0000FFFFFF00B8
:102E200000000000000000FFFFFFFF0000FF0000A7
:102E300000FF00FF000000FF00FFFFFFFF0000FF9A
:102E40000000000000FF0000000000FF0000000084
:102E50000000000000000000FFFFFF0000FF000076
:102E600000FF00FF000000FF00FF000000FF00FF68
:102E700000FF00FF00FF0000FF000000FFFF00FF59
:102E800000000000000000FFFFFFFF0000FF000047
:102E900000FF00FF000000FF00FFFFFFFF0000FF3A
:102EA0000000FF0000FF000000FF00FF000000FF27
:102EB0000000000000000000FFFFFF0000FF000016
:102EC00000FF00FF000000000000FFFFFF00000007
:102ED000000000FF00FF000000FF0000FFFFFF00F8
:102EE00000000000000000FFFFFFFFFF000000FFE8
:102EF0000000000000FF0000000000FF00000000D4
:102F000000FF0000000000FF0000000000FF0000C4
:102F100000000000000000FF000000FF00FF0000B4
:102F200000FF00FF000000FF00FF000000FF00FFA7
:102F3000000000FF00FF000000FF0000FFFFFF0097
:102F400000000000000000FF000000FF00FF000084
:102F500000FF00FF000000FF00FF000000FF00FF77
:102F6000000000FF0000FF00FF00000000FF000065
:102F700000000000000000FF000000FF00FF000054
:102F800000FF00FF00FF00FF00FF00FF00FF00FF49
:102F900000FF00FF00FF00FF00FF0000FF00FF0038
:102FA00000000000000000FF000000FF00FF000024
:102FB00000FF0000FF00FF00000000FF0000000015
:102FC000FF00FF0000FF000000FF00FF000000FF07
:102FD00000000000000000FF000000FF00FF0000F4
:102FE00000FF00FF000000FF0000FF00FF000000E6
:102FF00000FF0000000000FF0000000000FF0000D4
:1030000000000000000000FFFFFFFF0000000000C4
:10301000FF00000000FF00000000FF00000000FFB4
:103020000000000000FF0000000000FFFFFFFF00A5
:10303000000000000000000000FFFF000000FF0093
:1030400000000000FF00000000FFFF000000000083
:10305000FF0000000000FF000000000000FFFF0074
:10306000000000000000000000FFFF000000FF0063
:1030700000FF00FF00FFFF00FFFF00FF0000FFFF59
:1030800000FFFF00FF00FF0000FF000000FFFF0047
:103090000000000000000000FFFF00000000000032
:1030A000FF0000000000FF0000000000FFFF000024
:1030B0000000FF0000000000FF000000FFFF000014
:1030C0000000000000000000000000000000000000
:1030D00000000000000000000000000000000000F0
:1030E00000000000000000000000000000000000E0
:1030F00000000000000000FFFFFF7F7F24FFBBBB3C
:10310000BB1824FFBBFFBD18247FBBBD78181A7FF6
:10311000BB7878181A7FBB787818527FBB181818BC
:103120005224241A1A5252FFFFFF7F7F24FFECEC37
:10313000EC9024FFECFFF590247FECF5D9901A7FFA
:10314000ECD9D9901A7FECD9D990527FEC9090901D
:103150005224241A1A5252FFFFFF7F7F24FF6F6F01
:103160006F1424FF6FFFB714247F6FB71F141A7FEB
:103170006F1F1F141A7F6F1F1F14527F6F141414B8
:103180005224241A1A5252FFFFFF7F7F24FF7777C1
:10319000771C24FF77FFB71C247F77B72F1C1A7F7B
:1031A000772F2F1C1A7F772F2F1C527F771C1C1C08
:1031B0005224241A1A5252FFFFFF7F7F24FFE5E5B5
:1031C000E58A24FFE5FFEE8A247FE5EECB8A1A7FAD
:1031D000E5CBCB8A1A7FE5CBCB8A527FE58A8A8AF8
:1031E0005224241A1A5252FFFFFF7F7F24FFF3F369
:1031F000F39824FFF3FFF598247FF3F5F0981A7FF6
:10320000F3F0F0981A7FF3F0F098527FF3989898C3
:103210005224241A1A5252FFFFFF7F7F24FF5F5F60
:103220005F0424FF5FFFAF04247F5FAF07041A7FB2
:103230005F0707041A7F5F070704527F5F040404D7
:103240005224241A1A5252FFFFFFFFFF52FFADA46F
:10325000ADA452FFA4ADA4A452FFADADADA452FFE6
:10326000ADA4ADA452FFADADA4A452FFA4A4A4A4E8
:1032700052525252525252A4A4A4A4A4A4A45B49F0
:103280005B49A4A4495B495BA4A45B495B49A4A432
:10329000495B495BA4A45B495B49A4A4495B495BC6
:1032A000A4A4A4A4A4A4A4FFFFFFFFFFFFFFFFFFAB
:1032B000FFFFFFFFFFFFFFFFFFFFFFFFFFFFFFFF1E
:1032C000FFFFFFFFFFFFFFFFFFFFFFFFFFFFFFFF0E
:1032D000FFFFFFFFFFFFFFFFFF00000000FFF57F84
:1032E000000000FFECF57F00007FECFFD97F007F3E
:1032F000ECD9D924007FECD92400007FEC24000015
:1033000000242400000000FFFFFFBFBF3FFFFDFDC2
:10331000FD703FFFFDFFFF703FBFFDFF78702DBFC9
:10332000FD7878702DBFFD7878705BBFFD70707090
:103330005B3F3F2D2D5B5BFFFFFFBFBF3FFFFFFFED
:10334000FFD83FFFFFFFFFD83FBFFFFFF2D82DBFE1
:10335000FFF2F2D82DBFFFF2F2D85BBFFFD8D8D86A
:103360005B3F3F2D2D5B5BFFFFFFBFBF3FFFBFBF3D
:10337000BF1F3FFFBFFFFF1F3FBFBFFF371F2DBF57
:10338000BF37371F2DBFBF37371F5BBFBF1F1F1F83
:103390005B3F3F2D2D5B5BFFFFFFBFBF3FFFBFBF0D
:1033A000BF373FFFBFFFFF373FBFBFFF3F372DBFD7
:1033B000BF3F3F372DBFBF3F3F375BBFBF373737BB
:1033C0005B3F3F2D2D5B5BFFFFFFBFBF3FFFFFFF5D
:1033D000FFD53FFFFFFFFFD53FBFFFFFDED52DBF6E
:1033E000FFDEDED52DBFFFDEDED55BBFFFD5D5D539
:1033F0005B3F3F2D2D5B5BFFFFFFBFBF3FFFFDFD31
:10340000FDF03FFFFDFFFFF03FBFFDFFF8F02DBFD8
:10341000FDF8F8F02DBFFDF8F8F05BBFFDF0F0F01F
:103420005B3F3F2D2D5B5BFFFFFFBFBF3FFFAFAF9C
:10343000AF073FFFAFFFFF073FBFAFFF07072DBF3E
:10344000AF0707072DBFAF0707075BBFAF0707072A
:103450005B3F3F2D2D5B5B9A9A9A9A9A9A9A4848BD
:1034600048489A9A484848489A9A484848489A9AF0
:10347000484848489A9A484848489A9A4848484884
:103480009A9A9A9A9A9A9A00000000000000000006
:103490000000000000000000000000FF00FF00002E
:1034A0000000FF00000000FF00FF0000000000001F
:1034B00000000000000000999999999999999999AB
:1034C000999999999999999999999999999999996C
:1034D000999999999999999999999999999999995C
:1034E0009999999999999948484848484848484825
:1034F000994848484848E24848484848EA484848BF
:1035000099EAFEEA99484848EA4848484848E24863
:1035100048484848994848484848484848484848DA
:1035200048484848E2484848E24848EA48EA4848A3
:103530004848FE48484848EA48EA4848E248484877
:10354000E248484848484848484848484848484861
:10355000484848484848994848484848E248484800
:1035600048E2FEE248484848E24848484848994806
:1035700048484848484848484848484848484848CB
:103580004848484899484848484848E248E2484836
:103590004848FE48484848E248E2484848484848C1
:1035A000994848484848484848484848484848484A
:1035B000484848484848484848484848994848483A
:1035C0004899EA99484848489948484848484848E6
:1035D000484848484848484848484848484848486B
:1035E00048484848484848484848489948994848B9
:1035F0004848EA4848484899489948484848484807
:10360000484848484848484848484848484848483A
:10361000484848484848484848484848484848482A
:103620004848E24848484848484848484848484880
:10363000484848484848484848484848484848480A
:1036400048484848484848484848484848484848FA
:1036500048484848484848484848484848484848EA
:103660004848484848484800000000000000000062
:10367000990000000000E20000000000EA000000E5
:1036800099EAFEEA99000000EA0000000000E2006A
:103690000000000099000000000000000000000091
:1036A00000000000E2000000E20000EA00EA000082
:1036B0000000FE00000000EA00EA0000E200000056
:1036C000E200000000000000000000000000000018
:1036D000000000000000990000000000E20000006F
:1036E00000E2FEE200000000E2000000000099009D
:1036F00000000000000000000000000000000000CA
:103700000000000099000000000000E200E200005C
:103710000000FE00000000E200E2000000000000E7
:103720009900000000000000000000000000000000
:1037300000000000000000000000000099000000F0
:103740000099EA99000000009900000000000000C4
:103750000000000000000000000000000000000069
:103760000000000000000000000000990099000027
:103770000000EA000000009900990000000000002D
:103780000000000000000000000000000000000039
:103790000000000000000000000000000000000029
:1037A0000000E20000000000000000000000000037
:1037B00000000000000000999999999999999999A8
:1037C0009999999999999999999999999999999969
:1037D0009A5A9A999999995B1C5B9A99999A1C1C87
:1037E0001B9999995B2E36999999999999999999D3
:1037F0009999999999999999999999999999999939
:1038000099999999999999999999995B9A99999965
:10381000991C1B5B5A995A99999999999999999ACE
:103820009A999999995B5A9999995A1C1B51999906
:103830005B2E2552995A1C372E1B515B2E3737258C
:1038400052253737372E1B999999999999999999B2
:1038500099999999999999999999999999999999D8
:103860009999999999999999999999999999995A07
:103870005B519A5A5B1C2E999999999999999999A2
:1038800099999999999999999999999999999999A8
:10389000995A5A99995A5B5C5151995C2E534891A7
:1038A00099361C0949999999999999999999999948
:1038B0009999999999999999999999999999999978
:1038C000999999999999999999999999995A9A99A6
:1038D00099999A245B919900000000000000FFFF75
:1038E000FFFFFF000000FF00005A5A00FF00001C0D
:1038F0001C00FF00002E3700FF00001B1C00FF0013
:103900003751520000003700361C0000000037001D
:1039100000FFFF003700FF000000000000FFFFFF76
:10392000FF00000000000000000000373700FFFF2C
:10393000FF373700000000000000000000FF00FF1C
:10394000FFFF000000FF0000FF0000FF0000FFFF7E
:1039500000FFFFFF00FF00FF0000000000FF003736
:103960003700000000373700000000003700FF007C
:10397000FF000000FF00FFFF0000FF00FF00FF004E
:10398000FF00FF000000FF00FF000000FF00FF003D
:103990003700000000003700000091999900FF00F7
:1039A00099999900FF0099999900FF005A5A5AFF76
:1039B000FF001C1C1C00FF0037362D00FF002D1BD4
:1039C000120000001209499900000000000000A444
:1039D000A4A40000AD000000000000FFFF000013E1
:1039E000000000FF0000000000AD0000A4A4A4003F
:1039F00000000000000000000000003700A400A448
:103A0000000000AD00ADAD0000FF00FF00FF00FFB3
:103A100000FF0000FFAD00AD000000A400A4002ED8
:103A200000000000001B00000000000000A40000D7
:103A3000A4A4A4AD00AD000000FF00FF000000FF43
:103A400000FF00FFFFAD00AD0000ADA40000A4A486
:103A5000A400000000000000000037000000A400E7
:103A60003700A400AD003700AD00FF003700FF00B5
:103A7000FF003700FF00AD000000AD00A4A4A400CB
:103A8000A4000000000000000000005191A4A4A4C4
:103A9000005B5A00000000362DFFFF001C1C1C00BC
:103AA0000000131313000000005151A4A4A40099B6
:103AB00099000000009999999999999999999999DA
:103AC0009999999999999999999A5A5A5A5A5A99A0
:103AD0005A5B251C1C999951521B2599999999510A
:103AE000529999999999999999999A1B369999996D
:103AF000995B2E999999995A1C5A5A5A5A5A1C1CD0
:103B00001C1C1C1C1C2E37373737371B1C2E373715
:103B10003751521B2E373737361C1B5B5B37373715
:103B2000362E2E3737373737373737373737373738
:103B30003737373737373737373737373737373715
:103B4000373737373737372E373737372D37373718
:103B500037373737373737373737373737373737F5
:103B600037373737373737373737373737373737E5
:103B700037373737373737125B1C2E37372E2E370C
:103B800037373737373737372E37373737372E37D7
:103B900037373737373737373737373737373737B5
:103BA000373737373737372E12089199991C09491B
:103BB0009999991B099199999913525A5A5A5A1CD1
:103BC0001C1C1C1C1C37373737362D3737372D1B3D
:103BD0001237371C12094999999999999999999984
:103BE0009999999999999999995A5A5A5A5A9A1CFC
:103BF0002D1C5B51511C12090951990909519199C8
:103C00009951919999999999999999999A99999973
:103C10009999999999999999999999999999999914
:103C20009999999999995B645B5B5B995A5B1C2D97
:103C30002E99999951521C5B9A999999995B1C5BA1
:103C40009A99995A2D2E245B9A995B37372E25998C
:103C50005A2D3737375B5B25373737362E363737B0
:103C600037363737373737995A2E25519999643770
:103C70003652995A2E373725512D37373737253752
:103C800037373737373737373737373737373737C4
:103C900037373737373737999999995A5A99995AFF
:103CA0005B25125A642D371B492D37372D095137A3
:103CB00037371C499937373724535B373737362E18
:103CC0003637373737372D99999999999951999965
:103CD0009999999999999999999999999999999A53
:103CE0009A99999A995B5B645B5A992E251B1249A4
:103CF000991B0949519999999999999999999999DA
:103D00009999999999999999999999999A99999922
:103D100099995A5B9A99999999652E999A9A995B6A
:103D200037995B242D2D3799999999999999999952
:103D300099999999999999999999995B5A99999970
:103D40009A2E2491995B64372E5B6D37373737375E
:103D50003737373737373799999999999999999981
:103D60009999999999999999999999999999995B01
:103D70005B519999992E129199999925519A9A9AEC
:103D800099362D251B5299999999999999999999AB
:103D90009999999999999999999999999999999993
:103DA0009999999999999999999999999999999983
:103DB00099999999999A9A99999999999999999971
:103DC0009999999999999999999999999999999963
:103DD00099999999999999995A99995B9A63259979
:103DE0005B633636373625999999999999999999B6
:103DF0009999999999999999999999999999999933
:103E00009999999999999999999999599999999962
:103E1000995A9A9999999900000000003700A1A138
:103E2000A1000000FA0000FA0000FF0000FF0000FF
:103E3000FA0000FA0000A10000A100009999990081
:103E40000000000000003600000000000000A1A1FA
:103E50000000A1FA0000FA00FAFF0000FF00FFFADC
:103E60000000FA00FAA10000A100A1009999000049
:103E700000000000001B000000000000000000A186
:103E800000A1A10000FA00FA000000FF00FFFF00FF
:103E900000FA00FA000000A100A100999900009921
:103EA00099000000000000000000000037A10000A1
:103EB000A1003700FA00FA0037FF0000FF003700CA
:103EC000FA00FA003600A100A100009900009999BB
:103ED0009900000000000000000000000000A1A107
:103EE000A1A10000FA0000000000FFFFFF001C007D
:103EF000FA0000001300A1000000000099999999B0
:103F00000000000000000000000000000000272763
:103F10002727270000003700001C1C00FF001C138F
:103F2000130037001C51510027001C9999001500FF
:103F30002E9999000000360000000000000027279D
:103F400027000000370000370000FF0000FF0000DE
:103F50003737370000002700002700001500001544
:103F60000000000000000000000000000027002703
:103F7000272700370037000037FF00FF0000FF371A
:103F800000373737002700270000001500150037DD
:103F90003700000000372D00000037000000270028
:103FA00037002700370037003700FF003700FF00D9
:103FB00037003700370027000000270015151500CF
:103FC000150000000000000000001251912727009A
:103FD0002D5B5A00000037362DFFFF001C1C1C0013
:103FE0000000131313000000515151151500999949
:103FF00099000000999999999999999999999999FC
:10400000999A9A99999A9A5B1C999A5B1C2E1C5AB8
:104010005B5B5B131399515151515199999999993E
:1040200099999999999999995A5B2E37375B1C2ED2
:104030003737372E37373737371C1C1C1C1C1C13DF
:10404000131313131C51515149521C999999995B9F
:104050002E9999999A5C363737373737373737374C
:1040600037373737373737373737373737373737E0
:104070003737373737373737373737373737372ED9
:104080003637362E1C1B1B3737373737373737371E
:1040900037373737373737373737373737373737B0
:1040A00037373737373737373737373737373737A0
:1040B0003736373737372D3737373737373737379B
:1040C0003737373737373737373737373737373780
:1040D000373737373637373737372E2E3637373784
:1040E00037131B2E36373737371C12519137373677
:1040F0002D5B5A37373737362D1C1C1C1C1C1C1BDC
:1041000012131313131349515151511C5199999979
:10411000992E12919999999999999999999A999908
:104120009999991B5A9A9999991C2D1C5A999913E6
:104130001313135A9A51515151515199999999996F
:104140009999999999999999999999995299999926
:104150009A5B65999A5B24252E995B1B1B13139917
:104160005151515151999999999999999999999927
:104170009999999999999925373737373737373733
:104180003737372E2D2E373737121225373737511D
:10419000522D373737996437372E245A2E2E241252
:1041A000095B2412094991373737373737373737A3
:1041B000373737373737373737373737373737378F
:1041C000373737373725373737361C522E373724AE
:1041D000099964372E1248373737372E1237373759
:1041E00037372E3737372E2D2E37373724121337E0
:1041F00037371C49512D37372E5299521B25361C03
:1042000051999152132452495199999999645B9A01
:104210009999992D24645B9A9913131B1B5A9951F0
:10422000515151519999999999999999999999991E
:1042300099999999999999999951243737999A63A4
:104240002D3737995B1B1B1B3799919191633799D8
:1042500099999A251C9999995A525199999999998C
:104260009999999999999937373737373737373730
:104270003737373737373737372E2E37372D3751D0
:104280005B372D515A99992D13919999995A5199B2
:1042900099999999999999372E125191993736642C
:1042A0005A9A992D1B1B1B5A992E51919191992520
:1042B0005B99999999915251999999999999999943
:1042C0009999999999999999999999995B9999999C
:1042D00099995B99999999995199999999999999D4
:1042E000999999999999999999999999999999993E
:1042F000999999999999992E37373737372E3737B2
:104300003737365B2E2E372E255B995B24995B99C8
:104310009999519999999999999999999999999955
:1043200099999999999999245299999999245A996D
:104330009999995151999999995A999999999999BC
:1043400099999999999999999999999999999999DD
:10435000999999999999999999995B2E3699999AD8
:104360005B2E1B99995B1C1B09999A5A5208499913
:1043700099995191999999999999999999999999FD
:10438000999999999999992E1B131209521B1249BF
:104390004951994849519999995199999999999956
:1043A000999999999999999999999999999999997D
:1043B0009999999999999925373737361B5B2E37F3
:1043C000372D125A2537361B089A5B2E251248992D
:1043D0005A2D1B095199991B12489999995A49517B
:1043E000999999995199990951121B1C364899919B
:1043F00051121B5199999991519999999999999912
:10440000999999999999999999999999999999991C
:1044100099999999999999371C519999991C2D12A3
:10442000919999121B1B5199999951121199999926
:10443000999951519999999999999999999999997C
:104440009999999999999999999999999A999999DB
:1044500099999999999999999999999999999999CC
:1044600099999999999999999999999999999999BC
:10447000999999999999995A0949919999919199E3
:10448000999999999999999999999999999999999C
:10449000999999999999999999999999999999998C
:1044A00099999999999999995A2E24099199996468
:1044B00012499999995A4991999999915191999932
:1044C000999999999999999999999999999999995C
:1044D0009999999999999999999991521299999922
:1044E0009999919999999999999999999999999944
:1044F000999999999999999999999999999999992C
:10450000999999999999995199999999999199996B
:10451000999999999999999999999999999999990B
:1045200099999999999999999999999999999999FB
:1045300099999999999999999999999999999999EB
:104540009999999999999999999999999999990074
:10455000000000000000FFFFFF000000FF0000FF60
:104560000000FFFFFF0000999999999999999999ED
:1045700099999999999999999999999999A2A30031
:104580000000000000FFFFFF0000FFFF00FF00FF32
:1045900000FFFFFF00FF00999999999999999999BE
:1045A000999999999999999999ACEDEDEDACA300E8
:1045B0000000000000FF00FF0000FF0000FF00FF00
:1045C00000F600FFFF000099999999999999999996
:1045D00099999999999999999999999999999900E4
:1045E000AC9999999900FFF699999900F6FEA499CA
:1045F00099F6F6F6F65199999999999999999999FF
:10460000999999999999999999999999999999991A
:1046100099999999999999999999999999999AA3FF
:10462000A39AA3F5FFFFFF99999999999999999957
:1046300099999999999999999999999999999999EA
:104640009999999999999999999999ACECACA29958
:1046500099FFFFFFFFF6A3999999999999999999CB
:1046600099999999999999999999999999999999BA
:1046700099999999999999999999999999999999AA
:1046800099999999A2A3AC99999999999999999974
:10469000999999999999999999999999999999998A
:1046A000999999999999999999999999999999997A
:1046B00099A39A999999999999999A1B360000000A
:1046C00000000000FFFFFFFFFF000000FFFF001CD5
:1046D0001C003737002E3700FFFF001B1C00AAAA62
:1046E00000515200AAAA0037361C1B5B5B00003742
:1046F000362E2EFF003737373700000000003737DF
:104700003737370000FFFF0000FFFFAAAA000000B4
:10471000AAAAAAAA0000AA2E373737372D3737376B
:104720003737373737373737373737373737370050
:104730000000000000FFFF00FFFFFFAA0000AAAA80
:1047400000AA0000AAAA00125B1C2E37372E2E37B3
:104750003737373737373737003737000000000033
:104760000000373700FF0000FFFF00AAAA00AAAA36
:1047700000AAAA00AAAA002E120891999900000086
:1047800000009900FFFFFF0000FFFF00FFFF003760
:10479000370000FF0000FFFF00002D0000AAAA0064
:1047A00000000000AAAA009999999A1B36000000FF
:1047B0000000000047474747470000004747001CEC
:1047C0001C000606002E37009B9B001B1C009B9BB9
:1047D00000515200FFFF0037361C1B5B5B000037A7
:1047E000362E2E47003737373700000000003706D7
:1047F00006060600009B9B00009B9B9B9B00000005
:104800009BFFFFFF0000FF2E373737372D37373735
:10481000373737373737373737373737373737005F
:1048200000000000009B9B009B9B9B9B00009B9BB0
:1048300000FF0000FFFF00125B1C2E37372E2E37C3
:104840003737373737373737003737000000000042
:1048500000000606009B00009B9B009B9B009B9B0F
:1048600000FFFF00FFFF002E120891999900000041
:1048700000009900474747000047470047470006A8
:104880000600000600009B9B00002D00009B9B0083
:1048900000000000FFFF009999999A1B3600000064
:1048A0000000000032323232320000003232001C8E
:1048B0001C00FFFF002E3700FCFC001B1C003737DC
:1048C0000051520037370037361C1B5B5B00003746
:1048D000362E2E320037373737000000000037FF02
:1048E000FFFFFF0000FCFC0000FCFC37370000006D
:1048F000373737370000372E373737372D373737C9
:10490000373737373737373737373737373737006E
:104910000000000000FCFC00FCFCFC370000373706
:1049200000370000373700125B1C2E37372E2E372A
:104930003737373737373737003737000000000051
:104940000000FFFF00FC0000FCFC00373700373799
:10495000003737003737002E120891999900000070
:10496000000099003232320000323200323200FF51
:10497000FF0000FF0000FCFC00002D0000373700A6
:104980000000000037370099999999999999999958
:104990009999AC99999999ACB5999999A3B5AC990C
:1049A000999AADACAC9999A4ACA3A39999ADA3A3E2
:1049B000A3999AACA39B9B00FF0000FF0000FFFFA0
:1049C000FF0000000000000000ACACACAC00FFAC8D
:1049D000ACACAC0000A3A3A3A3A3000000000000A4
:1049E0000000FFFFFF0000FF00FF00FF00FF00FFCF
:1049F0000000FF000000000000FFFF00FFFFFFFFBE
:104A00000000FF00FFFF0000FFFFFF0000000000AC
:104A100000FFFFFF0000FF0000FF00FF00FF00FF9E
:104A20000000FF00000000000000ACACACACAC002B
:104A3000ACACACACAC00A3A3A3A3A30000000000EB
:104A400000FF00FF0000FF00F6F6F6519900B5B533
:104A5000F6499900ADADAD0899ACACAD9B4899ACA9
:104A6000ACAD495199A4AD52489999009B48919990
:104A70009900085199999999999999999999999918
:104A80009999999999999999999999999999999996
:104A9000999999999999999999999A999999999985
:104AA000A39999999999A39999999999A499999957
:104AB000A3F5F69999A3F6F6B599A3B5ADADADA357
:104AC000ADACACACACACACA4A4A4A4ACA3A3A3A369
:104AD000A3A39A9B9B9B9BF6FFFFFEFEFEF6F6F6BA
:104AE000F6F6F6B5B5B5B5B5B5ADADADADADADACEC
:104AF000ACACACACACA4A4A4A4A4A4A3A3A3A3A353
:104B0000A39B9B9B9B9B9BFEFEFEFEFFF6F6F6F691
:104B1000F6F6FEB5B5B5B5B5F6ADADADADADF5AC2A
:104B2000ACACACACADA4A4A4A4ACA3A3A3A3A4A418
:104B3000499A9AA3A451519A9999999999AC9199A2
:104B4000999999A45199999999A451999999995296
:104B50005199999999489999999999919999999966
:104B600099999999999999999999999999999999B5
:104B70009999A399999999A3F5999999A3ADAC9904
:104B8000999AACA3A399999AA35A9A99999AA35AD4
:104B90005A9999999A9A5A9AACF6FFFFFFF5F6F648
:104BA000F6F6F6B5ADB5B5B5B5ACACACACACACA342
:104BB000A3A3A3A3A39A9A9A9A9A9B5A5A5A5A5A67
:104BC0005B5A5A5A5A5251FFFFAC999999F6F6F628
:104BD0009A9999B5ADB65A9999ACACAC519999A33B
:104BE000AC52919999A35251999999519199999946
:104BF0009999999999999999999999999999999925
:104C00009999999999999999999999999999999914
:104C1000999999999A99999999999A999999999902
:104C200099999999999999999999999999999199FC
:104C30009A9A9999A3F6F6FEEDACB5B5ADADADA4D3
:104C4000A3A3A3A49A5A5A5A5A5A919A5A5191997B
:104C500099999999999999999999999999999999C4
:104C60009999995199999999995199999999999944
:104C700099999999999999999999999999999999A4
:104C800099999999999999995A006767005B1C00BD
:104C90006767002E3700FFFF001C1C003C3C001320
:104CA0001300ECEC00515100ECEC00999900060661
:104CB00000999900000000676700000067676700BF
:104CC000000067FFFF000000FF3C3C3C3C003CEC68
:104CD000ECECEC0000000000000037373737372ECF
:104CE0003637362E1C1B1B6700006767676700009E
:104CF000676700FF0000FFFF003C00003C3C000035
:104D00000000000000373737373737373737373746
:104D10003736373737372D6700006767006767001A
:104D2000676700FFFF00FFFF003C3C003C3C0000C9
:104D30000000ECEC003737000000002E3637373724
:104D400000131B2E36373700000067670000000095
:104D5000676700000000FFFF003C00003C3C00ECE7
:104D6000ECECECEC00ECECECEC00000006060000D7
:104D700099000000009999995A003333005B1C0098
:104D8000FAFA002E3700FAFA001C1C00FFFF00138D
:104D900013001F1F005151001F1F00999900373742
:104DA00000999900000000333300000033FAFA0044
:104DB0000000FAFAFA000000FAFFFFFFFF00FF1FF1
:104DC0001F1F1F0000000000000037373737372E45
:104DD0003637362E1C1B1B330000333333FA0000EA
:104DE000FAFA00FA0000FAFA00FF0000FFFF0000E4
:104DF0000000000000373737373737373737373756
:104E00003736373737372D330000333300FAFA009F
:104E1000FAFA00FAFA00FAFA00FFFF00FFFF0000BA
:104E200000001F1F003737000000002E36373737CD
:104E300000131B2E3637370000003333000000000C
:104E4000FAFA00000000FAFA00FF0000FFFF001F5E
:104E50001F1F1F1F001F1F1F1F00000037370000EC
:104E600099000000009999995A00FFFF005B1C000F
:104E70008686002E37008686001C1C00F2F2001386
:104E80001300323200515100FFFF00999900FFFFDB
:104E900000999900000000FFFF000000FF868600D7
:104EA000000086868600000086F2F2F2F200F232FE
:104EB0003232320000000000000037373737372E1B
:104EC0003637362E1C1B1BFF0000FFFFFF8600003D
:104ED000868600860000868600F20000F2F200005E
:104EE0000000000000373737373737373737373765
:104EF0003736373737372DFF0000FFFF0086860033
:104F0000868600868600868600F2F200F2F20000B5
:104F100000003232003737000000002E36373737B6
:104F200000131B2E363737000000FFFF0000000083
:104F3000868600000000868600FF0000F2F2003244
:104F40003232323200FFFFFFFF000000FFFF00009F
:104F500099000000009999999AAC5A5A5A9999ACBB
:104F60005A5A5A9999ACA35A59999999AC9B5A99FA
:104F70009999999BA49999999999519999999999DC
:104F80009999999999999900FF0000FF0000FFFFF6
:104F9000FF000000FF0000FF0000FFFFFF00000017
:104FA0000000000000525BA3A3A35A9991515151F4
:104FB00051999999999999FF00FF00FF00FFFFFF10
:104FC00000FF00FF00FF00FF00FF00FF0000FF00E8
:104FD000000000000052510848499151919199995F
:104FE000999999999999990000FF00FF005A00FF3B
:104FF000FF00000000FF00FF00FF00FF0000FF00B7
:10500000000000000099999999999999999999990D
:105010009999999999999900519999999951999929
:1050200099999900999999999900999999999900BB
:1050300099999999999999999999999999999999E0
:10504000999999999999999999999999A3999999C6
:105050009999A399999999999999999999999999B6
:1050600099999999999999999999999999999999B0
:10507000999999999999999B5A5A5A5A5AA35A594E
:10508000595959A39B5A595151999A5A5B9B9B99CB
:105090009999915151999999999999999999999918
:1050A000999999999999995A5A5A5A5A5A595959AA
:1050B000595A9B595A5A9B5B5A5B5A525249515101
:1050C00051519199999999999999999999999999E8
:1050D000999999999999995AA39B495199A3524998
:1050E00091999949519999999999999999999999D0
:1050F0009999999999999999999999999999999920
:10510000999999999999995A5251919999999999E5
:1051100099999999999999999999999999999999FF
:1051200099999999999999999999999999999999EF
:1051300099999999999999484848484848484848B8
:1051400048484848484848484848484848484848DF
:1051500048484848484848484848484848484848CF
:10516000B648484848B6B648484848484848484875
:1051700048484848484848484848484848484848AF
:105180004848484848484848484848B6B6B6B6B679
:10519000B6000000000000484848484848484848D1
:1051A000484848484848484848484848484848487F
:1051B0004848484848484848484848B64848484801
:1051C00048B6B64848484848484848484848484982
:1051D000484848484848484848484848484848484F
:1051E000484848484848484948484848484948483D
:1051F0004848480040484848484848B60048484859
:1052000048B60048484848B60048484848B60048AC
:10521000484848B60048484848B60048484848B654
:105220000048484848B60000B60048484800B60064
:1052300048484800B60048484800B600484848007A
:10524000B60048484800B60048484800B6004848FC
:105250004800B600484848484848484848484848F0
:105260004848484848484848524848484848F54807
:1052700048484851FE484848485AFE484848489BD4
:10528000FE4848484852FE48495AA39B485AF5FEF2
:10529000AC4948FEFEFE494848FEFEA4484848FE88
:1052A000FE9B484848FEFEA3484848FEFEAC4848DE
:1052B00048FEFEFE5A48484848484848484848483A
:1052C000484848484848484848484848484848485E
:1052D000484848484848484848484948484848484D
:1052E000484848484848484848000048484800005E
:1052F000004848400000000040000A5B5B0A48127A
:105300006D6E761C495B6D646D6D5151BFADB6AD70
:105310004849AD64AEA4484848484848F54848481C
:1053200048485A48484848484848484848484848EB
:1053300048484848484848484848484848484848ED
:1053400048484848484848FEFEFEFE9B48FEFEFE90
:10535000FEFEFEA3FEFEFEFEFE4851A4B5ACA34831
:1053600048484848484848484848484848484848BD
:1053700048484848484848484951484848F5F54948
:10538000484848F5524848484849484848484848E5
:10539000484848484848484848484848484848488D
:1053A0004848484848484851645C6D524848090A92
:1053B000124848495B5B5C494852ADADB6A44849C8
:1053C000A55BADA44849645C6D494849130A5B522A
:1053D0004849130B134948484848484848484848F2
:1053E000484848484848484848484848484848483D
:1053F000484848484848484848484848484848482D
:10540000484848494848484848484848484848481B
:10541000484848484848484849484848484809484A
:10542000484848480A48484848491248484848496E
:1054300013484848480A130913131352480A131310
:10544000135248131213131349131313131349134D
:10545000131313134A1313131313521313131313A6
:10546000520A1313131312484848484848484848FA
:1054700048484848484848484848484848484848AC
:10548000484848484848484848484849484848489B
:105490004849484848484848484848B60048484865
:1054A00048B60048484848B6B64848484848B6480C
:1054B000484848484848484848484848484848486C
:1054C000484848484848480000000000000000FFE5
:1054D0000000000000FF000000B600FFFFFFFF001B
:1054E00000FF0000004800FF00480048000000489E
:1054F00000484848484848000000000000FF0000FD
:10550000FFFFFFFF00FF000000FF00FF00B600FFED
:1055100000FF000000FF0000FFFFFF000000000090
:10552000004848484848480000000000000000FFCC
:10553000000000FF00FF000000FF00FF00B6B6FF04
:1055400000FF0000000000FFFFFFFF000000000060
:105550000048484848484800000000000000FFFF9D
:10556000FFFF0000FF000000FF00FF00B600FF008B
:10557000FF000000FF00FFFFFFFF00000000000031
:105580000048484848484800B60048484800B60027
:1055900048484800B600484848004000484848008D
:1055A000004848484800484848484848484848480B
:1055B000484848484848484848484848484848486B
:1055C000484848484848484848484848494848485A
:1055D0004848494848484848484848484848494849
:1055E0004848484849484848484949484848484838
:1055F0004948484848494948484848484948484827
:1056000048484848484848515B48484848525B48E1
:1056100048484848484848484848480A134848487D
:10562000490912484849A3095C4848496352AE48B1
:10563000485A64535B4800A4AD5B5B0000ADBFB744
:10564000B7F6FFBF6D656553130B0B0A13AD5B0A0D
:105650000AA56D5C640A0AAD5C65AD5B646D655B53
:1056600052091264655BADFFF65201B7B6AEAEBF2C
:10567000FF666E656E656E49484848484800484870
:1056800048484800514848484853514848484865A8
:105690005248484848095251484848FFFF51484835
:1056A0004876BFAD4948484848484848484848496E
:1056B000494848484849514848484849494848485D
:1056C0004849484848484849494848484849494855
:1056D000484848494048480000000000000000FFDA
:1056E0000000000000FF000000B600FFFFFFFF40C9
:1056F00000FF0000004800FF00480048000000488C
:105700000048484848484800B60048484800B600A5
:1057100048484800B600484848004000484848000B
:105720004048484848004848484848484848484849
:1057300048484848484848484848484848484848E9
:1057400048484848484848484848484848484848D9
:105750004848484848484848484848B6B6B6B6B6A3
:10576000B6B6B6B6B6B6B648484848000048484847
:105770004800FF4848484800FF4848484800FF485C
:1057800048484800FF4848484800FFB6B6B6B6004B
:10579000FFB6B6B6B60000000000000000FFFF0034
:1057A00000FF000000FF00FF000000FF00FF00FFFF
:1057B000FF0000FF0000000000FF0000B6B600FF81
:1057C000FF00B6B600000048480000000048000096
:1057D000FFFF004800FF0000FF4800FF0000FF48F7
:1057E00000FFFFFFFF0000FF0000FFFF00FF0000C1
:1057F000FF00000000000000000048000000FF0063
:105800004800FF00FF000000FF0000FF00FF000055
:105810000000FF0000004800FF004800B600FF0045
:10582000B600B6000000B600000000000000FFFF58
:10583000FF00FF00FF000000FF00FFFFFF00FF0070
:10584000FF000000FF00FF000000FF00FFFFFF005F
:10585000FF000000000000000000484848FFFF0073
:105860000048480000FF0048480000FF004848FF8B
:10587000FF000048480000FF0048480000FF00B655
:10588000B600000000B6B64800000048480000FF1F
:1058900000484800FFFF0048480000FF0048484813
:1058A00000FF0048480000FF00004800FFFFFF0025
:1058B000B60000000000B6484848484848484848F4
:1058C0004848484848484848484848484848484858
:1058D00048484848484848484848485B004848487D
:1058E00048B65B0048484848484840484848484906
:1058F0005B48484848495A48484848484848484802
:105900004848484848484849084848484849094894
:105910004848490909484848484848484848484884
:1059200048484848484848484848484848484848F7
:1059300048484848484848484848484848484848E7
:1059400051484848485B52484848494848484848B0
:10595000494848484849494848485152525148499D
:105960004952525B48494949495249009B40514973
:105970005B49AD009B5B4948B66D6413134812093F
:1059800012135B48526412B6004852B752655C006D
:105990001B125C6EB75BB612656E5B5B65651B1BAD
:1059A0005BA45B655C6EB7130A1D1302145B5C1C81
:1059B0000B5B6553FF5CAEB60A5C65145D5D0AB6B1
:1059C0006D14136EB7ADBF5365B6AE5B5C65655CB9
:1059D000136E5DAE655D6E1CB7FFF600480A65FF8D
:1059E000004848641B5A484848655C654848486E0A
:1059F000135C484848BF6512A448486D65B7A44881
:105A0000486514BF64484848485AA448484848492B
:105A100051494848484949484848484949484848F8
:105A2000490A09494848090A0A09494809090A016D
:105A3000490909090909014800000000480000FF60
:105A4000FF000000FF0000FF00000000FF00004812
:105A500000FF00004800FF0000000000FFFFFFFF04
:105A60000000000000000048484848B6B6484848D2
:105A700048B65B48484848B65B48484848B65B4823
:105A8000484848B65B48484848B65B48484848B626
:105A90005B48484848B65B5B5B5B5B5B5B00000058
:105AA00000000000000000000000000000000000F6
:105AB00000000000000000000000000000000000E6
:105AC000000000000000005B5B5B5B5B5B000000B4
:105AD000000000000000990000000000E20000004B
:105AE00000E2FEE200000000E20000000000990079
:105AF000000000000000005B5B5B5B5B5B00000084
:105B0000990000000000E20000000000EA00000030
:105B100099EAFEEA99000000EA0000000000E200B5
:105B2000000000009900005B5B5B5B5BB60000005F
:105B30000000000000000000000000000000000065
:105B40000000000000000000000000000000000055
:105B500000000000000000B65B00004848B65B0093
:105B6000004848B65B00004848B65B00004848B6AD
:105B70005B00004848B65B00004848B65B00004840
:105B800048B65B00004848484848484848484848A4
:105B900048484848484848484848484848480848C5
:105BA00048484808094848484911094848491B11CC
:105BB0001C48485B1B1B2548490909084849090935
:105BC0000900480909090000080800090000000848
:105BD00012080000001C1200090A091C0908121210
:105BE000001208111B0A0848484852AC484848515E
:105BF0009AAC4048489A9BED404849A39BF5480021
:105C000049EC9AFF914900F5A3FFEC0900ADECF7D0
:105C1000EC090952FF5352A4F640A4AE49EDF640F8
:105C2000A4FF52F6F740EDFF52FEFF48EDFF92F65B
:105C3000FF9AF6FF9AEDFF9AF6F69A9AFF51F6A4AC
:105C4000AC525C5A64529BEE525B6EB7B6ADA45B2D
:105C50005C5B13B5ED9B5C65B7B5F69BB66EB7FFA5
:105C6000F5A4B6B70AFFECED530000FFA4F6B6BFEB
:105C7000FF5BF5AD656625BFAE5C65B7B71B5C66BF
:105C80006E5B126D5C6E655C65B7AF531B6FB70AD8
:105C90005C64651D650009B6A50001BFBFB7B7FF0D
:105CA000B71D1D141C6566B76565644848B75C5B25
:105CB000BF08486513BFB649486E5C64524848BF88
:105CC0005C0AAD52485B0A01646348A55B0912494E
:105CD0004865ADA45BA4004848484848094848487E
:105CE00048480948484848090A484848480A0A486C
:105CF0004848490A0A484848091213484849490986
:105D00005C484849520A12090909090909090A1295
:105D10000A0A120A0A1212121212535C645B5C1213
:105D20001253135B5C135B645C6D645C5B64656D58
:105D30006D13535B5B65B54948484848485249482C
:105D40004848485B52484848486464494848486461
:105D50006D5A4848486DB6524848486D6D64484889
:105D600048B6BF524848485B5B5B5B5B5B0000002A
:105D7000000000000000000000000000990000008A
:105D80000099EA990000000099000000000000005E
:105D90000000000000000048484848B65B484848FA
:105DA00048B65B48484848B65B48484848B65B48F0
:105DB000484848B65B48484848B65B48484848B6F3
:105DC0005B48484848B65B4849645A652D48516D60
:105DD0005B6D6448516D636D6448496C646D6448E3
:105DE000486D64641248485A5B125B4848485BB788
:105DF000B6484848A3B66512111B1C09095A1A2453
:105E00001308525A1B2412525B1B6D1C5B5A121A48
:105E10005B12111A5B645B12091209AD65645C5B6D
:105E2000095C5C131252011112005B646D5B120974
:105E300064B6B75C12115BBFB611525209ADB60819
:105E4000524A49B7B700085240AD6E00094849AE02
:105E50006E00000049AE656465B76E6D5CB7B7B79C
:105E6000B7B7B7AEAE6E6EAEB7AEAEAE6E6E6EB765
:105E7000B7666EB76EAEAE256EB765AEAE256EB7C1
:105E800066AE6D256EB7655B645C65666E6F5C6E55
:105E90006E6E6E6E6E1D2525656EB7661D251DAE78
:105EA000651C1D1D1C6EB6651465AE6664651DAE71
:105EB000AE6665651D655C6E6EAD6566136E6EB62D
:105EC0006E650A25656E1D0B001D65FF650A001DC8
:105ED000655C0A0A091D65FF5C0B1366655B0A13A6
:105EE0001C6565F75B132501091212FFA4525B12B2
:105EF0000964FF0912121212000912120A120A0A88
:105F0000130A1212121C1325131C131C1C251C250A
:105F10001C247625771C6E4848495109094948498F
:105F200049647740484949531C49485B520965090F
:105F3000495B5B09651B4A5249496E251C124800A2
:105F40006524251C5B406E5B5C5B5B535A77B7B77F
:105F5000B7BFB76EB7B7B7B7B7AEB6B6B6B7BFAE1F
:105F6000B7B7B7B7BF66AEB66EB7BF66656E6E6ED3
:105F7000BF66656E661C6E5BAD49484848BF5B40B6
:105F8000484848BFAD48484848BF4948484848B6CF
:105F90004848484848BF49484848486D49484848E3
:105FA00048AE48484848484848485BAEAE4848482C
:105FB0005B6D6548484809B6AE48484800AE65483C
:105FC000484800AE6548484801655D484849095C55
:105FD0005C4952080A131365645C5209015C5C5207
:105FE0004A0909AD6552494A09655B4A52534A65F7
:105FF0005C535B5B52655C53520901135C0A63ADF1
:10600000B60B0909B7B7B6000000096566000000C5
:106010000912130100535212B60100B7656EB701A1
:1060200052BF6DB76D000A645BAE64525BFFFFFF49
:10603000FF64B6BF6EB6AF656525B7B61D135C6568
:10604000130A1DBF65015C6F6E77B7657677B75B26
:10605000AE6EAF5CB764ADAEAD5BADFFFFBFFFBF73
:10606000BFAFB7B76F6F6E25656666665C1D5C1265
:106070001264131C125BACADAD66136EB7B6B6B747
:106080006E661D25256D656E256666BFFFB76E6E53
:106090006E6E6EFFAE1C6E666665132525130A5C78
:1060A000091C25B6B6B7AE5C65B66E66661C1325D0
:1060B0001D261D14136665251D14656E6E1D66660E
:1060C0005C651D66660A5B2E6E6E77766D6E6E760B
:1060D00077766E6E766D6E6D7F12131B1B1B1A5BCF
:1060E000ADBFBFB6ADB7B7B7B7B7BFAEAEB76EAFA0
:1060F000B76E6E6E6EB7B7252D1C52495377256467
:10610000090912766D5B0A65655B64010A13135B0E
:1061100009136509B6FF0A5D655CBF650A6E0A135F
:106120006D650A135CB7B614655D13655D5C135C41
:1061300065145C5C015CFF655CAEFF6E5B125BBF6F
:10614000B7FF5B09FF6E656E6EAEB75C5C5C656445
:106150005CAEB7B7B7B7B70A404848484865534937
:106160004848485C5C6D484848B76E0A004848BFDC
:10617000FFAD0952486DBFFF6D53485C53AE6D5281
:1061800048B7AEAD6D524848484848484848484826
:10619000484848484848484848484848484848487F
:1061A000484848484848484848484848484848486F
:1061B0004948484848490949526D1212B64909AD43
:1061C000AD6DFF49095CAD5CAD4864B7B7B6FE483C
:1061D00064B7645B5200126DAD645252121BADA4E1
:1061E00052120A0AAD5B00BF1200ADAE65FFAD09E9
:1061F000AEAE65AD5B00AEAE65FFAEA5B6AEAE5C55
:106200005B52B6B6B5535B52531109525253B76E37
:10621000095C65AE6FAE5C5C12AEB7B7B75C0A6581
:10622000BFFFB765126EB7FFB7640A65AEBFB7525E
:106230000AAEAEFFB7000AB7AEBFB7126DBFAEFF72
:10624000FF015CFFB6FFADB7BFB7B7B7B7B7FFFF8A
:10625000FFB7BF6EB7FF6EB7B76EB7BF6EB777AF9A
:10626000B7FF6EAFB7B7B7FFAE6EB7BFBFFFB7BF71
:10627000FFAEBFBFBFFFFFB76F65125353FFB7132A
:10628000536500FFAF65AEAE65BF6D5C5C5C5CBF27
:106290006E656565AEFF666EAE5C64FF6F650A098C
:1062A00013B7B76E010A1312131B1309125B6501B2
:1062B000125C526D6D65655C525C645C5C524AAE0A
:1062C0005D6E530A126E5C65136E645C0A12527640
:1062D0005C0A0A130A12656E666E6EB7B7AE6E6E12
:1062E0006EB7B7B7BFBFBFBFFFA55B5B64A4A5090F
:1062F0005C64111152646F6F6464BF5C64656565B2
:10630000655C09536E6E126553531C6E6E650A0A06
:106310000B2526AE0A0A0B1D65AD010A0B656E52F0
:10632000090A0B5C6E6E5C0A026DB7655C5C0A65FF
:10633000AE65660A0A65656E6E6E66666E66666650
:106340006566666565652566256E6E6E6E6E6E6643
:1063500066666D6E6E5D6E5DB7BF25656E1CB7F7C8
:10636000255D651CB7F725B6B6B7B7F6496665650E
:1063700065A5486665656E5B486E6E6E6E52486ECA
:106380006E6EBF524866256EB74948661DB6B6099F
:1063900048651DAEAE09484848484809094848497B
:1063A000011313484911125C1B480A5B5B1B1B4815
:1063B0000112131312480900125B5B4809015B5C70
:1063C0005B48090901125B120A0965520012121298
:1063D0000A01001213120A09000A5B12120A0900CC
:1063E000091212090952000909010965650100092C
:1063F000095309090A091213655C125C6D12B7652D
:10640000526F6E65B75C645C5C5B13AEB665001280
:106410006EAF12B75B095C5C0A5C0A120A0A0901DA
:1064200052525BAD64645C0953FFB7FFAD6565FF15
:1064300066BFAE5CB7FF66FFAE0AB7FFB7FF6D0180
:10644000ADAD5C645B0064525B5B5BFFFFFFFFFF15
:10645000FFB6B6ADAE6E6EB6B7B7B7FFB7B6B7B7E5
:10646000B7FFB7B7B7AEB7FFB7B7BFAEBFFFB75B42
:10647000646464656552645C5B5B5BFFFFFFFFBF48
:10648000BF66656E66666EB7B7AE135C13AFB7AE28
:106490001353136EB7B6121212B7B76501095365DD
:1064A000AE6501010912130A095B5BFFFFFF645B24
:1064B0005B66656EAEAEAE14131312656E130A12F0
:1064C00001AE5C0A0A0A135B09121209655C5B0AD9
:1064D0000A0A1212A55B5B5B5312525B5B5B5B5259
:1064E00052AE6EAE655C5C665B6E6F6F6E135C5C2D
:1064F0005C65655CA5655B115CAF535C6663656656
:106500005B5465656452120909535C525252525BE6
:106510005B5B5B5B5264521B6E09096565B6651275
:1065200001656565130A005C645C5B5209535C524B
:106530005B5309525352535B12121252125B1209EF
:10654000095212535209095D651CB7B71C6566658F
:10655000B7FF6D6565655D5C6E655C5C655D656519
:106560005C5C656565655C5C6565655B12121C1C41
:106570001C5B5B5B5B5C646525AEAD49486D65AEDD
:10658000B64948B66E65AD4948B66565644948B6D2
:106590006565654948B765655D4A486E655C6552E5
:1065A000485C5C145B524848484848484800000032
:1065B00000000048484848484848484848484899E2
:1065C0009999999999484848484848999999999921
:1065D0009999999999999948484848B65B0000005B
:1065E00000B65B48484848B65B48484848B65B999F
:1065F000999999B65B48484848B65B99999999B674
:106600005B99999999B65B000000000000000000BA
:10661000000000000000000000000000000000007A
:1066200048484848480000000000000048484848E2
:1066300048004848484848000000000000000000AA
:106640000000000000000000000000000000004802
:10665000484848484800000000000048484848486A
:1066600048484848484848B65B00004848B65B0080
:10667000000000B65B00004848B65B00004848B622
:106680005B00509999B65B00004848B65B00509992
:1066900099B65B005099994848484848480000001E
:1066A00000000048484848484848484848484899F1
:1066B0009999999999484848484848999999999930
:1066C000B699999999B6B64809090A135B00090960
:1066D0001B1B5B484948494949484848484848992C
:1066E0009999999999484848484848B6B6B6B6B66F
:1066F000B60000000000005C5B0A090909530A01AA
:106700000909094948484848484848484848489974
:106710009999999999484848484848B6B6B6B6B63E
:10672000B600000000000009535C5B530A090A0927
:10673000090A5B48484949494948484848484899EE
:106740009999999999484848484848B6B6B6B6B60E
:10675000B600000000000064B6ADB6AFAE5CB6B6E1
:10676000AEAEAE4949494949494848484848489920
:106770009999999999484848484848B6B6B6B6B6DE
:10678000B60000000000006EB6B76EAEAF64AE6536
:10679000656E6549494949494948484848484899C2
:1067A0009999999999484848484848B69999999922
:1067B00099B6B699999999AE6E1C0B1313656E5CD8
:1067C0001212124949494949494848484848489994
:1067D000999999999948484848484899999999990F
:1067E000999999999999991313130A0909531212AE
:1067F000120911494949494949484848484848996E
:1068000099999999994848484848489999999999DE
:1068100099999999999999090901095C52524900E4
:106820005B5B1249484849494948484848484899A3
:1068300099999999994848484848489999999999AE
:10684000B699999999B6B65212125309095252093A
:106850005B0A0949494849494848484848484899CD
:106860009999999999484848484848B6B6B6B6B6ED
:10687000B6000000000000126E6565656E095C14CC
:106880001C1C1C48494949494948484848484899B6
:106890009999999999484848484848B6B6B6B6B6BD
:1068A000B60000000000006D65BFB7B65A1C126448
:1068B000ADAD64494949494949484848484848991B
:1068C0009999999999484848484848B6B6B6B6B68D
:1068D000B600000000000048484848484809000049
:1068E00000000049484848484848484848484899AE
:1068F0009999999999484848484848B6B6B6B6B65D
:10690000B600000000000048484848484800000021
:10691000000000484848484848484848484848997E
:106920009999999999484848484848B699999999A0
:1069300099B6B69999999999999999B65B999999AE
:1069400099B65B99999999B65B99999999B65B991A
:10695000999999B65B99999999B65B99999999B6CC
:106960005B99999999B65B0048484848480048485F
:10697000484848004848484848004848484848006F
:106980004848484848004848484848004848484817
:1069900048004848484848B65B00509999B65B00A3
:1069A000509999B65B00509999B65B00509999B689
:1069B0005B00509999B65B00509999B65B0050996D
:1069C00099B65B0050999999999999B600999999B6
:1069D00099B60099999999B60099999999B600999B
:1069E000999999B60099999999B60099999999B6F2
:1069F0000099999999B60000B64099999900B640C6
:106A000099999900B64099999900B6409999990039
:106A1000B64099999900B64099999900B6409999CC
:106A20009900B64099999999999999B60099999927
:106A300099B60099999999B6B69999999999B699EB
:106A400099999999999999999999999999999999B6
:106A5000999999999999990000000000000000FF08
:106A60000000000000FFFF0000B600FF00FF004034
:106A700000FF0000FF9900FF00000099000000994E
:106A800000999999999999000000000000FF00FF72
:106A9000FFFFFFFF00FF000000FF00FFFFFF00FF00
:106AA00000FF000000FF00FFFFFFFF0000000000EC
:106AB0000099999999999900000000000000FF0041
:106AC0000000FF0000FF00FF00B60000FF00000014
:106AD00000FF00FF0000FF000000FF000000990021
:106AE0000099999999999900000000000000FFFF12
:106AF000FFFFFF000000FF0000B6B600FF00B60079
:106B00004000FF0040009900FF009900990000003C
:106B10009999999999999900B64099999900B6408F
:106B200099999900B640999999B640409999994098
:106B3000409999999999999999999999999999991E
:106B400099999999999999B65B00509999B65B0072
:106B5000509999B65B00509999B65B00509999B6D7
:106B60005B005099B6B65B0050B6B6B65B0050B647
:106B700000B65B0050B60099999999990099999936
:106B80009900009999999900FF9999999900FFB6F0
:106B9000B6B6B600FF0000000000000000000000D4
:106BA00000000000000000000000000000FFFF00E7
:106BB00000FF00000000FF00FF00FF00FFFFFF00DC
:106BC000FF00FF00FFFFFF00FF00FF0000000000CC
:106BD0000000000000000000000000000000FFFFB7
:106BE0000000FF00FF00FF00FF00FFFF0000FF00AC
:106BF000FF00FF00FF00FF00FF00FF00000000009B
:106C000000000000000000000099000000FF0000EC
:106C100000FF0000FF00FF00FFFF0000FFFFFF007C
:106C2000FF00FF00FFFF0000FF00FF00000000006A
:106C3000000000000000009900000000000000FFBC
:106C4000FF00FF00FF000000FF00FF00FF00FF004B
:106C5000FF00FF00FF0000FFFF00FF00000000003A
:106C600000000000000000000099999999FF009928
:106C7000999999000099999999FF00999999990082
:106C800000B6B6B6B6FF000000000000000000002D
:106C90000000000000000099999999999999999993
:106CA000999999999999999999999999999999B637
:106CB0009999999999B6B69999999900B6409999DF
:106CC0009900B64099999999999999999999999909
:106CD0009999999999999999999999999999999924
:106CE00099999999B699999999B6B699999999B6A0
:106CF0000099999999B60099999999B65B9999993A
:106D000099B65B99999999B65B99999999B65BB639
:106D1000999999B65BB6B69999B65B00B64099B6A3
:106D20005B00B64099B65BB65B00FFFFFFB65BFF4A
:106D30002F7FFFB6FF1F2F7FFFFF071F2F7FFFB69D
:106D4000FF1F2F7FFFB652FF2F7FFFB65B00FFFFB5
:106D5000FFB65B00505200FFFFFF99B65BFF7F2F2D
:106D6000FFB65BFF7F2F1FFF5BFF7F2F1F07FFFF1C
:106D70007F2F1FFF5BFF7F2FFF525BFFFFFF99B647
:106D80005B00524099B65B99999999B65B9999992C
:106D900099B6B6999999995BB699999999905B9991
:106DA00099999999489999999999999999999999A4
:106DB00099999999999999004848484848B6B6B61A
:106DC000B6B6B6B6B6B6B6B6B65B5B5B5B5B5B40FB
:106DD0000000000000905050505050999999999996
:106DE00099999999999999484848484848B6B6B6A2
:106DF000B6B6B6B6B6B6B6B6B65B5B5B5B5B5B000B
:106E000000000000005050505050509999999999A5
:106E100099999999999999B65B0050B600B65B001B
:106E200050B6B65B5B005099B65B004090999900F4
:106E300040489999995090999999999999999999BE
:106E40009999999999999900000000000000000013
:106E5000000000B6B6B6B6B6B640404040404099D5
:106E60009999999999999999999999999999999992
:106E70009999999999999900B640999999B6B64076
:106E8000999999B6404099999940409999999999B9
:106E90009999999999999999999999999999999962
:106EA0009999999999999999999999B600999999CE
:106EB00099B6B69999999999B699999999999999EB
:106EC0009999999999999999999999999999999932
:106ED0009999999999999900B64099B65BB6B64037
:106EE00099B6B6B64040995BB640409999905B9987
:106EF0009999999948999999999999999999999953
:106F000099999999999999B65B00509999B65B00AE
:106F10005099995B5B005099995B0040909999005A
:106F200040489999995090999999999999999999CD
:106F30009999999999999900000000000000000022
:106F40000000000000000000000000000000000041
:106F50000000000000000000000000000000000031
:106F6000000000000001160000000000000000000A
:106F70000000000000000000000000000000000011
:106F80000000000000000B170A00001517170A0088
:106F90000016171600011500000000000000000098
:106FA00000000000000000000000000000000000E1
:106FB00000000000000000010C161501151717173E
:106FC0001717171717171600000000000000000021
:106FD00000000000000000000000000000000000B1
:106FE000000000000000000000000001000B0A0B80
:106FF00017000A170B171700000000000000000020
:107000000000000000000000000000000000000080
:1070100000000000000A0C1516171717171717178E
:1070200017171717171615000000000000000000C2
:107030000000000000000000000000000000000050
:1070400000000000001717150B0000171717171581
:10705000000C0B0C161700000000000000000000E0
:1070600000000000000000010C0000000B171600DB
:10707000000A1717170000000B171500000A171554
:10708000000015171500000000000A170C00000B87
:10709000170B0B0A0C170A001716171717171717D5
:1070A00017171717170B0B0B16170C00000A1717DB
:1070B0000100001517171616170A0A1717171500DB
:1070C000171717170101171717171701150A0017B8
:1070D0000B000000000100000000000B0000000099
:1070E0000001000000000017150A1717010A000C24
:1070F000170C001501171600000015170A000B01E8
:1071000017160001170C170A0016161717000C1790
:1071100001171715170B0000161715171701170C75
:10712000161716151700000000170A0000000015BA
:107130000000000A17000000001617000000000BF6
:1071400017000000001616160B0B170A0015001684
:10715000160000000B1701010B0A17171717171756
:1071600017160C0B0A1717160B010017171717170E
:1071700016000A1517171700000015160000000C5E
:10718000170C0015171716000017160B000000004B
:1071900000000000000000000000000C01000000E2
:1071A0000017170C0000000C170C000000150B0056
:1071B00000000000000000000000000000000000CF
:1071C00000000000000000000000000000000000BF
:1071D0000000000000000013090C17140A2700002B
:1071E0000000002700525B52522700499B9B9B27BF
:1071F0000048484848270051A3A3A327009AACA3FE
:10720000A327009AA3A3AC142727271D0A00000078
:10721000000000525B5200525B9B9B5248529B48BD
:107220004848484848A3A39A519AA3A3ACA391A362
:10723000ACA39A51485AA30B17170C1327000A0A3C
:107240000000005249495B52009B9B9B9B5248485F
:107250004848484848A3A3A3A39A51A3A3A3ACA317
:1072600091A3ACA3A39A49271C000C170A000000A5
:10727000170C00525209090900529B5B5A9B524855
:107280004848484848919A9A9A9A9A9AA3A3A3A3DD
:10729000A3495AA3A3A3A30A0000000B15271C00AF
:1072A00000000100271C001C26000027262700489C
:1072B00000002700005108002700519A48002700CD
:1072C000519A480027009A171717092627090C1604
:1072D00001000000000052A45B49524852A4A44897
:1072E00048484848489A9151919A9AA39A919AA3EA
:1072F0009AA2A299A29A51272727272727000000A0
:107300000009095B5BA45BADADA4A4A452FFFF48D8
:10731000484848A4A49A9A9A919AA39A9A9A9AA3A6
:10732000AC494949494951272727272727090909EE
:10733000090900ADADADADAD49FFFFFFFFF649A4B2
:10734000A4A4A4A309A39A9AA39208ACACACAC9A47
:1073500048515252514900271C00001C27002700A9
:107360001C270000271C27000900272700095200BE
:107370002700499B9A002700A3ADAD002700A3ADCD
:10738000AD002700A4EDED272727272727000000C1
:107390000000004900495252524948495252525144
:1073A00048484848489A51919A9A9AA3919AA39A20
:1073B0009AA3999A51494927272727272700000090
:1073C000000000525249004952525249484952481D
:1073D00048484848489A9A9151919A9A9A9A919A0B
:1073E0009A49494948494927272727271C0000006F
:1073F00000002752525209002752525108002748D4
:1074000048480000279A9A9A4900279A9A9A490070
:107410002749494900002700001C272727001C276F
:107420000000001C270009525B2700099B9B9B0062
:107430000048484848005AA3A3A3A300A3A3A3A3BA
:10744000AC009AA3ACA3A327272727272700000077
:107450000000005200525B52525248529B9B9B4884
:1074600048484848489A519AA3A3A3A391A3A4A328
:10747000A39A494949494927272727272700000078
:10748000000000525B520049009B9B5248525248F8
:107490004848484848A3A39A51919AA3ACA3919A0B
:1074A000A3495AA399A2A31C00001C2727271C004C
:1074B00027000000271C2700A400002727005B48A6
:1074C00000002700489A4900270051A349002700DF
:1074D0005AA349002700492727272727270000000C
:1074E0000000005B5B5BA45B00A4A4A4A45248481A
:1074F00048484848489A9A9A9A91519A9A9A9A9AD8
:1075000091494949495199272727272727000000F2
:107510000000005BA45B5B5BA452A4A4A4A4A448E9
:107520004848484848919A9A9A9A9A9AA39A9A9A55
:10753000A3A2A2A3AC9A512727272727270009092E
:107540000909005BADADADAD5252FFFFFFF65248E9
:10755000A4A4A4A349919AA3A39A499AA3ACACA4C6
:1075600051494951515209271C2727272700270035
:1075700000000000270049524900270049525200EC
:107580002700519B9A00270052ADAD0027009AAD0D
:10759000F50027009AEDED27272727272700000071
:1075A0000000004949524900495252524948499AFB
:1075B0009B9A514848ADADAD9A5191ADADAD9A9100
:1075C0009AEDEDA4514849272727272727000000D7
:1075D000000000525252525249525252525249489D
:1075E00048484848489A9A9A9A9A919A9A9A9AA395
:1075F0009A49495152A2A227271C00001C000027CB
:107600001C0027000000271C2748490000272748A6
:10761000484800002751919A490027919A9A4900B9
:107620002799A29A49002727272727272700000004
:1076300000000000525B52525200499B9B9B5A0033
:1076400048484848480051A3A3A39B009AACA3A371
:10765000A3009AA3A3ACA327271C00001C000027AB
:10766000001C274900271C270009002727000900C4
:107670000027000048490027005AA349002700A31B
:10768000A3490027009AA3272727272727000000C0
:1076900000000009525B5200529B9B9B524852488B
:1076A0004848484848A3A3A39A5191A3A3ACA391E7
:1076B0009AACA3A39A494927272727272700000028
:1076C0000000005B52525B52009B9B9B9B524848C0
:1076D00048484848489A9A9A9A9151A3A3A3A39AD2
:1076E0009149494949494827272727271C00000075
:1076F0000000275BA45B49002752A4A34900274848
:107700004848000027919A9A4900279A9A9A490076
:107710002749494909002727009BA3ECFF27009B25
:10772000ACA3EC2700A3EDACAC27009BECECEC2762
:10773000009AA3A3A32700A3EDEDED2700A4F6F57F
:10774000F52700ADF6F6F6AC52000008A3A34900F9
:1077500027009BA451002700A4AC49002700A3A345
:10776000490027009AAC51002700A4AD5200270021
:10777000ACF652002709ADECFFECA35200A3ECA33A
:10778000A34900ACACACAC4900ECECECAC4900A3B8
:10779000A3A3A34900EDEDEDAC4900F5F5F5ED52DD
:1077A00000F6F6F6F652000009A3ACACAC2700A335
:1077B000ACACAC2700A3ACACAC27009BABABAB270D
:1077C000009AA3A3A32700A3ECECEC2700A3EDED04
:1077D000ED2709ADF6F6F6A248002709A3A3490054
:1077E00027009AA3490027009AA3490027009BA3DA
:1077F000490027009AA449002700A3AC49002700AC
:10780000A3B552002709ADA3A39AA35100A3A39A3D
:10781000A34900ACA3A2A34900ABA3A3A35100A317
:10782000A3A3A35A08ECACACECEDADEDEDACF5F6D2
:10783000F6F6F6F6F6FFFF00000000000027272707
:1078400027272727000000000027272727272700B2
:107850000000000008A3A3A4A3A3ACF6F6F6EDED88
:10786000F6FFFFFFF6F6FF000000000000272727C5
:107870002727270000000000002727271C000008FA
:107880000000270000A45200270000F65200270045
:1078900000F65200270000002700A4F5ED2727007E
:1078A000A4F5F5002700A4F5F5002700ACF5F500D8
:1078B0002700A4F6F5002708ACF6F6002709ACF679
:1078C000F6002709ADFFFFA39A51000000A39A49D3
:1078D000002727AC9A49002700ECA249002700ECBA
:1078E000A349002700EDA349002727EDA451002755
:1078F00000F6AD52002709000000000000272727EE
:107900002727270000000000000000000000000002
:10791000000000000027272727272700000000007D
:1079200000A4ADACA4ACAD000000000027272727C1
:107930002727270000000000270000000000270084
:107940000000000027272727272727000000000026
:1079500027ADADA4520027009BECFFECA3009BA336
:10796000ECA3A300A4ACACACAC00A3ECECECAC007E
:107970009AA3A3A3A300A4EDEDEDAD00ACF5F5F53E
:10798000F609ADF6F6F6F6520000000000490027B1
:107990002727274900270000004900270000004949
:1079A00000270000005200272727279B0900080016
:1079B00000F6F5ADADADAD0008A39AA3AC27009BD2
:1079C0009AA3AC2700A3A2A3AC27009BA3A3AB2739
:1079D000009AA3A3A32709A4ACACEC0952F5ACED23
:1079E000EDADF6F6F6F6F6A34900270000A3490030
:1079F000272727A44900270000A34900270000A348
:107A00004900270000AC4900270000AC51002700C6
:107A100000F65200270000000000000899272727E1
:107A200027009900000027009A00000027009A0014
:107A3000000027009A00000027009B00000027009C
:107A4000A30000002709A4A3A3ECFF5200A3A3A353
:107A5000AC4900A3ACA3A34900A3ABABA34900A3CB
:107A6000A3A3A34900ECEDEDAC5100F5F6F6F552F9
:107A700000F6FFFFF6520000000000000027272755
:107A8000272727270000000000270000000000270C
:107A90000000000000270000000000270000000098
:107AA000002700000000000027009BEDED272700C5
:107AB0009AF5F50027009BF5F5002700A3F5F500E2
:107AC0002700A3F5F5002700A3F6F6002700A4F68B
:107AD000F6002700ADFFFFF5F55A000000F5ED5266
:107AE000002727F5ED52002727F6F59B090000F542
:107AF000F6F5AC9A9AF6F6F6EDACACF6F6F6EDAC19
:107B0000EDFFFFFFF6F6F600000009A2A3272727E6
:107B1000009AA327272700A3A300000049ABA39A3C
:107B20009AA3A3A3A3ECECECECECACF5F5F5F5F51E
:107B3000A3F6F6F6F6F65B9AA3A25100279AA3A342
:107B4000490027A2A3A3490027A3A39B090027A3B9
:107B50009A490000279B4900002727490000271C5D
:107B6000270000271C0027009BA3ECFFAC009BAC68
:107B7000A3ECA300A3EDACACA4009BECECECAC003C
:107B80009AA3A3A3A300A3EDEDEDAC00A4F6F5F535
:107B9000AD00ADF6F6F6F6490027009BEC4900274C
:107BA000009BA351002700A4AC49002700A3EC4987
:107BB0000027009AA351002700A4ED52002700AC33
:107BC000F5520027005BF6FFECA3520000ECA3A3E4
:107BD000490027ACACAC490027ECECAC510027A322
:107BE000A3A35A0800EDEDEDECA3A3F5F5F6F5AC73
:107BF000EDF6F6F6F6F6F60000000000002727275F
:107C00002727270000000000002727272727270015
:107C10000000000000A3A3A3A3A39BEDEDEDEDEDF9
:107C2000ACF6F6F6F6F6F600000000002727272748
:107C300027271C00000000000027271C0000000070
:107C400000271C0000520000271C00ED9B000027AD
:107C50001CF6F6A40000272709ADFFFFFF2709AD9A
:107C6000FFFFFF2709ADFFFFFF2709ADFFFFFF273C
:107C700009ADFFFFFF2709ADFFFFFF2709ADFFFF9C
:107C8000FF2709ADFFFFFFF652002709ADF65200AE
:107C90002709ADF652002709ADF652002709ADF6C7
:107CA00052002709ADF652002709ADF65200270908
:107CB000ADF652002709ADFFFFFFF65200FFFFFFB0
:107CC000F65200FFFFFFF65200FFFFFFF65200FFE3
:107CD000FFFFF65200FFFFFFF65200FFFFFFF652D4
:107CE00000FFFFFFF65200FFFFFFFFFFFFFFFFFF58
:107CF000FFFFFFFFFFFFFFAD5BFFFFFFFF5B00FF2D
:107D0000FFFFF65200FFFFFFF65200FFFFFFFF5B91
:107D100000FFFFFFFFA409FFFFFFFFFFFFF6F6F6DE
:107D2000F6F6F6525252525252000000000000275E
:107D30002727272727270000000000272727272796
:107D400027090909090909F65200270000B652005F
:107D5000270000520900270000000000270000272C
:107D600027271C00000000000000002727272727E6
:107D700027090909090900002709ADFFFF002709A4
:107D8000ADFFFF002709ADFFFF002709ADFFFF0092
:107D90002709ADFFFF002709ADFFFF272709ADFF2A
:107DA000FF002709ADFFFFFFF652002709FFF6523B
:107DB000002709FFF652002709FFF652002709FFA6
:107DC000F652002700FFF652002700FFFF5B002756
:107DD00027FFFFA4090909ADFFFFFFFFFFADFFFF6C
:107DE000FFFFFFADFFFFFFFFFFADF6F6FFFFFF5206
:107DF0005252A4FFFF00000009FFFF27272709F6C2
:107E0000FF09090952FFFFFFFFF6520027FFFFF6A7
:107E1000520027FFFFF6520027FFFFF6520027FF10
:107E2000FFF6520027FFFFF6520027FFFFF6520031
:107E300027FFFFF652002709ADFFFFFFFF09ADFF47
:107E4000FFFFFF09ADFFFFFFFF09ADFFFFFFFF09C8
:107E5000ADFFFFFFFF09ADFFFFFFFF09ADFFFFFF14
:107E6000F609ADFFFFFFF6FFFFFFFFFFFFFFFFFF7C
:107E7000FFFFFFFFFFFFFFFFFFFFF7F6F6F6F6AD90
:107E80005B525252525B000000000052002727272D
:107E900027520027000000FFFFFFFFFFFFFFFFFF4B
:107EA000FFFFFFFFFFFFFFFFFFF6FFFFFFFFFF5298
:107EB000A4FFFFFFFF0009F6FFFFFF2709ADFFFF4B
:107EC000FF2709ADFFFFFFF65200270000F6520022
:107ED000270000F65200270000F65200270000F6A7
:107EE0005200270000F65200270000F6520027003B
:107EF00000F652002700000000002709AD00000036
:107F00002709AD0000002709AD0000002709AD00DA
:107F100000002709AD0000002709AD000000270977
:107F2000AD0000002709AD27000000000027000079
:107F3000990000270000E20000270000EA00002767
:107F400099EAFEEA99270000EA0000270000E20013
:107F500000270000990000002709ADFFFF00270956
:107F6000ADFFFF002709ADFFFF002709ADFFFF00B0
:107F70002709ADFFFF002709ADFFFF002709ADFF6F
:107F8000FF002709ADFFFFFFFFFFFFFFFFFFFFFF20
:107F9000FFFFFFFFFFFFFFF6F6FFFFAD5B5252FF53
:107FA000FF5B000000FFF652002727FFF652002774
:107FB00000FFF652002700FFFFFFFFF652FFFFFF12
:107FC000FFFFA4F6F6F6FFFFFF525252A4FFFF0098
:107FD000000009F7FF27272709ADFF00002709AD9B
:107FE000FF00002709ADFF00271C0000270900271C
:107FF0001C0027A40900271C27FFA409002727FF2E
:10800000FFA4000027FFFFF6520027FFFFF65200F3
:1080100027FFFFF652002709ADFFFFFFF609ADFF6E
:10802000FFFFF609ADFFFFFFF609ADFFFFFFF60901
:10803000ADFFFFFFF609ADFFFFFFF609ADFFFFFF44
:10804000F609ADFFFFFFF65200270009A4520027F2
:108050002700095200271C2700520027001C275226
:10806000002700001C52002700000052002727278D
:1080700027520027000909FFFFFFFFFFFFA4F6F6C4
:10808000F6F6F6005252525252000000000000274D
:10809000272727272700000000000027272727275A
:1080A00027090909090909FFFFFFFFFFFFF6F6F697
:1080B000FFFFFF525252A4FFFF00000009F6FF2706
:1080C000272709ADFF00002709ADFF27272709B69D
:1080D000FF09090952FFFF2709ADFFFFFF2709AD7F
:1080E000FFFFFF2709ADFFFFFF2709ADFFFFFF27B8
:1080F00009ADF6F6F6270052525252270000000052
:10810000001C2727272727F652002709ADF6520023
:108110002709ADF652002709ADF652002709ADAE8A
:1081200052002709AD520900270052000000270025
:10813000002727271C2727FFFFFFF65200FFFFFF1E
:10814000F65200FFFFFFF65200FFFFFFF65200F667
:10815000F6F6AE52005252525209000000000000E2
:1081600000272727272727F652002709ADF65200B8
:108170002709ADF6520027005BF65200270009AE32
:108180005200272700520900271C27000000270063
:108190001C2727271C0000FFFFFFFFFFFFFFFFFF3B
:1081A000FFFFFFFFFFFFFFFFFFA4FFFFFFFFFF0930
:1081B000A4F6F6F6F60000525252522700000000D4
:1081C000001C2727272727ADADADADADADFFFFFFC5
:1081D000FFFFFFFFFFFFFFFFFFFFFFFFFFFFFFF6B8
:1081E000F6F6F6F6F65252525252520000000000D5
:1081F00000272727272727ADADADADAD52FFFFFFE5
:10820000FFF652FFFFFFFFF652FFFFFFFFF652F6A9
:10821000F6F6F6AE525252525252090000000000D9
:1082200000272727272727002709ADFFFF00270959
:10823000ADFFFF002700A4FFFF00270009A4FF00F7
:1082400027270009A400271C2700000027001C275F
:1082500000271C00001C27FFFFFFFFADADFFFFFF45
:10826000FFFFFFFFFFFFFFFFFFFFFFFFFFFFFFF627
:10827000F6F6F6F6F6525252525252000000000044
:1082800000272727272727ADADF6FFFFFFFFFFFFBA
:10829000FFFFFFFFFFFFFFFFFFFFFFFFFFFFFFF6F7
:1082A000F6F6F6F6F6525252525252000000000014
:1082B00000272727272727FFFFF6520027FFFFF673
:1082C000520027FFFFAD490027FFAD52000027AD48
:1082D0005200002727490000271C270000271C0008
:1082E0002727271C00001C09ADFFFFFFF609ADFF83
:1082F000FFFFF609ADFFFFFFF609ADFFFFFFF6092F
:10830000ADF6F6F6AE005252525252000000000096
:108310000027272727272752002700000052002781
:108320000000005200270000005200270000005209
:1083300000270000000900270000000000270000BF
:108340000027271C000000F65200270000F652000C
:10835000270000F65200270000F65200270000AE6A
:1083600052002700005209002700000000002700EB
:10837000002727271C00000000002709AD0000008F
:108380002709AD0000002709AD0000002709AD0056
:1083900000002709AD000000270052000000270060
:1083A000000000001C272727000000000027000015
:1083B0000000002700000000002700000000002748
:1083C000000000000027000000000027000000005F
:1083D000001C0000000000002709ADFFFF00270976
:1083E000ADFFFF002709ADFFFF002709ADFFFF002C
:1083F0002709ADF6F6002700525252002700000070
:1084000000001C27272727FFF652002700FFF652FF
:10841000002700FFF652002700FFF652002700F663
:10842000AE5200270052520900270000000000272A
:1084300000272727271C0000002709ADFF00002781
:1084400009ADFF00002709ADFF00002709ADFF00BF
:10845000002709ADF6000027005252000027000057
:108460000000001C272727FFFFF6520027FFFFF61A
:10847000520027FFFFF6520027FFFFF6520027F6B3
:10848000F6AE5200275252520900270000000000A9
:108490002727272727272652002709ADAD52002777
:1084A00009ADFF52002709ADFF52002709ADFF5269
:1084B000002709ADF60900270052520000270000EE
:1084C0000027271C272727ADADB6FFFFFFFFFFFFC3
:1084D000FFFFFFFFFFFFFFFFFFFFFFFFFFFFFFF6B5
:1084E000F6F6F6F6F65252525252520000000000D2
:1084F00000272727272727FFFFF6520027FFFFF631
:10850000520027FFFFAD090027FFAD52000027AD45
:10851000520000271C090000271C000000271C0037
:108520000027271C00000028001C001A001D00ADB9
:1085300000AE00AE00AE00AE00AF001C001D001D7E
:108540000018001D001D001A001D001D001C001D4C
:10855000001D001D00B0001A001D001C001D001DA4
:10856000001D001D001D001D001D001D001A00AD96
:1085700000AE00AE00AE00AE00AF001D001D00B1A9
:10858000000000000000002200B2001D0016001DC7
:10859000001D001D001D001D001D00B300B4001DC6
:1085A000001800B500B6001D001D001D0016001DBE
:1085B000001D001C001D001D0016001D001D00B147
:1085C000000000000000001E00B2001D001600B1F7
:1085D0000000001E0000000000B2001D001D001D74
:1085E000001D001A001D001D001800B700B800B9DA
:1085F000001D001D00BA001D001D001C001D001DF7
:108600000018001D001A001D001D001D001C00B1F7
:10861000001E00000020000000B2001D001D00B17F
:10862000000000000024000000B2001D001D001822
:10863000001D001D001D0016001D001D001A001D5C
:1086400000BB00BC00BD00BE0018001D001D001DC9
:10865000001D001D001D001D0018001D001D00B1A3
:10866000000000000022002400B2001D001C00BF1A
:1086700000C000C100C200C300C4001D001D001DD9
:10868000001D0018001D001D001D001D00C5001D5F
:1086900000C600C700C800C9001C00CA001D001D9C
:1086A000001D0016001D001D001D001D001600BF4E
:1086B00000CB00C100C200C300CC001C001D00ADF7
:1086C00000CD00CE00CF00D000D100D200D300D426
:1086D00000CD00CD00D5001D001A001D00D600D72A
:1086E00000D800D900DA00DB001D00DC001D001AF4
:1086F000001D00AD00CD00CE00CF00D000D100D2D3
:1087000000D300DD00CD00CD00D5001D001D00DE32
:1087100000DF00E000DF00DF00DF00DF00DF00DF60
:1087200000E100E200E3001C001D00E400E500E6BB
:1087300000E700E800E900EA00EB00EC00ED001DB6
:10874000001D00DE00DF00DF00EE00DF00DF00E1E3
:1087500000DF00DF00DF00E200E3001D001800EF93
:1087600000000000000000240000002000000000C5
:108770000000000000E3001D001D00F000F100F209
:1087800000F300F400F500F600F700F800F9001D12
:10879000001C00EF0020000000000000002200008C
:1087A0000000001E0000002400E3001D001D00EF7B
:1087B00000000000001E0000002200000000000079
:1087C0000022000000E30018001D00FA00FB00FC7E
:1087D00000FD00FE00FF0000010101020103011D78
:1087E000001D00EF0000000000200000000000005D
:1087F000000000000000000000E3001C001A00EF71
:108800000020000000000000000000000000000048
:108810000000000000E3001D00040105010601073F
:1088200001080109010A010B010C010D010E011DD6
:10883000001800EF000000000000001E0000000013
:10884000000000000020000000E3001D001D00EFFC
:108850000000000000240000002000000000001EB6
:108860000000000000E3001D000F011001110112C3
:108870000113011401150116011701180119011C3A
:10888000001D00EF0000001E000000000000001EA0
:10889000000000240000000000E3001A011A011B80
:1088A000011C011D011D011D011D011D011D011DD9
:1088B000011D011D011E011F0120012101220123B3
:1088C000012401250126012701280129012A012B64
:1088D000012C011B011C011D011D011D011D011D9C
:1088E000011D011D011D011D011E01150015002D99
:1088F000012E011D001D001D001D001D001D001D7D
:10890000001D001D002F01300100000000000000CC
:1089100000310115001500300100000000000000CA
:108920000031012D012E011D001D001D001D001D27
:10893000001D001D001D001D002F01150015002D3C
:10894000012E011D001D001D001D001D001D001D2C
:10895000001D001D002F013001000000000000007C
:10896000003101150015003001000000000000007A
:108970000031012D012E011D001D001D001D001DD7
:10898000001D001D001D001D002F01150015002DEC
:10899000012E011D001D001D001D001D001D001DDC
:1089A000001D001D002F013001000000000000002C
:1089B000003101150015003001000000000000002A
:1089C0000031012D012E011D001D001D001D001D87
:1089D000001D001D001D001D002F01150015002D9C
:1089E000012E011D001D001D001D001D001D001D8C
:1089F000001D001D002F0132013301340135013605
:108A000001370115001500320133013401350136FB
:108A10000137012D012E011D001D001D001D001D2F
:108A2000001D001D001D001D002F01150015002D4B
:108A3000012E011D001D001D001D001D001D001D3B
:108A4000001D001D002F0115001500150015001553
:108A5000001500150015001500150015001500156E
:108A60000015002D012E011D001D001D001D001D03
:108A7000001D001D001D001D002F01150015002DFB
:108A8000012E011D001D001D001D001D001D001DEB
:108A9000001D001D002F0115001500150015001503
:108AA000001500150015001500150015001500151E
:108AB0000015002D012E011D001D001D001D001DB3
:108AC000001D001D001D001D002F01150015002DAB
:108AD000012E011D001D001D001D001D001D001D9B
:108AE000001D001D002F01150015001500150015B3
:108AF00000150015001500150015001500150015CE
:108B00000015002D012E011D001D001D001D001D62
:108B1000001D001D001D001D002F01150015002D5A
:108B2000012E011D001D001D001D001D001D001D4A
:108B3000001D001D002F0115001500150015001562
:108B4000001500150015001500150015001500157D
:108B50000015002D012E011D001D001D001D001D12
:108B6000001D001D001D001D002F01150015002D0A
:108B7000012E011D001D001D001D001D001D001DFA
:108B8000001D001D002F0115001500150015001512
:108B9000001500150015001500150015001500152D
:108BA0000015002D012E011D001D001D001D001DC2
:108BB000001D001D001D001D002F01150015002DBA
:108BC000012E011D001D001D001D001D001D001DAA
:108BD000001D001D002F01150015001500150015C2
:108BE00000150015001500150015001500150015DD
:108BF0000015002D012E011D001D001D001D001D72
:108C0000001D001D001D001D002F01150015002D69
:108C1000012E011D001D001D001D001D001D001D59
:108C2000001D001D002F0115001500150015001571
:108C3000001500150015001500150015001500158C
:108C40000015002D012E011D001D001D001D001D21
:108C5000001D001D001D001D002F01150015002D19
:108C6000012E011D001D001D001D001D001D001D09
:108C7000001D001D002F0115001500150015001521
:108C8000001500150015001500150015001500153C
:108C90000015002D012E011D001D001D001D001DD1
:108CA000001D001D001D001D002F01150015002DC9
:108CB000012E011D001D001D001D001D001D001DB9
:108CC000001D001D00380139013A013B013C013D06
:108CD000013E013F01400139013A013B013C013DA8
:108CE000013E0141012E011D001D001D001D001D42
:108CF000001D001D001D001D002F01150015002D79
:108D0000012E011D001D001D001D001D001D001D68
:108D1000001D001D004201000000000000000000D6
:108D200000000031013001000000000000000000E0
:108D300000000043012E011D001D001D001D001D2F
:108D4000001D001D001D001D002F01150015004411
:108D500001450146014601460146014601460146DC
:108D600001460146014701480148014801480148C0
:108D700001480149014A01480148014801480148A8
:108D80000148014B014501460146014601460146A5
:108D90000146014601460146014C0115001500152A
:108DA000001500150015001500150015001500151B
:108DB000001500150015001500150015001500150B
:108DC00000150015001500150015001500150015FB
:108DD00000150015001500150015001500150015EB
:108DE00000150015001500150015002100090000F0
:108DF0000000000000000000000000200000000053
:108E00000000000000000000000000000020000042
:108E10000000000000000000000000000022000030
:108E20000000000000000000000000000000000042
:108E3000000000200000004D014E014F0150015183
:108E40000152012400000000001E0000000000008C
:108E5000002200000000002400000000001E0000AE
:108E600000000020000000000000000000200000C2
:108E70000000000000000053015401550156015745
:108E800001580159012200000000000000200000EC
:108E9000000000000000001E0000000000000000B4
:108EA00000000000002200000000001E0000000082
:108EB0000022000000220000005A015B015C015DFD
:108EC000015E015F0160016101620163016401658E
:108ED0000166016701680169016A016B016C016D3E
:108EE000016E016F017001710172017301740175EE
:108EF00001760100001E00000000002000770178CC
:108F00000179017A017B017C017D017E017F018075
:108F10000181018201830184018501860187018825
:108F20000189018A018B018C018D018E018F0190D5
:108F300001910192012400000000001E0000009336
:108F4000019401950193019401960197019801996B
:108F5000019A019B019C019D019E019F01A001A11D
:108F6000019501A201A301A401A501A601A701A8E1
:108F700001A901AA019C01000000000000000000FE
:108F800000AB01AC01AD01AB01AE01AF01B001B16D
:108F900001B201B301B401B501B601B701AB01B82B
:108FA00001B901AD01BA01BB01BC01BD01BE01B6F1
:108FB00001BF01B001C001C1011E0000002400007A
:108FC000002200000000002000000000001E000041
:108FD0000024000000000000001E0000002200002D
:108FE000002400000000000000000000002000003D
:108FF000000000200000000000220000002400000B
:1090000000000000000000000000001E0000000042
:10901000000000000020000000000000002200000E
:10902000000000000000001E000000000000000022
:1090300000000020000000000022000000000000EE
:10904000000700040015002500260027002800293D
:10905000001500350036003700380039003A003B73
:10906000005100520053005400550056005700159F
:1090700000630064006500660067001500070004D7
:10908000001500150015002A001500150015001523
:10909000003C003D003E003F004000150015005818
:1090A0000059005A005B005C00150015006800695B
:1090B000006A006B006C0015000700040015001525
:1090C00000150015001500150015001500150041CC
:1090D000004200430015001500150015005D005EFC
:1090E000005F00150015001500150015001500158E
:1090F00000150015000700040015001500150015E7
:109100000015001500150015001500440045004627
:1091100000150015001500150060006100620015C3
:109120000015001500150015001500150015001597
:109130000005000200750076007700780079009441
:10914000009500960097009800050002007A007BC9
:10915000007C007D007E0099009A009B009C009D91
:1091600000050002007F0080008100820083009ED5
:10917000009F00A000A100A200050001002B002C10
:10918000002D002E002F00050001003000310032BC
:109190000033003400050001004700480049004A40
:1091A000004B00050001004C004D004E004F0050E8
:1091B000000500030015006D006E006F0070008454
:1091C000008500860087008800A300A400A500A6F3
:1091D00000A70005000300150015007300740015BA
:1091E0000015008E008F009000150015006800AC7F
:1091F00000150015000500030015001500150015E9
:10920000001500150091009200930015001500153F
:10921000001500150015000002060000FB00FF000D
:1092200000F405030C05040C05030C05040C0505EE
:109230000000FF00FF0002090000F10400F900FF38
:1092400000010A0000E2020105010103010101021F
:10925000050000FF0000E702030C04050000FF000A
:1092600000F100085A020403020404020405020487
:109270000602050000FF0001010007900000E2085F
:10928000050000FF0002080107C80106000100E711
:1092900000FF0001000007A00000EC0100FE00013B
:1092A0000100FF0001030000E203010604010903BD
:1092B000050000FF0002010107C80106000100ECE3
:1092C00000FF0002040000F10400F900FF000201A9
:1092D0000000F100FF0000ED00010602010100FFA7
:1092E0000000EC0001020107000207FF000103007B
:1092F000FF0002080007640100140500F700FF00EA
:1093000002090000F100FF0002040000F80008500C
:1093100003084E03085402084C02085802084A0188
:10932000085C0000FC03086003085A030860030897
:109330005A03086003085A01050000FF00020400F8
:1093400000FB00083E0103020103020103020103C6
:109350000201030201040A010302010302010302E4
:1093600001030201030201040201030201030201DD
:10937000030201030201030201040A0103020103C3
:1093800002010302010302010302010405010302B9
:1093900001030201030201030201030201040501AA
:1093A000030201030201030201030201030201049B
:1093B000050103020103020103020103020103028A
:1093C00001050000FF00020300085602040A02041F
:1093D0000802040602040402040200084202030513
:1093E000020402020305020305020402020305004F
:1093F00000F804030504040504030504040504033C
:109400000504040504030501050000FF0002040033
:1094100000FB0008340103020103040103060104F8
:109420000A01030201030401030601040A01030205
:109430000103040103060104050103020103040101
:1094400003060203020203040203060304050303E6
:1094500002030304030306040405040302040304D3
:1094600004030601050000FF0007000402040007D2
:10947000FF000990000A3C0000FB010850030305AF
:10948000030405030305030405030305030405039F
:10949000030503040503030503040503030503048F
:1094A0000503030503050000FF0007000402040094
:1094B00007FF000990000A3C0000FB01085303036A
:1094C000050304050303050304050303050304055D
:1094D0000303050304050303050304050303050350
:1094E000040503030503050000FF00070004020450
:1094F0000007FF000990000A3C0000FB010856032A
:10950000030503040503030503040503030503041E
:10951000050303050304050303050304050303050D
:1095200003040503030503050000FF000700040210
:10953000040007FF000990000A3C0000FB010859E5
:1095400003030503040503030503040503030503DF
:1095500004050303050304050303050304050303CE
:109560000503040503030503050000FF00020201D3
:1095700006000100E000FF0002010106000100E01A
:1095800000FF0002080106000100E000FF000205E4
:109590000106000100E000FF0002090106000100D1
:1095A000E000FF0000001792000000000000001F14
:1095B0009200000000000000339200000000000054
:1095C0000035920000000001000040920000000001
:1095D0000000005492000000000000005F920000B4
:1095E000000001000076920000000000000084925C
:1095F0000000000001000092920000000001000045
:10960000A39200000000000000B4920000000000DF
:109610000000C29200000000000000CD9200000097
:1096200000010000D59200000000010000E092005F
:10963000000000000000F19200000000000000FFA8
:1096400092000000000000000793000000000000EE
:10965000003C9300000000000000C59300000000E3
:109660000000000C9400000000000000689400005E
:109670000000000000A99400000000000000EA942F
:10968000000000000000002B95000000000000001A
:109690006C950000000000000077950000000000BD
:1096A00000008295000000000000008D9500000081
:1096B0000000000098950000000011241FBECFEFAD
:1096C000D0E1DEBFCDBF14BE88E10FB6F894809321
:1096D0006000109260000FBE11E0A0E0B1E0ECE786
:1096E000F5EF02C005900D92A830B107D9F71EE042
:1096F000A8E0B1E001C01D92AB3DB107E1F7F894DD
:10970000E9E0F1E080E090E020E802C021930196DA
:1097100032E08C309307D4F389E091E09093160304
:109720008093150310921703EAE1F3E080E090E0E4
:1097300003C0108201963A9684309105D4F3909339
:10974000480C8093470C91E090933A0390933B032D
:10975000909339031092810015BC8FEF87B984B9BB
:1097600080E88AB98CE081B983EF82B91092200C2D
:1097700086E08093210C109285001092840083E093
:10978000809389008DE88093880089E08093810030
:1097900082E080936F0082E484BD17BC95BD83E8AE
:1097A0008093B0001092B3009093B10081E185B92D
:1097B00078940E94ED4B0E94FA780C94BC7A0C9439
:1097C000000028E088E190E00FB6F894A895809317
:1097D00060000FBE209360000895EF92FF920F93F8
:1097E0001F9303E318E0C8010E94904C80E7E82E25
:1097F00080E0F82EC7010E940C5FC7010E94075F3E
:109800000E94805E8FE090E00E94C759C8010E94CC
:10981000904C41E06FEF80E00E940E5000EC17E0AA
:10982000A8016CE082E10E947A5983E090E00E94F6
:10983000C75944EF57E06CE082E10E947A5982E018
:1098400090E00E94C759A8016CE082E10E947A5919
:109850008EE190E00E94C7590E94805E84E190E012
:109860000E94C7591F910F91FF90EF90089590E0CB
:1098700025E130E0829FF001839FF00D929FF00D73
:109880001124E55BF34F61870895609339030895D0
:1098900090E025E130E0829FF001839FF00D929FE0
:1098A000F00D1124E55BF34F12861182089590E0CC
:1098B00025E130E0829FF001839FF00D929FF00D33
:1098C0001124E55BF34F81E0828B089590E025E160
:1098D00030E0829FF001839FF00D929FF00D1124E4
:1098E000E55BF34F6087089590E025E130E0829FCB
:1098F000F001839FF00D929FF00D1124E55BF34F73
:109900006483089590E025E130E0829FF001839F19
:10991000F00D929FF00D1124E55BF34F65830895E0
:109920009093A20C8093A10C8FE68093A70C1092C9
:109930000801EBE4FCE021E09FEF88E1208317823F
:10994000968313861182858375963CE0EF39F30781
:10995000A9F7089510924C0C1092610C1092760C9D
:1099600010928B0C01969093AB0C8093AA0C909361
:109970004A0C8093490C9093AE0C8093AD0C1092DE
:10998000A90C1092A80C1092A00C10929F0C10928F
:10999000A30C81E0809308011092A60C1092A50CF4
:1099A00008958091490C90914A0C0E94AA4C089508
:1099B0008091540C87FD03C08AEF8093540C8091F2
:1099C000690C87FD03C08AEF8093690C80917E0C3F
:1099D00087FD03C08AEF80937E0C8091930C87FDF6
:1099E00003C08AEF8093930C10920801089581E0E0
:1099F000809308010895DC01ED91FC911197AF016E
:109A00004F5F5F4F11965C934E93E4912E2F30E0A1
:109A1000E7FF13C02F7730703695322F2227379506
:109A20002795FA014F5F5F4FE4918E2F8F77280FB4
:109A3000311DE7FDF1CF4D935C93C90108958093EB
:109A4000A70C089508950E941F510895EF92FF9268
:109A50000F931F93CF93DF93182F062FF42EE22E30
:109A6000C82FD0E085E190E0C89FF001C99FF00DBC
:109A7000D89FF00D1124E55BF34F8285882321F0F8
:109A80008181882309F087C0EE2091F485E190E080
:109A9000C89FF001C99FF00DD89FF00D1124E55B20
:109AA000F34F128A8185882309F075C0178273C02D
:109AB000133059F481E091E090933B0380933A0393
:109AC00081E0809339030F2D08C060E0812F0E9450
:109AD0001F516F2D812F0E9400510F3799F485E19E
:109AE00090E0C89FF001C99FF00DD89FF00D1124A0
:109AF000E55BF34F8091A40C868785EA9CE0948B0C
:109B0000838B30C089E0089FC0011124E091A10C33
:109B1000F091A20CE80FF91F33964591549141152D
:109B2000510571F485E190E0C89FF001C99FF00DE7
:109B3000D89FF00D1124E55BF34F148A138A12C0ED
:109B4000FA01249185E190E0C89FF001C99FF00DD2
:109B5000D89FF00D1124E55BF34F26874F5F5F4FD1
:109B6000548B438B85E190E0C89FF001C99FF00DB5
:109B7000D89FF00D1124E55BF34F178611860387FC
:109B800011828FEF8087E782F282108A81E08287DC
:109B9000128A118A1482DF91CF911F910F91FF9049
:109BA000EF900895CF92DF92FF920F931F93CF9380
:109BB000DF93E3E5FCE08181282F332727FD3095F3
:109BC0008081280F311D2F3F310519F014F02FEF40
:109BD00030E0C90137FF02C080E090E080837596D5
:109BE0004CE0E73AF40739F780910801882309F03F
:109BF00019C135C1E091AA0CF091AB0C9F012F5F08
:109C00003F4F3093AB0C2093AA0C44914F3F69F522
:109C1000A9014F5F5F4F5093AB0C4093AA0CF90121
:109C200084918F3219F4109208010AC1863009F02C
:109C3000EAC0FA013196CF0101969093AB0C809364
:109C4000AA0CE491E33529F49093AE0C8093AD0C0B
:109C5000DAC0E53409F0D7C08091AD0C9091AE0C1C
:109C60009093AB0C8093AA0CCEC047FF02C04093E8
:109C7000A30C542F5F70842F90E0807F9070803B06
:109C8000910529F1803C910579F18039910509F020
:109C900042C0C9010196F901449101969093AB0C21
:109CA0008093AA0C0197FC012491852F90E08C9F52
:109CB000F0018D9FF00D9C9FF00D1124E55BF34F9B
:109CC0008081882309F49FC0220F638552C0C90197
:109CD0000196F901449101969093AB0C8093AA0CE4
:109CE0000197FC01249153C02F5F3F4F3093AB0C81
:109CF0002093AA0C21503040F9012491852F90E047
:109D00008C9FF0018D9FF00D9C9FF00D1124E55B61
:109D1000F34F238778C08091A30C582F5F7090E099
:109D2000807F9070803B910541F1803C910509F462
:109D30005EC08039910509F066C02F5F3F4F3093B8
:109D4000AB0C2093AA0C21503040F9012491852FAF
:109D500090E08C9FD0018D9FB00D9C9FB00D112481
:109D6000A55BB34F8C91882309F44DC0220F1B963D
:109D70006C91852F0E94264D46C02F5F3F4F309338
:109D8000AB0C2093AA0C21503040F90124914730AC
:109D900071F4852F90E08C9FF0018D9FF00D9C9FBA
:109DA000F00D1124E55BF34F220F26832CC04C35B8
:109DB00071F4852F90E08C9FF0018D9FF00D9C9F9A
:109DC000F00D1124E55BF34F220F24831CC04436B1
:109DD000D1F4852F90E08C9FF0018D9FF00D9C9F1A
:109DE000F00D1124E55BF34F220F25830CC0852F66
:109DF00090E08C9FF0018D9FF00D9C9FF00D112441
:109E0000E55BF34F43878AEA9CE00E94FB4C969502
:109E100087959093A90C8093A80C1092A00C109297
:109E20009F0C02C0C5E1D0E060919F0C7091A00C26
:109E30008091A80C9091A90C6817790709F4DACEE3
:109E40006F5F7F4F7093A00C60939F0C8091A50C67
:109E50009091A60C01969093A60C8093A50C0AE114
:109E600013E0CCE4DCE0FF24BFEFCB2ED12C8989BA
:109E7000882309F05EC08A899B89892B09F456C022
:109E80009E858D85981708F04CC050C08A852A8918
:109E90003B898F37E9F4D9018D91BB8BAA8B8F3F1A
:109EA00001F1F90161811196BB8BAA8BE82FF0E0DB
:109EB000EE0FFF1FE45CF74F0190F081E02D8F2D36
:109EC0000995EA89FB8981918D87FB8BEA8B28C0F4
:109ED000A9014F5F5F4F5B8B4A8BF90184918F3FE4
:109EE00021F418821B8A1A8A21C04F5F5F4F5B8B57
:109EF0004A8B41505040FA01649190E0880F991FBD
:109F0000845C974FFC01259134918F2DF9010995BF
:109F1000EA89FB893196FB8BEA8B3197E491ED87D7
:109F20001E869E858D85981709F4B0CF8E858F5F2C
:109F30008E878985882319F420E030E05DC08F8505
:109F40008F3F11F08F5F8F879E81992309F44EC058
:109F50002F81222309F44AC08D81882309F446C049
:109F60004091A70C442309F441C0899FC0011124EA
:109F700080509F4F892F992730E0BC01629FC0011C
:109F8000639F900D729F900D112480509F4F892FD9
:109F90009927242F30E0FC01E29FC001E39F900D40
:109FA000F29F900D112480509F4F292F33278B81D2
:109FB0008823F1F0EA81F0E0E050FB45E491E058BD
:109FC000E89FC001112480509F4F892F9927A60137
:109FD000481B590B429FC001439F900D529F900D0B
:109FE000112480509F4F292F332702C020E030E0FA
:109FF0008A819C81890F8A83F8012083F394065F0C
:10A000001F4F6596F4E0FF1609F031CFDF91CF9135
:10A010001F910F91FF90DF90CF9008951F93CF93E2
:10A02000DF93582F89E0589FC00111242091A10C83
:10A030003091A20C280F391FC9010396FC01A5918C
:10A04000B491F90184918150823010F413E01DC065
:10A050008091610C8823B1F080916C0C851711F40C
:10A06000442381F48091760C882371F08091810CD7
:10A07000851711F4442341F49091700C8091850C64
:10A08000891710F411E001C012E0212F30E0FD012A
:10A09000449185E190E0289FE001299FD00D389FF1
:10A0A000D00D1124C55BD34F4E871196BC8BAB8B63
:10A0B0001F8680E58A836F838FEF888719861A8AC7
:10A0C000188A21E02A87198A5C8729831C82133029
:10A0D00049F481E091E090933B0380933A0320930D
:10A0E000390308C060E5812F0E9400516989812FE2
:10A0F0000E941F51DF91CF911F910895FF920F93FE
:10A100001F93082FF62E0E94005110E085E190E089
:10A11000089FF001099FF00D189FF00D1124E55BD9
:10A12000F34FF2821F910F91FF900895962F482FC1
:10A1300050E025E130E0429FF001439FF00D529F37
:10A14000F00D1124E55BF34F6281691B62830E946D
:10A1500000510895482F50E025E130E0429FF00182
:10A16000439FF00D529FF00D1124E55BF34F928158
:10A17000690F62830E9400510895000000000000F2
:10A1800000000000000000000000000000000000CF
:10A1900000000000000000000000000000000000BF
:10A1A00000000000000000000000000000000000AF
:10A1B000000000000000000000000000000000009F
:10A1C000000000000000000000000000000000008F
:10A1D000000000000000000000000000000000007F
:10A1E000000000000000000000000000000000006F
:10A1F000000000000000000000000000000000005F
:10A2000099277727833008F00895E0E0FFEA660F8A
:10A21000771FE60FF71FA591B491EAE1F3E02AE07A
:10A22000289FE00DF11DA183B28311240895909120
:10A2300039039170880F892B8093390308959927EA
:10A240007727EAE1F3E02AE0289FE00DF11D6E3F59
:10A2500031F4609139036E7F609339030BC06F3F17
:10A2600031F4609139036E6F6093390303C075EA6E
:10A27000760F75831124089599277727EAE1F3E093
:10A280002AE0289FE00DF11D6083112408952F938B
:10A290003F934F935F936F937F938F939F93AF936E
:10A2A000BF93789411240E94735D0E94D24D2F9227
:10A2B0003F924F925F926F927F928F929F92AF9256
:10A2C000BF92CF92DF92EF92FF920F931F93CF93A3
:10A2D000DF9300901703002019F4A9E0B1E002C059
:10A2E000AFE0B2E001E000260092170302E0009325
:10A2F00018035091380360913A0370913B038091A9
:10A300003C0320901B0330901C0340901E03509090
:10A310001F0360901D0310911A0370902503809015
:10A32000260390902703A0902803B0902903209142
:10A330002403C0902F03D0903003E0903203F090BC
:10A3400033030091310330912E039FEF620C431CC5
:10A35000F2014491410300240008C12DD02D970C37
:10A36000A81CF5014491420300240008C10DD01D32
:10A370000C0DED1CF7014491430300240008C10DAE
:10A38000D01D8A956AF440913903842F8695062E54
:10A390000694062600FA7695679576F940FF66F9E9
:10A3A00040E860FD4FE7450300240008C10DD01DC3
:10A3B0000024C038D0050CF0CFE70A94C038D0058F
:10A3C0000CF4C0E8C058CD939A9509F0BFCF4091E6
:10A3D00018034A954093180397E009F0B7CF6092AD
:10A3E0001D0340921E0390922703A092280300931E
:10A3F0003103E092320360933A0370933B038093FE
:10A400003C03DF91CF911F910F91FF90EF90DF9070
:10A41000CF90BF90AF909F908F907F906F905F9004
:10A420004F903F902F9099278091200C7727609133
:10A43000210C11240E94224DBF91AF919F918F91C9
:10A440007F916F915F914F913F912F9108950C945F
:10A4500029520C942B520F931F932ABDE0911503A0
:10A46000F0911603019100000093B30003E0E53181
:10A47000F00710F40000000010F0E9E0F1E0E093D4
:10A480001503F0931603C895C895C895C895C89547
:10A49000C8950000000000002AB51F910F91089593
:10A4A0000000E091210CE0FFD6CFE1E1EA95F1F761
:10A4B00000000000089500000000000000000000FF
:10A4C000000000000000000000000000000000008C
:10A4D000000000000000000000000000000000007C
:10A4E000000000000000000000000000000000006C
:10A4F000000000000000000000000000000000005C
:10A50000000306090C101316191C1F2225282B2ED8
:10A51000313336393C3F414447494C4E51535558ED
:10A520005A5C5E60626466686A6B6D6F70717374AA
:10A53000757678797A7A7B7C7D7D7E7E7E7F7F7F63
:10A540007F7F7F7F7E7E7E7D7D7C7B7A7A79787649
:10A5500075747371706F6D6B6A68666462605E5C5F
:10A560005A585553514E4C494744413F3C39363374
:10A57000312E2B2825221F1C191613100C09060337
:10A5800000FDFAF7F4F0EDEAE7E4E1DEDBD8D5D23E
:10A59000CFCDCAC7C4C1BFBCB9B7B4B2AFADABA809
:10A5A000A6A4A2A09E9C9A9896959391908F8D8C2C
:10A5B0008B8A888786868584838382828281818153
:10A5C0008181818182828283838485868687888A4D
:10A5D0008B8C8D8F9091939596989A9C9EA0A2A417
:10A5E000A6A8ABADAFB2B4B7B9BCBFC1C4C7CACDE2
:10A5F000CFD2D5D8DBDEE1E4E7EAEDF0F4F7FAFDFF
:10A60000808182838485868788898A8B8C8D8E8FD2
:10A61000909192939495969798999A9B9C9D9E9FC2
:10A62000A0A1A2A3A4A5A6A7A8A9AAABACADAEAFB2
:10A63000B0B1B2B3B4B5B6B7B8B9BABBBCBDBEBFA2
:10A64000C0C1C2C3C4C5C6C7C8C9CACBCCCDCECF92
:10A65000D0D1D2D3D4D5D6D7D8D9DADBDCDDDEDF82
:10A66000E0E1E2E3E4E5E6E7E8E9EAEBECEDEEEF72
:10A67000F0F1F2F3F4F5F6F7F8F9FAFBFCFDFEFF62
:10A68000000102030405060708090A0B0C0D0E0F52
:10A69000101112131415161718191A1B1C1D1E1F42
:10A6A000202122232425262728292A2B2C2D2E2F32
:10A6B000303132333435363738393A3B3C3D3E3F22
:10A6C000404142434445464748494A4B4C4D4E4F12
:10A6D000505152535455565758595A5B5C5D5E5F02
:10A6E000606162636465666768696A6B6C6D6E6FF2
:10A6F000707172737475767778797A7B7C7D7E7FE2
:10A7000000020406080A0C0E10121416181A1C1E59
:10A7100020222426282A2C2E30323436383A3C3E49
:10A7200040424446484A4C4E50525456585A5C5E39
:10A7300060626466686A6C6E70727476787A7C7E29
:10A740007F7D7B79777573716F6D6B696765636109
:10A750005F5D5B59575553514F4D4B4947454341F9
:10A760003F3D3B39373533312F2D2B2927252321E9
:10A770001F1D1B19171513110F0D0B0907050301D9
:10A78000FFFDFBF9F7F5F3F1EFEDEBE9E7E5E3E1C9
:10A79000DFDDDBD9D7D5D3D1CFCDCBC9C7C5C3C1B9
:10A7A000BFBDBBB9B7B5B3B1AFADABA9A7A5A3A1A9
:10A7B0009F9D9B99979593918F8D8B898785838199
:10A7C00080828486888A8C8E90929496989A9C9E99
:10A7D000A0A2A4A6A8AAACAEB0B2B4B6B8BABCBE89
:10A7E000C0C2C4C6C8CACCCED0D2D4D6D8DADCDE79
:10A7F000E0E2E4E6E8EAECEEF0F2F4F6F8FAFCFE69
:10A800007F7F7F7F7F7F7F7F7F7F7F7F7F7F7F7F58
:10A810007F7F7F7F7F7F7F7F7F7F7F7F7F7F7F7F48
:10A820007F7F7F7F7F7F7F7F7F7F7F7F7F7F7F7F38
:10A830007F7F7F7F7F7F7F7F7F7F7F7F7F7F7F7F28
:10AB00000309131E28313A40464C5054585B5E618D
:10AB1000636567696B6C6E6F70717273747576774D
:10AB2000777879797A7A7B7B7C7C7C7D7D7D7E7E73
:10AB30007E7E7F7F7F7F7F7F7F7F7F7F7F7F7F7F27
:10AB40007F7F7F7F7F7F7F7F7F7F7F7F7F7E7E7E18
:10AB50007E7D7D7D7C7C7C7B7B7A7A79797877774A
:10AB6000767574737271706F6E6C6B696765636113
:10AB70005E5B5854504C46403A31281E130903007E
:10AB8000C6CCD5DBDFE3E5E7E9EAEBECEDEEEFEF92
:10AB9000F0F0F0F1F1F1F1F2F2F2F2F2F2F2F2F39E
:10ABA000F3F3F3F3F3F3F3F3F3F3F3F3F3F3F3F375
:10ABB000F3F3F3F3F3F3F3F3F3F3F3F3F3F3F3F365
:10ABC000F3F3F3F3F3F3F3F3F3F3F3F3F3F3F3F355
:10ABD000F3F3F3F3F3F3F3F3F3F3F3F3F3F3F3F345
:10ABE000F2F2F2F2F2F2F2F2F1F1F1F1F0F0F0EF52
:10ABF000EFEEEDECEBEAE9E7E5E3DFDBD5CCC60011
:10AC000000283D42302D2C2B2C2D2E2F3032333569
:10AC100037393B3D3F414345484A4C4E50535557C9
:10AC2000595B5D5F61636567696B6C6E70717374AE
:10AC3000757778797A7B7C7D7D7E7E7F7F7F7F7F55
:10AC40007F7F7F7F7F7F7E7E7D7D7C7B7A7978773B
:10AC500075747371706E6C6B69676563615F5D5B62
:10AC600059575553504E4C4A484543413F3D3B3957
:10AC700037353332302F2E2D2C2B2C2D30423D28C2
:10AC800000E9E5FED4D7D7D7D6D4D2D0CECCCAC827
:10AC9000C6C3C1BFBDBAB8B6B4B1AFADABA9A7A565
:10ACA000A3A19F9E9C9A999795949391908F8D8C38
:10ACB0008B8A898888878685858484848383838337
:10ACC0008383838383848484858586878888898A2F
:10ACD0008B8C8D8F909193949597999A9C9E9FA120
:10ACE000A3A5A7A9ABADAFB1B4B6B8BABDBFC1C338
:10ACF000C6C8CACCCED0D2D4D6D7D7D7D4FEE5E9F1
:10AD0000F9F8F9F5EBE1DDDEE0E2E4E5E6E5E4E2C1
:10AD1000DED9D2CAC1B7ACA299918A8683818080DC
:10AD20008182838586888A8C8D8F90929395969761
:10AD300098999A9B9B9C9D9D9D9E9E9E9F9F9F9F49
:10AD40009F9F9F9E9E9E9D9D9D9C9B9B9A99989741
:10AD500096959392908F8D8C8A8886858382818048
:10AD6000808183868A9199A2ACB7C1CAD2D9DEE22A
:10AD7000E4E5E6E5E4E2E0DEDDE1EBF5F9F8F90033
:10AD80000708070B151F2322201E1C1B1A1B1C1E45
:10AD900022272E363F49545E676F767A7E7F7F7F0B
:10ADA0007F7E7D7B7A7876747371706E6D6B6A6965
:10ADB000686766656564646363626262616161615C
:10ADC0006161616262626363636465656667686945
:10ADD0006A6B6D6E7071737476787A7B7D7E7F7F1F
:10ADE0007F7F7E7A766F675E54493F362E27221E1C
:10ADF0001C1B1A1B1C1E2022231F150B07080700F3
:10AE00001F313D444E5354565A5F64696E747679CF
:10AE10007C7F7F7F7F7F7F7F7F7F7F7F7F7F7F7F45
:10AE20007F7F7F7F7F7F7F7F7F7F7F7F7F7F7F7F32
:10AE30007F7F7F7F7F7F7F7F7F7F7F7F7F7F7F7F22
:10AE40007F7F7F7F7F7F7F7F7F7F7F7F7F7F7F7F12
:10AE50007F7F7F7F7F7F7F7F7F7F7F7F7F7F7F7F02
:10AE60007F7F7F7F7F7F7F7F7F7F7F7F7F7F7F7FF2
:10AE70007F7F7F7F7F7F7F7F7F7F7F7C7871684C44
:10AE80002C1C120C0A0B0A05FDF3E9DFD4CAC0B76B
:10AE9000AEA69E97918B8685828080808080808000
:10AEA00080808080808080808080808080808080A2
:10AEB0008080808080808080808080808080808092
:10AEC0008080808080808080808080808080808082
:10AED0008080808080808080808080808080808072
:10AEE0008080808080808080808080808080808062
:10AEF000808080808087919DACC4CBD4DDF2FAFA4B
:10AF000022002400260028002B002D0030003300F2
:10AF1000360039003D004000440048004C0051001C
:10AF200056005B00600066006C00730079008100D1
:10AF3000880090009900A200AC00B600C100CC00CF
:10AF4000D800E500F30001011001210132014401A4
:10AF500057016C0181019801B001CA01E5010202AB
:10AF60002102410264028802AE02D70203033003C9
:10AF700061039403CB03050442048304C704100552
:10AF80005D05AF0505066106C20629079607090893
:10AF9000830805098E09200ABA0A5D0B0A0CC10C48
:10AFA000840D510E2B0F121007110A121D1340149D
:10AFB0007415BA1614188319071BA31C571E2420D6
:10AFC0000E22142439267F28E82A752D29300633CD
:10AFD0000F364539AD3C49401B442848734CFE5060
:10AFE000CF55EA5A51600C661D6C8B725A7992806B
:10AFF00037885090E598FDA19FABD3B5A3C0000062
:10B000001F93CF93DF93FA01549131961491C52F7A
:10B01000D0E09F012F5F3F4F70E095E0660F771FF4
:10B020009A95E1F7680F711D40E00FC084918C93F1
:10B0300011961C9211979F5F319612969517B0F357
:10B040004F5F2C0F3D1F605E7F4F411740F4DB01C7
:10B05000AA0FBB1FA05ABC4FF90190E0EFCFDF91C0
:10B06000CF911F9108958F929F92AF92BF92CF92EE
:10B07000DF92EF92FF920F931F93CF93DF93882E6F
:10B08000962E5A016901F02E00E010E080EEF80ED5
:10B090000CC04F2D6E2D882D8C0F0E94D05E2196F6
:10B0A000CA15DB05B4F30F5F1F4F0C151D052CF4FB
:10B0B000C0E0D0E0E02EE90CF3CFDF91CF911F91FB
:10B0C0000F91FF90EF90DF90CF90BF90AF909F9047
:10B0D0008F90089540520E94D05E0895FF920F9382
:10B0E0001F93CF93DF938C01F62EEA01FE0144916A
:10B0F0002196442349F0802F0F5F1F4F4F77405216
:10B100006F2D0E94D05EF2CFDF91CF911F910F91F2
:10B11000FF900895FF920F931F93182F062FF42E80
:10B1200042954F704A3010F4405F01C0495E602F75
:10B13000812F0E94D05E4F2D4F70812F8F5F4A303C
:10B1400010F4405F01C0495E602F0E94D05E1F91E5
:10B150000F91FF900895FF920F931F93F82E162FD3
:10B16000042F452F0E948A58402F612F8F2D8E5F0C
:10B170000E948A581F910F91FF900895EF92FF92BD
:10B180000F931F93F62E042F182F28E0E22EE80EBF
:10B1900007FF02C041E101C040E16F2D812F0E94F5
:10B1A000D05E1F5F1E1511F0000FF2CF1F910F919F
:10B1B000FF90EF900895FF920F931F93CF93DF932B
:10B1C000F62E042FEC0110E0002311F4112339F4C2
:10B1D000802F6AE00E94F679905F492F01C040E01D
:10B1E0006F2D8C2F0E94D05E1F5F2197133031F09E
:10B1F000802F6AE00E94F679082FE6CFDF91CF9189
:10B200001F910F91FF900895CF92DF92EF92FF92DE
:10B210000F931F93CF93DF93C62E79018A01EC0120
:10B22000DD24E114F1040105110511F4DD2059F4C8
:10B23000C801B7012AE030E040E050E00E94157AF2
:10B24000462F405F01C040E06C2D8C2F0E94D05EE5
:10B25000D394219786E0D81669F0C801B7012AE097
:10B2600030E040E050E00E94157AC901DA017C012B
:10B270008D01D7CFDF91CF911F910F91FF90EF906C
:10B28000DF90CF9008957F928F929F92AF92BF925E
:10B29000CF92DF92EF92FF920F931F93CF93DF93A2
:10B2A000782E862E5A016901780100E010E00CC06A
:10B2B000A701692D872D8C0F0E94E85E2196CA1583
:10B2C000DB05B4F30F5F1F4F0C151D052CF4C0E018
:10B2D000D0E0902E980CF3CFDF91CF911F910F917A
:10B2E000FF90EF90DF90CF90BF90AF909F908F90A6
:10B2F0007F9008957F928F929F92AF92BF92CF924C
:10B30000DF92EF92FF920F931F93CF93DF93782EEC
:10B31000862EEA01FA01C590D490FA013296A590E2
:10B32000B49000E016C0FC01EE0DFF1D3296EE0F4A
:10B33000FF1FEC0FFD1F45915491692D812F870D43
:10B340000E94E85E1F5F812F90E08C159D055CF3E5
:10B350000F5F802F90E08A159B055CF48C9D700137
:10B360008D9DF00C9C9DF00C112410E0902E980CFB
:10B37000EACFDF91CF911F910F91FF90EF90DF9077
:10B38000CF90BF90AF909F908F907F9008950F9334
:10B390001F93CF93DF938C01C0E0D0E007C00E94E1
:10B3A000115F8823E1F30E94145F2196C017D10733
:10B3B000B4F3DF91CF911F910F9108953E5E485EE7
:10B3C000565E615DEEEDC8950000EA95E1F700007C
:10B3D00000000000000000000000C0E6D3E000EE26
:10B3E000A02E662776E03BD434E23A95F1F70E942E
:10B3F000295A3FE03A95F1F70000AA94A9F000001D
:10B40000639500000000683029F0C895C895C8957C
:10B410000000E9CF6627002430E5C30FD01D0000EF
:10B42000000000000000DFCFC895C895C895C895FA
:10B43000C8950000000013D411E00091230C0127EF
:10B440000093230C00FF1093220CE2E0E0933600FF
:10B4500008958F939F93DE01679FC00100004D9177
:10B460005D91480F591FFA01059108B94D91059159
:10B4700008B95D91059108B900C0059108B900C0EF
:10B48000059108B9480F591F059108B90000FA0144
:10B49000059108B94D91059108B95D91059108B9DB
:10B4A00000C0059108B900C0059108B9480F591F9F
:10B4B000059108B90000FA01059108B94D9105916F
:10B4C00008B95D91059108B900C0059108B900C09F
:10B4D000059108B9480F591F059108B90000FA01F4
:10B4E000059108B94D91059108B95D91059108B98B
:10B4F00000C0059108B900C0059108B9480F591F4F
:10B50000059108B90000FA01059108B94D9105911E
:10B5100008B95D91059108B900C0059108B900C04E
:10B52000059108B9480F591F059108B90000FA01A3
:10B53000059108B94D91059108B95D91059108B93A
:10B5400000C0059108B900C0059108B9480F591FFE
:10B55000059108B90000FA01059108B94D910591CE
:10B5600008B95D91059108B900C0059108B900C0FE
:10B57000059108B9480F591F059108B90000FA0153
:10B58000059108B94D91059108B95D91059108B9EA
:10B5900000C0059108B900C0059108B9480F591FAE
:10B5A000059108B90000FA01059108B94D9105917E
:10B5B00008B95D91059108B900C0059108B900C0AE
:10B5C000059108B9480F591F059108B90000FA0103
:10B5D000059108B94D91059108B95D91059108B99A
:10B5E00000C0059108B900C0059108B9480F591F5E
:10B5F000059108B90000FA01059108B94D9105912E
:10B6000008B95D91059108B900C0059108B900C05D
:10B61000059108B9480F591F059108B90000FA01B2
:10B62000059108B94D91059108B95D91059108B949
:10B6300000C0059108B900C0059108B9480F591F0D
:10B64000059108B90000FA01059108B94D910591DD
:10B6500008B95D91059108B900C0059108B900C00D
:10B66000059108B9480F591F059108B90000FA0162
:10B67000059108B94D91059108B95D91059108B9F9
:10B6800000C0059108B900C0059108B9480F591FBD
:10B69000059108B90000FA01059108B94D9105918D
:10B6A00008B95D91059108B900C0059108B900C0BD
:10B6B000059108B9480F591F059108B90000FA0112
:10B6C000059108B94D91059108B95D91059108B9A9
:10B6D00000C0059108B900C0059108B9480F591F6D
:10B6E000059108B90000FA01059108B94D9105913D
:10B6F00008B95D91059108B900C0059108B900C06D
:10B70000059108B9480F591F059108B90000FA01C1
:10B71000059108B94D91059108B95D91059108B958
:10B7200000C0059108B900C0059108B9480F591F1C
:10B73000059108B90000FA01059108B94D910591EC
:10B7400008B95D91059108B900C0059108B900C01C
:10B75000059108B9480F591F059108B90000FA0171
:10B76000059108B94D91059108B95D91059108B908
:10B7700000C0059108B900C0059108B9480F591FCC
:10B78000059108B90000FA01059108B94D9105919C
:10B7900008B95D91059108B900C0059108B900C0CC
:10B7A000059108B9480F591F059108B90000FA0121
:10B7B000059108B94D91059108B95D91059108B9B8
:10B7C00000C0059108B900C0059108B9480F591F7C
:10B7D000059108B90000FA01059108B94D9105914C
:10B7E00008B95D91059108B900C0059108B900C07C
:10B7F000059108B9480F591F059108B90000FA01D1
:10B80000059108B94D91059108B95D91059108B967
:10B8100000C0059108B900C0059108B9480F591F2B
:10B82000059108B90000FA01059108B94D910591FB
:10B8300008B95D91059108B900C0059108B900C02B
:10B84000059108B9480F591F059108B90000FA0180
:10B85000059108B94D91059108B95D91059108B917
:10B8600000C0059108B900C0059108B9480F591FDB
:10B87000059108B90000FA01059108B94D910591AB
:10B8800008B95D91059108B900C0059108B900C0DB
:10B89000059108B9480F591F059108B90000FA0130
:10B8A000059108B94D91059108B95D91059108B9C7
:10B8B00000C0059108B900C0059108B9480F591F8B
:10B8C000059108B90000FA01059108B94D9105915B
:10B8D00008B95D91059108B900C0059108B900C08B
:10B8E000059108B9480F591F059108B90000FA01E0
:10B8F000059108B94D91059108B95D91059108B977
:10B9000000C0059108B900C0059108B9480F591F3A
:10B91000059108B90000FA01059108B94D9105910A
:10B9200008B95D91059108B900C0059108B900C03A
:10B93000059108B9480F591F059108B90000FA018F
:10B94000059108B94D91059108B95D91059108B926
:10B9500000C0059108B900C0059108B9480F591FEA
:10B96000059108B90000FA01059108B94D910591BA
:10B9700008B95D91059108B900C0059108B900C0EA
:10B98000059108B9480F591F059108B90000FA013F
:10B99000059108B94D91059108B95D91059108B9D6
:10B9A00000C0059108B900C0059108B9480F591F9A
:10B9B000059108B90000FA01059108B94D9105916A
:10B9C00008B95D91059108B900C0059108B900C09A
:10B9D000059108B9480F591F059108B90000FA01EF
:10B9E000059108B94D91059108B95D91059108B986
:10B9F00000C0059108B900C0059108B9480F591F4A
:10BA0000059108B90000FA01059108B94D91059119
:10BA100008B95D91059108B900C0059108B900C049
:10BA2000059108B9480F591F059108B90000FA019E
:10BA3000059108B94D91059108B95D91059108B935
:10BA400000C0059108B900C0059108B9480F591FF9
:10BA5000059108B90000FA01059108B94D910591C9
:10BA600008B95D91059108B900C0059108B900C0F9
:10BA7000059108B9480F591F059108B90000FA014E
:10BA8000059108B94D91059108B95D91059108B9E5
:10BA900000C0059108B900C0059108B9480F591FA9
:10BAA000059108B90000FA0100000027000008B95C
:10BAB00008E00A95F1F70000000000009F918F91C7
:10BAC000089528980E942752E7E1EA95F1F7289A0D
:10BAD00010D1E0E0F6E0F3D0E0FF4ED0E0FF02C08E
:10BAE0000E9447510895129A0C94765D0C94785DEB
:10BAF000129844275527662777278CE00C94805DA1
:10BB00000C94825D0C94845D0C94865D0C94885D2D
:10BB10000C948A5D440F551F00994160660F771F92
:10BB200001996160139A0C94955D0C94975D13983C
:10BB30000C949A5D0C949C5D0C949E5D0C94A05D9D
:10BB40008A9541F740955095609570955F707F702C
:10BB500040932A0C50932B0C60932C0C70932D0C5B
:10BB60009BE04830590711F40E94E14B6830790797
:10BB700011F40E94E14B0895EF93E091210CE93E0E
:10BB8000E0F5E930D0F12F923F924F925F926F92A1
:10BB90007F928F929F92AF92BF92CF92DF92EF925D
:10BBA000FF920F931F932F933F934F935F936F9346
:10BBB0007F938F939F93AF93BF93CF93DF930E9415
:10BBC000E259DF91CF91BF91AF919F918F917F917A
:10BBD0006F915F914F913F912F911F910F91FF9026
:10BBE000EF90DF90CF90BF90AF909F908F907F901D
:10BBF0006F905F904F903F902F90EF910895FF933B
:10BC0000EF93EFB7EF93E0918400EE50E13000F056
:10BC1000E23000F0E33000F0E43000F0E53000F016
:10BC2000E63000F0E73000F0E83000F0E93000F0F6
:10BC300005D0EF91EFBFEF91FF9118950F921F92F2
:10BC4000ECEBF3EB0090200C000C1124E00DF11D47
:10BC500005901490F00109951F900F900895289871
:10BC60000E942752E5E1EA95F1F7E091210CEA956F
:10BC7000E093210C289A00000000089528980E9463
:10BC80005052289A0000E1E0F6E019D02BD0089538
:10BC900028980E945052E0EB0000EA95E9F7000076
:10BCA0000000289AF6E0E2E00AD0089528980E9461
:10BCB0005052289A0000E3E0FDEF01D00895009073
:10BCC000210C0A9410905F0011FC0F2E0092210CA1
:10BCD0000090200C11FC0E2E0092200CE0E011FCD4
:10BCE000E1E00895E3E0E0938900EDE8E093880067
:10BCF0000895E7E0E0938900EBE1E0938800089580
:10BD0000E0E6F4E0A0E6B3E06091280C7091290C25
:10BD10006D937D933197E1F7112408950F931F934D
:10BD200080E694E0A0E6B3E0E091260CF091270CC9
:10BD300040E30091240C1091250C65917591649F4E
:10BD40009001749F300D200F311F2D933D9301976B
:10BD5000A1F711241F910F91089599277727332771
:10BD600020E5629F880F080E131EE091260CF091CB
:10BD7000270CE00DF11D45915591A0E6B3E0A00D13
:10BD8000B11D20E3429FB001529F700D4091240CE1
:10BD90005091250C640F751F6D937C9311240895A9
:10BDA0009927552728E2220F629F880F080E191E37
:10BDB000A0E6B3E0A00DB11D6091280C7091290C94
:10BDC00020E3429F600D711D6D937C9311240895B3
:10BDD0009927772728E2220F629F880F080E191EE5
:10BDE000A0E6B3E0A00DB11D6091240C7091250C6C
:10BDF00020E3429F600D711D529F700D6D937C93E7
:10BE0000112408958093260C9093270C0895809315
:10BE1000280C9093290C08958093240C9093250C62
:10BE200008958091220C089511241092220C0895F7
:10BE3000882329F480912A0C90912B0C08958091ED
:10BE40002C0C90912D0C089580E891E08093610076
:10BE500090936100089580E890E080936100909352
:10BE600061000895813081F42091420C3091430C9F
:10BE700086E191E0289FF001299FF00D389FF00D99
:10BE80001124EE53F24F11C0882391F42091420CFB
:10BE90003091430C86E191E0289FF001299FF00D3D
:10BEA000389FF00D1124ED53F24F8DE280830895F9
:10BEB000823089F42091420C3091430C86E191E06C
:10BEC000289FF001299FF00D389FF00D1124EC53AD
:10BED000F24F8DE280830895AF92BF92CF92DF92AE
:10BEE000EF92FF920F931F93CF93DF935C01CA01F0
:10BEF000F6E0880F991FFA95E1F7840F951FFC0172
:10BF0000EE52F64FE491EE2EFF244091420C5091F8
:10BF1000430CEC01CD52D64FE4E0220F331FEA95DB
:10BF2000E1F7C20FD31F00E010E086E191E0489FE7
:10BF30006001499FD00C589FD00C11241DC08491E2
:10BF4000882359F06631710594F537FD30C02A30E9
:10BF500031056CF58C91882351F54F5F5F4F319619
:10BF600011962F5F3F4F4E155F054CF30F5F1F4F2C
:10BF7000CE0DDF1D6F5F7F4F0E151F0514F081E0A2
:10BF800017C0DB01AA0FBB1FCB0123E0880F991F4D
:10BF90002A95E1F7A80FB91FAA0DBB1DAC0DBD1D59
:10BFA000A852B34F9501FE0140E050E0C8CF80E0B9
:10BFB000DF91CF911F910F91FF90EF90DF90CF9085
:10BFC000BF90AF9008959C01FC01B3E0EE0FFF1FFE
:10BFD000BA95E1F7220F331FE20FF31F2091420CB5
:10BFE0003091430C86E191E0AC01249FC001259F74
:10BFF000900D349F900D1124E80FF91FE852F34F74
:10C0000020E030E08081882311F080E008952F5FE8
:10C010003F4F31962A303105A9F781E008959C0100
:10C02000FC0193E0EE0FFF1F9A95E1F7220F331FFB
:10C03000E20FF31F2091420C3091430C86E191E016
:10C04000AC01249FC001259F900D349F900D1124B9
:10C05000E80FF91FE852F34F20E030E08081882399
:10C0600039F02F5F3F4F31962A303105B9F781E023
:10C0700008959C01FC0153E0EE0FFF1F5A95E1F774
:10C08000220F331FE20FF31F2091420C3091430C1B
:10C0900086E191E0AC01249FC001259F900D349F63
:10C0A000900D1124E80FF91FE852F34F80E090E063
:10C0B000619301968A309105D9F708959F92AF92C6
:10C0C000BF92CF92DF92EF92FF920F931F93CF9385
:10C0D000DF93982EA62E6A01790100E010E00BC0D4
:10C0E0006B2D892D8C0F0E94AD5E2196CC15DD0540
:10C0F000BCF30F5F1F4F0E151F052CF4C0E0D0E0FE
:10C10000B02EBA0CF3CFDF91CF911F910F91FF901A
:10C11000EF90DF90CF90BF90AF909F9008952F92B7
:10C120003F924F925F926F927F928F929F92AF92C7
:10C13000BF92CF92DF92EF92FF920F931F93DF9304
:10C14000CF9300D00F92CDB7DEB7382E4801E982E9
:10C150002C2CCA01A6E0880F991FAA95E1F7840F3D
:10C16000951FFC01EE52F64FE491AE2EBB24F3ED89
:10C17000CF2EF9E0DF2EC80ED91EE4E0220F331FC8
:10C18000EA95E1F7C20ED31E7B836A833B016A0CFA
:10C190007B1C66E1462E61E0562E44C0760100E02D
:10C1A00010E0F7018491482F50E04115510559F1F5
:10C1B0002220B9F08091420C9091430C849DF001B3
:10C1C000859DF00D949DF00D1124E155F34F878569
:10C1D000992787FD909501962A813B8182179307C5
:10C1E00094F43981332331F06A81832D800F0E94CA
:10C1F000AD5E09C08114910409F0A4016A81832D08
:10C20000800F0E94E85E0F5F1F4F0894E11CF11C35
:10C210000A151B0534F2CA0CDB1C8A819B8101962E
:10C220009B838A83EA81FB81E615F70509F0B6CF87
:10C230000F900F900F90CF91DF911F910F91FF9072
:10C24000EF90DF90CF90BF90AF909F908F907F90B6
:10C250006F905F904F903F902F900895BF92CF9234
:10C26000DF92EF92FF920F931F93CF93DF93B82E3D
:10C270008091420C9091430C26E131E0829FF001C5
:10C28000839FF00D929FF00D1124E155F34F86A18D
:10C29000882309F456C0818500E010E0E82EFF24D1
:10C2A000E7FCF094B6E1CB2EB1E0DB2EE801CE0D39
:10C2B000DF1D8091420C9091430C8C9DF0018D9D6F
:10C2C000F00D9C9DF00D1124E155F34F2285458121
:10C2D000808530E050E0BE01992787FD90950E944F
:10C2E0006C5F0F5F1F4F882309F72091420C30913C
:10C2F000430C86E191E0289FF001299FF00D389FC3
:10C30000F00D1124E155F34F22854581678577278C
:10C3100067FD7095615070406C0F7D1F8485992773
:10C3200087FD9095E085FF27E7FDF095CC24C39429
:10C33000EB2C03E110E030E050E08E0F9F1F0E94D5
:10C340008F60DF91CF911F910F91FF90EF90DF9061
:10C35000CF90BF9008955F926F927F928F929F923D
:10C36000AF92BF92CF92DF92EF92FF920F931F9303
:10C37000CF93DF93EC012091420C3091430C86E186
:10C3800091E0289FF001299FF00D389FF00D1124B6
:10C39000E155F34F8285833019F4209741F40CC0A6
:10C3A000882329F4C330D10511F4552407C055243E
:10C3B00090E08C179D0714F455245394F6E1AF2EAA
:10C3C000F1E0BF2E2A9DF0012B9DF00D3A9DF00D5E
:10C3D0001124E155F34F808561854581433011F487
:10C3E00081E0A5C1C82EDD24C7FCD094E62EFF2431
:10C3F000E7FCF0949E0150E0B701C6010E946C5F1B
:10C40000882311F04601ECC046010894811C911C60
:10C410008091420C9091430C8A9DF0018B9DF00D10
:10C420009A9DF00D1124E155F34F45819E0150E096
:10C43000B701C4010E946C5F882309F0D1C03601A6
:10C440000894610871088091420C9091430C8A9D78
:10C45000F0018B9DF00D9A9DF00D1124E155F34FE5
:10C4600045819E0150E0B701C3010E946C5F8823A3
:10C4700011F04301B5C08091420C9091430C8701AB
:10C48000015010408A9DF0018B9DF00D9A9DF00D9A
:10C490001124E155F34F2285458130E050E0B80189
:10C4A000C6010E946C5F882339F18091420C909103
:10C4B000430C8A9DF0018B9DF00D9A9DF00D112487
:10C4C000E155F34F45819E0150E0B801C6010E943D
:10C4D0006C5F882389F08091420C9091430C8A9D77
:10C4E000F0018B9DF00D9A9DF00D1124E155F34F55
:10C4F00081E085A3460177C08091420C9091430C66
:10C50000B7016F5F7F4F552009F421C18B01E6E130
:10C510008E2EE1E09E2E889DF001899DF00D989D64
:10C52000F00D1124E155F34F45819E0150E0C30108
:10C530000E946C5F882309F055C087010E5F1F4F72
:10C540008091420C9091430C889DF001899DF00DE3
:10C55000989DF00D1124E155F34F45819E0150E067
:10C56000B801C3010E946C5F8823E1F552E0852E7B
:10C57000912C8C0C9D1C8091420C9091430C06E1F7
:10C5800011E0809FF001819FF00D909FF00D11242C
:10C59000E155F34F45819E0150E0B701C4010E946F
:10C5A0006C5F8823E9F44EEF842E4FEF942E8C0CB1
:10C5B0009D1C8091420C9091430C809FF001819FC3
:10C5C000F00D909FF00D1124E155F34F45819E0130
:10C5D00050E0B701C4010E946C5F882309F4A7C032
:10C5E000870101C043018091420C9091430C26E1E8
:10C5F00031E0829FF001839FF00D929FF00D112496
:10C60000E155F34F85A1882369F038010894611C36
:10C61000711C45819E0150E0B301C4010E946C5F12
:10C62000882309F4380181E00E942E618091420C38
:10C630009091430C36E1A32E31E0B32E8A9DF00198
:10C640008B9DF00D9A9DF00D1124E155F34F22853D
:10C6500045816785772767FD70958185992787FDD7
:10C660009095680F791F8485992787FD9095E085BF
:10C67000FF27E7FDF095CC24C394EE24E39400E07B
:10C6800010E030E050E08E0F9F1F0E948F6080917D
:10C69000420C9091430C8A9DF0018B9DF00D9A9D68
:10C6A000F00D1124E155F34FC2878086618680E04A
:10C6B0000E942E618091420C9091430C8A9DF00162
:10C6C0008B9DF00D9A9DF00D1124E155F34F2285BD
:10C6D00045816785772767FD70958185992787FD57
:10C6E0009095680F791F8485992787FD9095E0853F
:10C6F000FF27E7FDF095EE2430E050E08E0F9F1FFE
:10C700000E948F608091420C9091430C8A9DF001B1
:10C710008B9DF00D9A9DF00D1124E155F34FEE5EC7
:10C72000FE4F81E08083E251F140118A108ADF914F
:10C73000CF911F910F91FF90EF90DF90CF90BF901E
:10C74000AF909F908F907F906F905F9008958B0136
:10C7500026E1622E21E0722E869DF001879DF00D6C
:10C76000969DF00D1124E155F34F45819E0150E057
:10C77000C4010E946C5F882309F035CF87010E5FEA
:10C780001F4F8091420C9091430C869DF001879D34
:10C79000F00D969DF00D1124E155F34F45819E015A
:10C7A00050E0B801C4010E946C5F882309F4DECE1A
:10C7B0001ACFAF92BF92CF92DF92EF92FF920F9378
:10C7C0001F93CF93DF93EC01D62E2091420C309132
:10C7D000430C86E191E0289FF001299FF00D389FDE
:10C7E000F00D1124E155F34F10852285458130E08D
:10C7F00050E0CE010E946C5F882309F491C0FF24B1
:10C80000812F992787FD90958C179D0729F0FF248C
:10C81000F39481E00E942E618091420C9091430C30
:10C82000B6E1AB2EB1E0BB2E8A9DF0018B9DF00DE1
:10C830009A9DF00D1124E155F34F228545816785BE
:10C84000772767FD70958185992787FD9095680FFB
:10C85000791F8485992787FD9095E085FF27E7FD5F
:10C86000F095CC24C394EE24E39400E010E030E093
:10C8700050E08E0F9F1F0E948F608091420C90911C
:10C88000430C8A9DF0018B9DF00D9A9DF00D1124B3
:10C89000E155F34FC087D186FF2019F080E00E9458
:10C8A0002E618091420C9091430CA6E1AA2EA1E04A
:10C8B000BA2E8A9DF0018B9DF00D9A9DF00D1124EA
:10C8C000E155F34F228545816785772767FD709590
:10C8D0008185992787FD9095680F791F8485992711
:10C8E00087FD9095E085FF27E7FDF095CC24C39464
:10C8F000EE2400E010E030E050E08E0F9F1F0E9419
:10C900008F608091420C9091430C8A9DF0018B9D29
:10C91000F00D9A9DF00D1124EF53F24F108281E03B
:10C92000DF91CF911F910F91FF90EF90DF90CF900B
:10C93000BF90AF900895AF92BF92CF92DF92EF92E7
:10C94000FF920F931F93CF93DF932091420C30916E
:10C95000430C86E191E0289FF001299FF00D389F5C
:10C96000F00D1124E155F34F818500E010E0E82E31
:10C97000FF24E7FCF09436E1A32E31E0B32EE8016A
:10C98000CE0DDF1D8091420C9091430C26E1C22E0A
:10C9900021E0D22E8A9DF0018B9DF00D9A9DF00D25
:10C9A0001124E155F34F22854581808530E050E028
:10C9B000BE01992787FD90950E946C5F0F5F1F4F06
:10C9C0008823E9F621978091420C9091430C8C9D2D
:10C9D000F0018D9DF00D9C9DF00D1124E155F34F5C
:10C9E0008085BE01992787FD90950E94D96380912B
:10C9F000420C9091430C8C9DF0018D9DF00D9C9DFF
:10CA0000F00D1124E155F34F108A118A138A81E049
:10CA10008383DF91CF911F910F91FF90EF90DF9073
:10CA2000CF90BF90AF900895CF93DF938091420C49
:10CA30009091430CC6E1D1E08C9FF0018D9FF00DE9
:10CA40009C9FF00D1124E155F34F8089882351F00C
:10CA500081898F5F818B80314CF1108A118A138A12
:10CA600081E025C083898F5F838B92898917F4F0D9
:10CA7000138A6185772767FD70956F5F7F4F80858B
:10CA8000992787FD90950E94D963882379F4809136
:10CA9000420C9091430C8C9FF0018D9FF00D9C9F58
:10CAA000F00D1124E155F34F81E0808B80E0DF91A0
:10CAB000CF9108952F923F924F925F926F927F9203
:10CAC0008F929F92AF92BF92CF92EF92FF920F936D
:10CAD0001F93DF93CF9300D000D0CDB7DEB7809106
:10CAE000420C9091430CF6E1AF2EF1E0BF2E8A9DEF
:10CAF000F0018B9DF00D9A9DF00D1124E155F34F3F
:10CB00008181882321F0813009F051C01CC0228529
:10CB100045816785772767FD70958185992787FD12
:10CB20009095680F791F8485992787FD9095E085FA
:10CB3000FF27E7FDF095CC24C394EE240AE010E033
:10CB400030E050E01CC0458150E08A01045F1F4F77
:10CB500022856785772767FD70958185992787FDF1
:10CB60009095680F791F8485992787FD9095E085BA
:10CB7000FF27E7FDF095CC24C394EE2430E08E0F20
:10CB80009F1F0E948F602091420C3091430C86E1E0
:10CB900091E0289FF001299FF00D389FF00D11249E
:10CBA000E155F34F81818F5F818380E05EC12285F3
:10CBB00045816785772767FD70958185992787FD72
:10CBC0009095680F791F8485992787FD9095E0855A
:10CBD000FF27E7FDF095CC24C394EE2400E010E09D
:10CBE00030E050E08E0F9F1F0E948F600091420C3A
:10CBF0001091430C0A9D90010B9D300D1A9D300D34
:10CC00001124D901A155B34F1596EC91159781E4E4
:10CC1000E89FF0011124EE52F64FC4902C2C3324DF
:10CC200027FC309460E070E01C821B822901E5E063
:10CC30006E2E712C6A0E7B1E51E4F52E4AE0842E76
:10CC4000912C8A0E9B1E38E0A32EB12CAA0EBB1E7F
:10CC50009D01275F3F4F3A83298348C0D301EC9061
:10CC6000EF9CF0011124ED52F64FD4018C9190E02D
:10CC700024E0880F991F2A95E1F72B813C81820FD0
:10CC8000931F840F951FE80FF91FE491EE2309F11C
:10CC9000D5018C91992787FD9095E981FA812081B2
:10CCA000332727FD3095260F371FF901B3E0EE0F2C
:10CCB000FF1FBA95E1F7220F331FE20FF31FE40DB8
:10CCC000F51DE155F34FE40FF51FE80FF91FE3944D
:10CCD000E1A64F5F5F4F4C150CF4C0CF6F5F7F4FE5
:10CCE0002B813C81220D331D3C832B836C151CF45E
:10CCF00040E050E0F0CF86E191E0089FA001099F5D
:10CD0000500D189F500D1124DA01A155B34F5196C3
:10CD10001C92519750961C92509713961C92139701
:10CD200015968C911597843009F09EC0FD01EE5E3A
:10CD3000FE4F8081882309F497C019968C9119972A
:10CD4000282F30E018968C91682F70E0F901EE0FD3
:10CD5000FF1FC901A3E0880F991FAA95E1F7E80F0B
:10CD6000F91FE40FF51FE155F34FE60FF71F81A5FB
:10CD7000811181E0482FDB011296F901EE0FFF1FB0
:10CD8000C90153E0880F991F5A95E1F7E80FF91F81
:10CD900086E191E07C010E9DC0010F9D900D1E9DCE
:10CDA000900D1124E80FF91FE155F34FEA0FFB1F17
:10CDB00081A581114F5F2E5F3F4FF901EE0FFF1FDD
:10CDC000C90153E0880F991F5A95E1F7E80FF91F41
:10CDD00086E191E07C010E9DC0010F9D900D1E9D8E
:10CDE000900D1124E80FF91FE155F34FE60FF71FDF
:10CDF00081A581114F5FF90163E0EE0FFF1F6A9576
:10CE0000E1F7220F331FE20FF31F86E191E09C014F
:10CE1000029FC001039F900D129F900D1124E80FF7
:10CE2000F91FE155F34FEA0FFB1F81A581114F5FF9
:10CE3000433070F086E191E0089FF001099FF00D0A
:10CE4000189FF00D1124E054F24F81E080830DC053
:10CE500086E191E0089FF001099FF00D189FF00D09
:10CE60001124E054F24F108281E00F900F900F9048
:10CE70000F90CF91DF911F910F91FF90EF90CF9086
:10CE8000BF90AF909F908F907F906F905F904F90EA
:10CE90003F902F9008957F928F929F92AF92BF9272
:10CEA000CF92DF92EF92FF920F931F93CF93DF9376
:10CEB000782E862E5A016901780100E010E00CC03E
:10CEC000A701692D872D8C0F0E94E85E2196CA1557
:10CED000DB05B4F30F5F1F4F0C151D052CF4C0E0EC
:10CEE000D0E0902E980CF3CFDF91CF911F910F914E
:10CEF000FF90EF90DF90CF90BF90AF909F908F907A
:10CF00007F9008954F925F926F927F928F929F923F
:10CF1000AF92BF92CF92DF92EF92FF920F931F9347
:10CF2000CF93DF935A01141615060CF089C04C01FB
:10CF3000089481089108840E951E8B0101501040C1
:10CF4000040F151FEE24FF24E6E14E2EE1E05E2ED5
:10CF500065C08091420C9091430C849DA001859DF9
:10CF6000500D949D500D1124D601A40FB51FA1554D
:10CF7000B34FAC0FBD1FC301F30173E0EE0FFF1FF2
:10CF80007A95E1F7880F991FE80FF91FE40FF51F55
:10CF9000E155F34FEC0FFD1F81A599968C93DA01B3
:10CFA000A155B34F1F966C911F97862F992787FD28
:10CFB00090959801280F391F0196821793070CF559
:10CFC000C301F30133E0EE0FFF1F3A95E1F7880F3D
:10CFD000991FE80FF91FE40FF51FE155F34FEC0F10
:10CFE000FD1F41A5600F442331F41C968C918C0FDA
:10CFF0000E94AD5E06C01C968C9150E08C0F0E9482
:10D00000E85E2196CA30D10509F0A3CF0894E11C4F
:10D01000F11CEA14FB04A4F401501040C4018E1961
:10D020009F093C01C0E0D0E06801CC0CDD1CC801C8
:10D03000A3E0880F991FAA95E1F7C80ED91E89CFE2
:10D04000DF91CF911F910F91FF90EF90DF90CF90E4
:10D05000BF90AF909F908F907F906F905F904F9018
:10D0600008950E94E67967E070E00E94027A0895D0
:10D07000AF92BF92CF92DF92EF92FF920F931F93E6
:10D08000CF93DF932091420C3091430C86E191E0E5
:10D09000289FF001299FF00D389FF00D1124E155D4
:10D0A000F34F80A5882309F4D5C000E010E066E1C5
:10D0B000A62E61E0B62E44C08091420C9091430CA4
:10D0C0008A9D90018B9D300D9A9D300D1124F601A3
:10D0D000E20FF31FE155F34FEC0FFD1FD701A20F35
:10D0E000B31FA155B34FAC0FBD1F99968C91999763
:10D0F00081A7F901E155F34F6785862F992787FDB1
:10D1000090959801280F391F0196821793077CF498
:10D1100099964C91600F442329F484858C0F0E94CA
:10D12000AD5E05C0848550E08C0F0E94E85E2196BC
:10D13000CA30D10509F60F5F1F4F05311105D9F02F
:10D1400098012F5F3F4FC0E0D0E06801CC0CDD1CA0
:10D15000C80143E0880F991F4A95E1F7C80ED91E10
:10D16000790183E0EE0CFF1C8A95E1F7220F331F53
:10D17000E20EF31EA1CF0E94E67969E070E00E9402
:10D18000027A8C01C0E0D0E0A6E1EA2EA1E0FA2EFE
:10D19000F8E0DF2E8091420C9091430CC017D1072C
:10D1A000F9F48E9DF0018F9DF00D9E9DF00D1124E0
:10D1B000E155F34F848566858C0F0E94AD5E8091AA
:10D1C000420C9091430C8E9DF0018F9DF00D9E9D21
:10D1D000F00D1124EC0FFD1FE655F24F108220C018
:10D1E0008E9DF0018F9DF00D9E9DF00D1124E15557
:10D1F000F34F848548E050E066858C0F0E94E85E1E
:10D200008091420C9091430C8E9DF0018F9DF00D0A
:10D210009E9DF00D1124EC0FFD1FE655F24FD082BC
:10D220002196CA30D10509F0B5CF8091420C90917A
:10D23000430C26E131E0829FF001839FF00D929F25
:10D24000F00D1124E155F34F80A5815080A788236C
:10D2500079F40CC04091D70C69E181E10E948A58B1
:10D260004091ED0D69E189E10E948A5881E004C096
:10D2700081818F5F818380E0DF91CF911F910F913A
:10D28000FF90EF90DF90CF90BF90AF9008951F93E5
:10D2900080E00E94185F182F8823D1F380E00E945D
:10D2A000185F892BD9F7812F1F910895CF93DF93B2
:10D2B00043E25CE060E170E085E090E00E946E583F
:10D2C00049E25CE061E170E085E090E00E946E5828
:10D2D000C0E0D0E02D9680E00E94185F90FFFACF6A
:10D2E00080E00E94185F90FDFBCF22E030E045E037
:10D2F00050E060E170E085E090E00E945E60CE0169
:10D300000E94EB79DF91CF910895CF92DF92EF9257
:10D31000FF920F931F93CF93DF932091420C309194
:10D32000430C86E191E0289FD001299FB00D389FE2
:10D33000B00D1124A155B34F1596EC91159781E4CA
:10D34000E89FF0011124EE52F64FE491EE2EFF24F7
:10D3500019968C91482F552747FD5095C701840F8A
:10D36000951F47972CF0E6E1EE2EF12CE41AF50A12
:10D370008BE890E0289FF001299FF00D389FF00D79
:10D380001124EE0FFF1FEF54F34F8081082F10E0A0
:10D390000115110509F4C1C186E191E0289FF00152
:10D3A000299FF00D389FF00D1124E155F34F618155
:10D3B000662309F040C0E701219700E010E066E134
:10D3C000C62E61E0D62E33C08091420C9091430C62
:10D3D0008C9D90018D9D300D9C9D300D1124F90187
:10D3E000E155F34F8185A82FBB27A7FDB095CE014E
:10D3F0008A0F9B1FFC0153E0EE0FFF1F5A95E1F7C8
:10D40000880F991FE80FF91FE20FF31FE852F34F3F
:10D4100020E030E08081882339F42F5F3F4F319640
:10D420002A303105B9F7A3C121970F5F1F4F0E15A1
:10D430001F0554F280C1862F90E0081719072CF4BD
:10D4400040E050E0A6E1B1E021C0BC0101970E949C
:10D45000826771C18091420C9091430C8A9FF001C8
:10D460008B9FF00D9A9FF00D1124E60FF71FE155E9
:10D47000F34FE20FF31F11A62F5F3F4F2A30310504
:10D4800049F74F5F5F4F4017510774F420E030E0D9
:10D49000BA01660F771FCA01E3E0880F991FEA956A
:10D4A000E1F7680F791FD6CF41E060EA8AE00E9479
:10D4B0000E502091420C3091430C86E191E0289F60
:10D4C000F001299FF00D389FF00D1124E054F24F28
:10D4D0008081882321F0E801CC0FDD1F52C102308A
:10D4E000110519F4C1E0D0E05EC10330110509F463
:10D4F00058C10430110509F442C1C0E0D0E053C165
:10D50000219690E045968A31910514F089E190E0EA
:10D5100041E06FEF0E940E502091420C3091430C7D
:10D5200086E191E0289FF001299FF00D389FF00DD2
:10D530001124ED53F24F8DE28083FF24F394809108
:10D54000440C882389F08091420C9091430C892BE4
:10D5500031F48091ED0D8C0F8093ED0D05C080911D
:10D56000D70C8C0F8093D70C4091D70C69E181E1E7
:10D570000E948A584091ED0D69E189E10E948A5824
:10D580002091420C3091430C86E191E0289FF001FC
:10D59000299FF00D389FF00D1124E155F34F808D38
:10D5A000918D800F911F918F808F0130110519F49B
:10D5B00044E650E00EC00230110519F44CE251E08F
:10D5C00008C00330110519F040E253E002C044EFF7
:10D5D00051E02091420C3091430C86E191E0289F6C
:10D5E000F001299FF00D389FF00D1124E155F34F04
:10D5F00067A1662339F0CA01880F991F480F591F88
:10D6000055954795FF2071F086E191E0289FF00144
:10D61000299FF00D389FF00D1124E155F34F6F5FF6
:10D6200067A30CC086E191E0289FF001299FF00DCF
:10D63000389FF00D1124E155F34F17A22091420CB1
:10D640003091430C86E191E0289FF001299FF00D75
:10D65000389FF00D1124E155F34F848D258D829F65
:10D66000C00111249C01249FC001259F900D349F6F
:10D67000900D1124AA2797FDA095BA2F24893589EA
:10D6800046895789820F931FA41FB51F848B958BE2
:10D69000A68BB78B80549244AF40B04040F08FE3EC
:10D6A00092E4AFE0B0E0848B958BA68BB78B209192
:10D6B000420C3091430C86E191E0289FF001299FB4
:10D6C000F00D389FF00D1124E155F34F208D318D71
:10D6D000828D938D82179307E0F48289181614F4D3
:10D6E0008150828B2091420C3091430C86E191E075
:10D6F000289FF001299FF00D389FF00D1124E1556E
:10D70000F34F858D8F5F858F828D938D0A96938FD2
:10D71000828F2091420C3091430C86E191E0289F4A
:10D72000F001299FF00D389FF00D1124E054F24FC5
:10D73000108281E013C02091420C3091430C86E1AD
:10D7400091E0289FF001299FF00D389FF00D1124E2
:10D75000E155F34F81818F5F818380E0DF91CF912D
:10D760001F910F91FF90EF90DF90CF900895BD0132
:10D770006F5F7F4FAE01CD010E94826756CEC4E03D
:10D78000D0E086E191E0289FF001299FF00D389FBD
:10D79000F00D1124E155F34F87A1882309F0B0CE95
:10D7A000CCCEC2E0D0E0FF24CACEAF92BF92CF92DF
:10D7B000DF92EF92FF920F931F93CF93DF936091CD
:10D7C000420C7091430C86E191E0689FD001699F03
:10D7D000B00D789FB00D1124A155B34F1596EC9163
:10D7E000159781E4E89FF0011124EE52F64F249141
:10D7F00019963C91832F992787FD9095820F911D53
:10D80000479714F4D22E03C046E1D42ED31A86E1F2
:10D8100091E0689FA001699F500D789F500D1124E1
:10D82000FA01E155F34F2181222339F02D3008F41C
:10D8300089C060E0EF0129963BC18BE890E0689FCA
:10D84000F001699FF00D789FF00D1124EE0FFF1F7E
:10D85000EF54F34F1082FF24C6E1D1E09BE8A92EDC
:10D86000B12C2DC04C9F90014D9F300D5C9F300D11
:10D870001124F901E155F34F8185682F772767FD62
:10D8800070956F0D711DFB01EE0FFF1FCB0103E0C3
:10D89000880F991F0A95E1F7E80FF91FE20FF31FB0
:10D8A000E852F34F20E030E08081882339F02F5F89
:10D8B0003F4F31962A303105B9F71DC1F39440919D
:10D8C000420C5091430CFD1468F286E191E0489FB0
:10D8D000D001499FB00D589FB00D1124A155B34FF1
:10D8E000AF5EBE4F8C91A151B140882349F0FD013C
:10D8F000ED5EFE4F8DE2808341E06FEF83E118C063
:10D900008BE890E0489FF001499FF00D589FF00D83
:10D910001124EE0FFF1FEF54F34FE081E43059F470
:10D92000FD01EB5EFE4F8DE2808341E06FEF84E10D
:10D930000E940E50C0C0EE2309F4D1C041E060EC5B
:10D9400082E1F6CF8BE890E0689FF001699FF00DCF
:10D95000789FF00D1124EE0FFF1FEF54F34F8081DD
:10D96000843018F5273028F4243030F4213068F062
:10D9700006C0293050F406C0E8E1FE2E08C056E18A
:10D98000F52E05C04AE1F42E02C03CE1F32E86E1FB
:10D9900091E0689FF001699FF00D789FF00D1124D0
:10D9A000E155F34F2F5F218304C0F22EF69486E1F8
:10D9B000F80EEE24C6E1D1E098E0C92ECF0C4CC0A1
:10D9C0004091420C5091430C4C9F90014D9F300D63
:10D9D0005C9F300D1124F901E155F34F8185682FCB
:10D9E000772767FD70956E0D711DFB01EE0FFF1F10
:10D9F000CB0103E0880F991F0A95E1F7E80FF91FA3
:10DA0000E20FF31FE852F34F20E030E080818823DB
:10DA100011F12F5F3F4F31962A303105B9F799C088
:10DA20000C2D4C9FF0014D9FF00D5C9FF00D1124CB
:10DA3000E155F34F8785992787FD9095680F791FEA
:10DA4000848510E021E030E04AE050E0992787FD2E
:10DA500090950E944B67E394ED1408F4B1CF2BC06E
:10DA60008881992787FD9095860F911DFC0113E011
:10DA7000EE0FFF1F1A95E1F7880F991FE80FF91FA6
:10DA8000E40FF51FE852F34FDF0120E030E08C9106
:10DA9000882369F02F5F3F4F11962A303105B9F77F
:10DAA00080E090E0119201968A309105D9F76F5F7E
:10DAB0006D15B0F214C02091420C3091430C86E1F8
:10DAC00091E0289FF001299FF00D389FF00D11245F
:10DAD000E155F34F81818F5F818380E001C081E058
:10DAE000DF91CF911F910F91FF90EF90DF90CF903A
:10DAF000BF90AF9008954C9FF0014D9FF00D5C9F3B
:10DB0000F00D1124E155F34F8785992787FD9095F6
:10DB1000680F791F84850AE010E021E030E04AE0D8
:10DB200050E0992787FD90950E944B678091420CA9
:10DB30009091430C8A9DF0018B9DF00D9A9DF00D04
:10DB40001124EE0FFF1FEF54F34F80818F5F80830E
:10DB5000B5CE683071050CF463CF0F2D62CFDF9224
:10DB6000EF92FF920F931F93CF93DF938091BB0CA3
:10DB700062E0D62ED80E6091BE0C772767FD7095B7
:10DB80006E5F7F4F24E130E04AE050E0992787FD47
:10DB900090950E945E606091D40D772767FD709527
:10DBA0006E5F7F4F8091D10D24E130E04AE050E07C
:10DBB000992787FD90950E945E600D2D10E00F5F04
:10DBC0001F4F44E55CE06FE070E0C8010E946E58B2
:10DBD0004FE45CE060E170E0C8010E946E584BE0E9
:10DBE00050E06FE08D2D0E94E85E00E080E00E9432
:10DBF000185FEC0190FF11C080E00E94185F892B34
:10DC0000D9F780E0002309F481E0DF91CF911F91E3
:10DC10000F91FF90EF90DF90089550E8E52EF12CE2
:10DC2000E822F92287FD04C080749270892BF1F2FA
:10DC3000602F615F8D2D0E94AD5E41E060E981E063
:10DC40000E940E50EF2831F0002311F401E00BC0C8
:10DC5000015009C0C074D270CD2B29F0013011F4ED
:10DC600000E001C00F5F602F615F4BE050E08D2D41
:10DC70000E94E85E80E00E94185F892BD9F7B6CF3A
:10DC8000882319F0813051F405C08CE592E10E949F
:10DC9000AA4C08958EE69CE00E94AA4C08950E942A
:10DCA000D84C80E00E94185F90FDFBCF80E00E947E
:10DCB000185F90FFFBCF80E00E94185F90FDFBCFC4
:10DCC0000E94F74C08950F931F93CF93DF93082F73
:10DCD000C82FD0E086E191E0C89FF001C99FF00D08
:10DCE000D89FF00D1124ED53F24FE081EE23D1F1D6
:10DCF000002311F086E101C08FE0E43001F1E5304E
:10DD000038F4E230B1F0E330B8F4E130E9F407C0C0
:10DD1000E63291F0E83269F0E432B1F410C023E069
:10DD200030E045E050E060E170E090E00E945E602D
:10DD30000BC045EF51E905C043ED51E902C041EB8D
:10DD400051E960E10E947A5986E191E0C89FF001B3
:10DD5000C99FF00DD89FF00D1124ED53F24F808133
:10DD60008150808386E191E0C89FF001C99FF00D4A
:10DD7000D89FF00D1124EE53F24FE081EE2309F409
:10DD800074C0002311F085E101C08EE0E530A1F1FF
:10DD9000E63070F4E23031F1E33020F4E13009F0A4
:10DDA00056C016C0E33009F1E43009F050C021C07C
:10DDB000EB32F9F0EC3230F4E93209F1EA3209F0F1
:10DDC00046C01AC0EC3289F0ED3209F040C00AC0FA
:10DDD00024E030E047E050E063E170E090E00E9432
:10DDE0005E6035C045EF50E902C049EB50E963E1A0
:10DDF0002CC04DE750E9FBCF41E450E9F8CF182F94
:10DE00001F5F49E751E964E1812F0E947A598BE84D
:10DE100090E0C89FF001C99FF00DD89FF00D11242C
:10DE2000EE0FFF1FEF54F34FE081E13019F447E8A4
:10DE300051E909C0E23019F445E951E904C0E33081
:10DE400031F443EA51E965E1812F0E947A5986E174
:10DE500091E0C89FF001C99FF00DD89FF00D1124EB
:10DE6000EE53F24F80818150808386E191E0C89F1C
:10DE7000F001C99FF00DD89FF00D1124EC53F24F23
:10DE8000E081EE2309F466C0002311F085E101C0B2
:10DE90008EE0E53069F1E63060F4E23001F1E33024
:10DEA00018F4E13049F511C0E330E1F0E43021F538
:10DEB0001CC0EB32D1F0EC3218F4EA32E9F418C0AD
:10DEC000EC3281F0ED32C1F40AC024E030E047E0EA
:10DED00050E063E170E090E00E945E602DC045EF8D
:10DEE00050E908C049EB50E905C04DE750E902C0D0
:10DEF00041E450E963E11EC0F0E0E770F070F59591
:10DF0000E795E130F10591F0E230F1051CF4EF2BDB
:10DF100039F012C0E230F10531F0339769F406C0F0
:10DF200041E351E905C041E651E902C049E451E944
:10DF300064E18F5F0E947A5986E191E0C89FF00109
:10DF4000C99FF00DD89FF00D1124EC53F24F808142
:10DF500081508083DF91CF911F910F9108950F938E
:10DF60001F93CF93DF938C01C0E0D0E00DC00E94DF
:10DF7000115F8823E1F30E94145F80E00E94636ECA
:10DF800081E00E94636E2196C017D10784F3DF9170
:10DF9000CF911F910F9108953F924F925F926F9290
:10DFA0007F928F929F92AF92BF92CF92DF92EF9229
:10DFB000FF920F931F93CF93DF932091420C3091E8
:10DFC000430C41E0A22EA42686E191E0289FF001B7
:10DFD000299FF00D389FF00D1124E155F34F468F26
:10DFE0000E94D84C41E06FEF85E10E940E5089E11C
:10DFF00090E00E94AF6F8EE494E20E94AA4CC0E0D1
:10E00000D0E076E1872E71E0972E8A2D90E09C017A
:10E01000289DC001299D900D389D900D112481559A
:10E02000934F6FE0462E512C480E591E5CE0652E32
:10E03000712C680E791EA0C03CE13C1510F40DE176
:10E0400001C00C2DEB2CFF24CE018E199F098431C9
:10E0500091050CF084C00D3109F446C0069714F008
:10E06000D02E03C048E0D42ED00E8091420C909167
:10E07000430C889DF001899DF00D989DF00D1124B1
:10E08000E155F34F6785772767FD70956E5F7F4F8A
:10E090006C0F7D1F6E197F0984850D2D10E021E026
:10E0A00030E04AE050E0992787FD90950E9443595F
:10E0B0008091440C882309F452C0F20160817727D3
:10E0C00067FD70956E5F7F4F6C0F7D1F6E197F0926
:10E0D000F301808121E030E04AE050E0992787FD9C
:10E0E00090950E9443593BC08091420C9091430C03
:10E0F000889DF001899DF00D989DF00D1124E1554A
:10E10000F34F6785772767FD70956E5F7F4F6C0FC4
:10E110007D1F6E197F09848521E030E04AE050E0E0
:10E12000992787FD90950E945E608091440C88231A
:10E13000B1F0F2016081772767FD70956E5F7F4FC8
:10E140006C0F7D1F6E197F09F301808121E030E0A3
:10E150004AE050E0992787FD90950E945E60B39455
:10E16000C3943B1408F068CF81E090E00E94AF6F49
:10E170002196CB31D10529F03C2EBB2436E1C32EAC
:10E180005BCF00E010E0C6E1D1E08A2D90E09C0179
:10E190002C9FC0012D9F900D3C9F900D1124815507
:10E1A000934F2FE0822E912C880E991EBCE0CB2E2F
:10E1B000D12CC80ED91E8091440C8823E9F5002388
:10E1C000F9F08091420C9091430C8C9FF0018D9F4F
:10E1D000F00D9C9FF00D1124E155F34F67857727D3
:10E1E00067FD70956F5F7F4F600F711F848521E021
:10E1F00030E04AE050E0992787FD90950E945E60EC
:10E200008091420C9091430C8C9FF0018D9FF00DFA
:10E210009C9FF00D1124E155F34F6785772767FD2B
:10E2200070956E5F7F4F600F711F848544E05CE0E6
:10E23000992787FD909566C0F02E0023F9F0809114
:10E24000420C9091430C8C9FF0018D9FF00D9C9F90
:10E25000F00D1124E155F34F6785772767FD709521
:10E260006F5F7F4F600F711F848521E030E04AE0CF
:10E2700050E0992787FD90950E945E608091420C46
:10E280009091430C8C9FF0018D9FF00D9C9FF00DA1
:10E290001124E155F34F6785772767FD70956E5F11
:10E2A0007F4F600F711F848548E15CE0992787FDEF
:10E2B00090950E946E58FF20A1F0F40160817727AD
:10E2C00067FD70956F5F7F4F600F711FF601808152
:10E2D00021E030E04AE050E0992787FD90950E94C8
:10E2E0005E60F4016081772767FD70956E5F7F4FF8
:10E2F000600F711FF6018081992787FD90954FE08F
:10E300005CE001960E946E5881E090E00E94AF6F41
:10E310000F5F1F4F0A30110509F04DCF8091440C5B
:10E320002091420C3091430C882309F586E191E05D
:10E33000289FF001299FF00D389FF00D1124E15521
:10E34000F34F6785772767FD7095655F7F4F8485FD
:10E3500044E05CE0992787FD90950E946E5882E02A
:10E3600090E00E94AF6F80E00E94185F48C006E115
:10E3700011E0209FF001219FF00D309FF00D11243E
:10E38000E155F34F6785772767FD7095655F7F4F90
:10E39000848548E15CE0992787FD90950E946E583E
:10E3A0008A2D90E0809F7001819FF00C909FF00C6F
:10E3B00011242FEA3CE0E20EF31EF7016785772770
:10E3C00067FD7095665F7F4F84850AE110E023E06A
:10E3D00030E04AE050E0992787FD90950E9443592C
:10E3E000F7016785772767FD7095655F7F4F8485A7
:10E3F000992787FD90954FE05CE00196AECF80E0D5
:10E400000E94185F892BD9F7DF91CF911F910F914F
:10E41000FF90EF90DF90CF90BF90AF909F908F9044
:10E420007F906F905F904F903F900895AF92BF9212
:10E43000CF92EF92FF920F931F93CF93DF93AC0194
:10E440008FEF4F3F580711F0EA017DC02091420C39
:10E450003091430C86E191E0289FF001299FF00D57
:10E46000389FF00D1124E155F34FDF01A05FBE4F3F
:10E470006C91673009F05EC00E943168F82E0E94EE
:10E480003168A82E8F15D9F30E943168C82E8A15DD
:10E49000D9F38F15C9F30E943168E82E8C15D9F392
:10E4A0008A15C9F38F15B9F30E943168082F8E15AC
:10E4B000D9F38C15C9F38A15B9F38F15A9F30E9406
:10E4C0003168182F8017D9F38E15C9F38C15B9F35D
:10E4D0008A15A9F38F1599F30E943168482F811787
:10E4E000D9F38017C9F38E15B9F38C15A9F38A15E2
:10E4F00099F38F1589F32091420C3091430C86E1FA
:10E5000091E0289FF001299FF00D389FF00D112414
:10E51000E155F34FE75FFE4FF192A192C192E19274
:10E52000019311934193CF2DDD27C7FDD09581E055
:10E53000808309C0E60FF11DE75FFE4F8081C82F81
:10E54000D0E06F5F6C938091420C9091430CE6E1B8
:10E55000AE2EE1E0BE2E8A9DF0018B9DF00D9A9DBE
:10E56000F00D1124E155F34F4481552747FD509597
:10E57000EA5FFE4F6081CC24EE24E39400E010E0DB
:10E5800020E030E070E0829190E00E948F60809106
:10E59000420C9091430C8A9DF0018B9DF00D9A9D49
:10E5A000F00D1124E155F34FEA5FFE4F6081EE2438
:10E5B00020E030E0AE0170E0829190E00E948F6038
:10E5C0008091420C9091430C8A9DF0018B9DF00D3F
:10E5D0009A9DF00D1124E155F34F84818583C48306
:10E5E00083E080871186128615A281E0878F60E024
:10E5F00070E083E090E00E94D963882311F40E94C8
:10E60000CC6FDF91CF911F910F91FF90EF90CF9042
:10E61000BF90AF900895CF92DF92EF92FF920F9349
:10E620001F93CF93DF93509100018EE1A82FA51B7C
:10E6300040910101841BEFEAFCE020E030E099E129
:10E64000C92E04E0D02E6AE070E001E093E0BFEF55
:10E6500017E0E12E1DE0FF246894F1F82115310543
:10E6600029F45093CC0CA093C10C04C04093E20D4C
:10E670008093D70D138A118A108AC686D786168E84
:10E6800011A210A212A213A215A2118E108E738FC6
:10E69000628F148A158A168A178A048F90871186CA
:10E6A0001286B6831482078FB387E05FFE4FE08245
:10E6B0003A9710833296F082E850F14010A617A2E4
:10E6C000EF5EFE4F108232961082329611922F5FCB
:10E6D0003F4F2230310511F69093BB0C1093BC0CC8
:10E6E0008FE08093B40D9093B60D8DE18093D10DA2
:10E6F00087E28093D20D87E18093CA0E83E28093F4
:10E70000CC0E20E030E00FC01082EA5EFE4F108297
:10E710000196E551F1408A309105B1F72F5F3F4FE7
:10E720002631310581F0F901EE0FFF1FC901A3E089
:10E73000880F991FAA95E1F7E80FF91FE852F34FE8
:10E7400080E090E0E1CF1092430C1092420C8FEFEA
:10E750009FEF0E9416728091420C9091430CC6E18B
:10E76000D1E08C9FF0018D9FF00D9C9FF00D112446
:10E77000E155F34F848185838FEF9FEF0E941672DE
:10E780000E94856980E00E942E618091440C88235C
:10E7900011F181E090E09093430C8093420C8FEF55
:10E7A0009FEF0E9416728091420C9091430C8C9FB7
:10E7B000F0018D9FF00D9C9FF00D1124E155F34F5A
:10E7C000848185838FEF9FEF0E9416720E94856976
:10E7D00080E00E942E61DF91CF911F910F91FF90F9
:10E7E000EF90DF90CF900895AF92BF92CF92EF92CB
:10E7F0000F931F93CF93DF938091420C9091430C22
:10E8000026E1A22E21E0B22E8A9DF0018B9DF00D13
:10E810009A9DF00D1124E155F34F878D882309F45B
:10E82000BCC081E00E942E618091420C9091430C0B
:10E830008A9DF0018B9DF00D9A9DF00D1124E155FC
:10E84000F34F228545816785772767FD7095818520
:10E85000992787FD9095680F791F8485992787FDF3
:10E860009095E085FF27E7FDF095CC24C394EE2436
:10E87000E39400E010E030E050E08E0F9F1F0E9414
:10E880008F608091420C9091430C8A9DF0018B9D8A
:10E89000F00D9A9DF00D1124E155F34F4681DF01F3
:10E8A000A85FBE4FEF01C95FDE4F4F3FA1F4458126
:10E8B0004683552747FD50956C91CC24EE2420E0EB
:10E8C00030E070E0888190E00E948F608FEF9FEFD2
:10E8D0000E9416724FC0552747FD50956C91CC246D
:10E8E000EE24E39400E010E020E030E070E0888166
:10E8F00090E00E948F608091420C9091430C8A9D21
:10E90000F0018B9DF00D9A9DF00D1124E155F34F10
:10E910004581E85FFE4F6081EE2420E030E050E06A
:10E9200070E0829190E00E948F608091420C909103
:10E93000430C8A9DF0018B9DF00D9A9DF00D1124E2
:10E94000E155F34F858146814583868383E0808747
:10E950001186128615A2118A108A20E030E050E05C
:10E9600060E070E083E090E00E946C5F882311F427
:10E970000E94CC6F80E00E942E612091420C309169
:10E98000430C86E191E0289FF001299FF00D389F0C
:10E99000F00D1124E155F34F178EDF91CF911F91A8
:10E9A0000F91EF90CF90BF90AF900895EF92FF92AC
:10E9B0000F931F93CF93DF938091420C0E94185FB7
:10E9C0008C0187FF1AC08091420C9091430C26E184
:10E9D00031E0829FF001839FF00D929FF00D112492
:10E9E000E155F34F80A187FD08C004FD06C005FD79
:10E9F00004C011A300A381E084C111FF13C02091C2
:10EA0000420C3091430C86E191E0289FF001299F50
:10EA1000F00D389FF00D1124E155F34F80A191A125
:10EA200091FF14C000FF15C02091420C3091430C9F
:10EA300086E191E0289FF001299FF00D389FF00DAD
:10EA40001124E155F34F80A180FD03C00E94F473AF
:10EA500046C110FF16C02091420C3091430C86E154
:10EA600091E0289FF001299FF00D389FF00D1124AF
:10EA7000E155F34F80A191A190FD03C00E944F6E1C
:10EA80003FC104FF21C08091420C9091430C26E1CC
:10EA900031E0829FF001839FF00D929FF00D1124D1
:10EAA000E155F34F80A184FD03C041E050E00EC06A
:10EAB00082A1843048F020E030E083A1823010F061
:10EAC00021E030E0A90102C040E050E005FF1AC09B
:10EAD0008091420C9091430C26E131E0829FF0013D
:10EAE000839FF00D929FF00D1124E155F34F80A10B
:10EAF00085FF06C082A1843028F083A1823010F007
:10EB00004FEF5FEF30E4E32EF12CE022F12206FF1D
:10EB100016C08091420C9091430C26E131E0829F17
:10EB2000F001839FF00D929FF00D1124E155F34FFA
:10EB300084A1823020F014A261E070E002C060E0A5
:10EB400070E04115510519F461157105A1F180912D
:10EB5000420C9091430CC6E1D1E08C9FF0018D9F57
:10EB6000F00D9C9FF00D1124E155F34F81859927FD
:10EB700087FD9095680F791F8085992787FD90956F
:10EB8000840F951F0E94D9638823A9F08091420CBD
:10EB90009091430C8C9FF0018D9FF00D9C9FF00D88
:10EBA0001124E155F34F118A108A13A241E060E469
:10EBB00085E00E940E50C801807390702091420C35
:10EBC0003091430C892B91F086E191E0289FF00170
:10EBD000299FF00D389FF00D1124E155F34F82A1CC
:10EBE0008F5F82A383A18F5F83A30DC086E191E035
:10EBF000289FF001299FF00D389FF00D1124E15559
:10EC0000F34F12A213A22091420C3091430CEF2833
:10EC100079F086E191E0289FF001299FF00D389F5F
:10EC2000F00D1124E155F34F84A18F5F84A30CC034
:10EC300086E191E0289FF001299FF00D389FF00DAB
:10EC40001124E155F34F14A203FF23C08091420C1D
:10EC50009091430C26E131E0829FF001839FF00DFB
:10EC6000929FF00D1124E155F34F80A183FD11C057
:10EC70008285C82FD0E02196C430D10511F4C0E0C0
:10EC8000D0E041E060E485E00E940E50CE010E9499
:10EC9000AB6113FF24C08091420C9091430C26E19C
:10ECA00031E0829FF001839FF00D929FF00D1124BF
:10ECB000E155F34F80A191A193FD11C08285882376
:10ECC00019F4C3E0D0E003C0C82FD0E0219741E0A1
:10ECD00060E485E00E940E50CE010E94AB6120915D
:10ECE000420C3091430C86E191E0289FF001299F6E
:10ECF000F00D389FF00D1124E155F34F11A300A33F
:10ED000080E0DF91CF911F910F91FF90EF900895D8
:10ED10001F93CF93DF938091420C9091430CC6E1F7
:10ED2000D1E08C9FF0018D9FF00D9C9FF00D112480
:10ED3000E155F34F1081143009F44AC0153040F406
:10ED40001130E1F0113070F0133009F089C02BC0A0
:10ED5000163009F466C0163008F44FC0173009F0B9
:10ED60007FC068C00E941465882309F065C00E94B6
:10ED7000D674813009F074C017E072C00E945A65E1
:10ED8000882309F46DC08091420C9091430C8C9FB4
:10ED9000F0018D9FF00D9C9FF00D1124E155F34F74
:10EDA000118213E05DC00E94D56B882309F458C01E
:10EDB0008091420C9091430C8C9FF0018D9FF00D3F
:10EDC0009C9FF00D1124E155F34F118214E048C0CF
:10EDD0000E948569882309F443C08091420C909178
:10EDE000430C8C9FF0018D9FF00D9C9FF00D112422
:10EDF000E155F34F118215E033C00E943868882333
:10EE000079F18091420C9091430C8C9FF0018D9F81
:10EE1000F00D9C9FF00D1124E155F34F118216E087
:10EE20001FC08FEF9FEF0E94167280E00E942E613C
:10EE300010E016C00E949B6441E060E984E00E94FB
:10EE40000E508091420C9091430C8C9FF0018D9F4D
:10EE5000F00D9C9FF00D1124E155F34F118211E04C
:10EE60002091420C3091430C86E191E0289FF00103
:10EE7000299FF00D389FF00D1124E155F34F1083B9
:10EE8000DF91CF911F910895CF93DF93C1E0D0E040
:10EE90000E948E5E0E940B7348E050E069E18FE0B3
:10EEA0000E94E85E44E150E069E180E10E94E85E92
:10EEB00040E069E181E10E948A5848E050E069E160
:10EEC00087E10E94E85E44E150E069E188E10E9448
:10EED000E85E40E069E189E10E948A588091450C32
:10EEE0000E94406E1092AF0C1092C50D1CC00E9483
:10EEF000115F8823C1F00E94145F1092430C10929E
:10EF0000420C0E94887680E00E94636E8091440CDF
:10EF1000882349F0D093430CC093420C0E9488761A
:10EF200081E00E94636E8091CD0C882321F4809152
:10EF3000E30D8823E1F20E94AF6D882309F0A8CF8A
:10EF4000DF91CF910895EF92FF920F931F930E944C
:10EF5000805E4FE25CE068E070E08FE090E00E944D
:10EF60006E584CE35CE06DE070E08CE090E00E9455
:10EF70006E584091450C6DE082E10E948A5849E547
:10EF80005CE06EE070E08CE090E00E946E58809152
:10EF9000D50C882319F046E65CE002C04AE65CE046
:10EFA0006EE070E089E190E00E946E5842E45CE01F
:10EFB0006FE070E08CE090E00E946E584BE050E013
:10EFC0006DE08BE00E94E85E10E0EE2480E00E949D
:10EFD000185FF82E082F83FF1DC080E00E94185F85
:10EFE000892BD9F7112369F4EE2021F00E94D84C27
:10EFF000EE2410C08091450C0E94406EEE24E394F4
:10F0000009C0123039F40E94D84C1F910F91FF9023
:10F01000EF90089505FF3CC0112389F44091450C01
:10F02000442389F141504093450C6DE082E10E94F8
:10F030008A5841E060E981E00E940E5024C01130FE
:10F0400011F541E060E981E00E940E508091D50CFD
:10F05000882369F04AE65CE06EE070E089E190E0C8
:10F060000E946E581092D50C1092EB0D0CC046E623
:10F070005CE06EE070E089E190E00E946E581093D1
:10F08000D50C1093EB0D80E00E94185F892BD9F707
:10F0900004FF3CC0112389F44091450C433088F5AE
:10F0A0004F5F4093450C6DE082E10E948A5841E039
:10F0B00060E981E00E940E5024C0113011F541E05A
:10F0C00060E981E00E940E508091D50C882369F0A0
:10F0D0004AE65CE06EE070E089E190E00E946E58E4
:10F0E0001092D50C1092EB0D0CC046E65CE06EE081
:10F0F00070E089E190E00E946E581093D50C109357
:10F10000EB0D80E00E94185F892BD9F7F7FC02C055
:10F1100006FF5CCF612F635F40E050E08BE00E9410
:10F12000E85E41E060E981E00E940E50F7FE06C013
:10F13000112311F412E009C0115007C006FF05C0E9
:10F14000123011F410E001C01F5F612F635F4BE0CC
:10F1500050E08BE00E94E85E80E00E94185F892BFF
:10F16000D9F734CF0E94805E43EE5BE06FE070E041
:10F1700080E190E00E946E584CEE5BE060E170E050
:10F1800080E190E00E946E5845EF5BE061E170E045
:10F1900080E190E00E946E584CEF5BE062E170E02D
:10F1A00080E190E00E946E584CE566E170E08BE0F3
:10F1B00090E00E946A5849E95BE066E170E08DE00A
:10F1C00090E00E946E5849EC5BE067E170E088E0F7
:10F1D00090E00E946E584BEA5BE069E170E086E0E7
:10F1E00090E00E946E584BEE5DE863E084E00E9480
:10F1F0007A590895CF92DF92EF92FF920F931F9367
:10F20000CF93DF9383EA95E90E94904C81E080934D
:10F21000D50C8093EB0D87E295E20E94075F87ECA7
:10F2200090E30E940C5F8BE295E80E94025F0E94CF
:10F23000B2784BE050E06FE08FE00E94E85ECC24B3
:10F24000DD2410E001E08DE090E0C80ED91E80E0E2
:10F250000E94185FEC0188709170892B09F180E0A1
:10F260000E94185F892BD9F7C6010E94EB79112300
:10F2700019F41092440C06C0812F8150823028F47A
:10F280000093440C0E94447702C00E94A3770E941E
:10F29000B278612F615F4BE050E08FE00E94E85E42
:10F2A000C5FF05C080E00E94185F892BD9F7C4FF15
:10F2B00005C080E00E94185F892BD9F740E8E42E52
:10F2C000F12CEC22FD22C7FD06C0CE0180749270A5
:10F2D000892B09F4B8CF612F615F40E050E08FE0E7
:10F2E0000E94E85E41E060E981E00E940E50EF2854
:10F2F00031F0112311F413E00BC0115009C0C07498
:10F30000D270CD2B29F0133011F410E001C01F5F33
:10F31000612F615F4BE050E08FE00E94E85E80E08B
:10F320000E94185F892BD9F78ECFA0E0B0E0EBE9FF
:10F33000F9E70C948D7AEC01A880B980CA80DB8053
:10F34000A114B104C104D10441F484E2A82E89EDD2
:10F35000B82E8BE5C82E87E0D82EC601B5012DE169
:10F3600033EF41E050E00E946A7A27EA31E440E05E
:10F3700050E00E944B7A7B018C01C601B5012DE162
:10F3800033EF41E050E00E946A7ACA01B9012CEEE5
:10F3900034EF4FEF5FEF0E944B7A6E0D7F1D801FA1
:10F3A000911F97FF04C0615070408040904868836F
:10F3B00079838A839B839B013F77C901CDB7DEB7F1
:10F3C000EAE00C94A97A0E949579089583E091E08F
:10F3D0000E9495790895A0E0B0E080930301909396
:10F3E0000401A0930501B09306010895991B79E0EB
:10F3F00004C0991F961708F0961B881F7A95C9F7C5
:10F400008095089597FB092E07260AD077FD04D032
:10F410002ED006D000201AF4709561957F4F089584
:10F42000F6F7909581959F4F0895A1E21A2EAA1B99
:10F43000BB1BFD010DC0AA1FBB1FEE1FFF1FA217A4
:10F44000B307E407F50720F0A21BB30BE40BF50BA1
:10F45000661F771F881F991F1A9469F7609570952A
:10F46000809590959B01AC01BD01CF010895AA1B29
:10F47000BB1B51E107C0AA1FBB1FA617B70710F09F
:10F48000A61BB70B881F991F5A95A9F780959095D1
:10F49000BC01CD010895629FD001739FF001829F4E
:10F4A000E00DF11D649FE00DF11D929FF00D839F13
:10F4B000F00D749FF00D659FF00D9927729FB00DB0
:10F4C000E11DF91F639FB00DE11DF91FBD01CF01C3
:10F4D0001124089597FB092E05260ED057FD04D060
:10F4E000A4DF0AD0001C38F4509540953095219542
:10F4F0003F4F4F4F5F4F0895F6F790958095709569
:10F5000061957F4F8F4F9F4F08952F923F924F925B
:10F510005F926F927F928F929F92AF92BF92CF92A3
:10F52000DF92EF92FF920F931F93CF93DF93CDB7AC
:10F53000DEB7CA1BDB0B0FB6F894DEBF0FBECDBF24
:10F5400009942A88398848885F846E847D848C84F5
:10F550009B84AA84B984C884DF80EE80FD800C81FE
:10F560001B81AA81B981CE0FD11D0FB6F894DEBFE1
:0CF570000FBECDBFED010895F894FFCF51
:08F57C0014010201000000006F
:00000001FF
